:020000022000DC
:10600000000004209DBA0200659B02001DB0020042
:10601000659B0200659B0200659B0200000000007A
:10602000000000000000000000000000659B02006E
:10603000659B020000000000659B0200659B02005A
:1060400049B90200659B0200EDBE0200F1BA0200F0
:1060500001BB0200659B020045AE0200659B020089
:10606000659B0200CDBE0200DDBE02006DBA0200DB
:10607000659B0200659B0200659B0200659B020018
:1060800015BF02007DBA0200659B0200659B0200FD
:10609000659B0200659B020029BC0200659B020013
:1060A000659B0200659B0200659B0200659B0200E8
:1060B000659B0200659B02000000000000000000DC
:1060C000659B0200659B0200659B020011BB0200FC
:1060D0008DBA0200659B0200659B02000DBF0200A5
:1060E000FDBE020049BA0200659B020099BB020096
:0860F00000000000659B0200A6
:107000004C600B00CC9A0B004C600B0028A30B00CB
:107010004C600B0030A30B004C600B0038A30B003E
:107020004C600B00E0A40B004C600B00E8A40B00CC
:107030004C600B008CA90B004C600B00A4A90B004A
:107040004C600B0048AA0B004C600B000CB60B0008
:107050004C600B0014B60B004C600B001CB60B0010
:107060004C600B00F4B60B004C600B00FCB60B0040
:107070004C600B0064B80B004C600B006CB80B004C
:107080004C600B0074B80B004C600B008CB80B000C
:107090004C600B0094B80B004C600B0060B90B0007
:1070A0004C600B00F8B90B004C600B0010BA0B00E1
:1070B0004C600B0018BA0B004C600B0020BA0B00A0
:1070C0004C600B0028BA0B004C600B00E4BA0B00BC
:1070D0004C600B00ECBA0B004C600B008CBB0B003F
:1070E0004C600B0094BB0B004C600B0020BC0B00F1
:1070F0004C600B0028BC0B004C600B0030BC0B003C
:107100004C600B0038BC0B004C600B0040BC0B000B
:107110004C600B00DCBC0B004C600B00E4BC0B00B3
:107120004C600B00ECBC0B004C600B00F4BC0B0083
:107130004C600B0078BD0B004C600B0080BD0B0059
:107140004C600B0088BD0B004C600B0048BF0B006F
:107150004C600B0050BF0B004C600B0044C20B0096
:107160004C600B006CC20B004C600B00E4C40B00C5
:107170004C600B00ECC40B004C600B0038C50B00DE
:107180004C600B007CC50B004C600B00E0C50B0095
:107190004C600B00E8C50B004C600B008CC70B006B
:1071A0004C600B00A4C70B004C600B005CC80B00CC
:1071B0004C600B00CCC90B004C600B00D4C90B0019
:1071C0004C600B0008CB0B004C600B0010CB0B008D
:1071D0004C600B009CCB0B004C600B00B0CC0B0048
:1071E0004C600B00B8CC0B004C600B00ACCD0B001E
:1071F0004C600B00C4CD0B004C600B00E8D90B00B9
:107200004C600B0000DA0B004C600B0008DA0B003E
:107210004C600B0000DD0B004C600B00BCDE0B0073
:107220004C600B005CE30B004C600B0064E30B0054
:107230004C600B006CE30B004C600B0028E60B006D
:107240004C600B0030E60B004C600B0038E60B0086
:107250004C600B0008E80B004C600B0010E80B00C2
:107260004C600B0018E80B004C600B0020E80B0092
:107270004C600B0064EA0B004C600B007CEA0B00D6
:107280004C600B0084EA0B004C600B008CEA0B0096
:107290004C600B0094EA0B004C600B0030EB0B00D1
:1072A0004C600B0058ED0B004C600B0070ED0B00B8
:1072B0004C600B0078ED0B004C600B007CEF0B007A
:1072C0004C600B0084EF0B004C600B008CEF0B004C
:1072D0004C600B0094EF0B004C600B00A4EF0B0014
:1072E0004C600B00ACEF0B004C600B00B4EF0B00DC
:1072F0004C600B00BCEF0B004C600B0044F00B002B
:107300004C600B0054F20B004C600B005CF20B0065
:107310004C600B0064F20B004C600B006CF20B0035
:107320004C600B00D8F20B004C600B001CF50B00FE
:107330004C600B0024F50B004C600B0094F60B0026
:107340004C600B0064F90B004C600B006CF90B00F7
:107350004C600B0074F90B004C600B007CF90B00C7
:107360004C600B0084F90B004C600B008CF90B0097
:107370004C600B0080000C004C600B0088000C007F
:107380004C600B0000040C004C600B0008040C0067
:107390004C600B00BC090C004C600B00C4090C00D5
:1073A0004C600B00CC090C004C600B00D4090C00A5
:1073B0004C600B00DC090C004C600B001C0D0C0039
:1073C0004C600B00740E0C004C600B007C0E0C002B
:1073D0004C600B00E40E0C004C600B00900F0C0096
:1073E0004C600B00B4110C004C600B00C8140C0076
:1073F0004C600B00D8140C004C600B0048170C00BC
:107400004C600B0050170C004C600B00EC170C008C
:107410004C600B00F4170C004C600B00FC170C00C8
:107420004C600B0004180C004C600B00A0190C0001
:107430004C600B00A8190C004C600B00C49A0B00A8
:10744000BC9A0B004C600B0000A30B00F8A20B00D1
:107450004C600B0010A30B0008A30B004C600B004A
:1074600054B60B004CB60B004C600B0064B60B001E
:107470005CB60B004C600B0074B60B006CB60B00D6
:107480004C600B0084B80B007CB80B004C600B0008
:1074900000BA0B00F0B90B004C600B00DCBA0B001B
:1074A000D4BA0B004C600B0060BF0B0058BF0B0040
:1074B0004C600B0054C20B004CC20B004C600B0024
:1074C00064C20B005CC20B004C600B0094C30B0049
:1074D0008CC30B004C600B000E0000004CC60B0070
:1074E0004C600B00C4C90B00BCC90B004C600B0006
:1074F000ACCB0B00A4CB0B004C600B00BCCB0B0047
:10750000B4CB0B004C600B00CCCB0B00C4CB0B00FE
:107510004C600B00D0CC0B00C8CC0B004C600B00B7
:10752000E0D90B00D8D90B004C600B00F8D90B0048
:10753000F0D90B004C600B0018DA0B0010DA0B00CE
:107540004C600B0028DA0B0020DA0B004C600B00BB
:10755000B4DE0B00ACDE0B004C600B00CCDE0B008D
:10756000C4DE0B004C600B00E4DF0B00DCDF0B0023
:107570004C600B0050E10B0048E10B004C600B002D
:1075800060E10B0058E10B004C600B0070E10B0058
:1075900068E10B004C600B0080E10B0078E10B0010
:1075A0004C600B00E8E30B00E0E30B004C600B00C9
:1075B000ACE50B00A4E50B004C600B00BCE50B0038
:1075C000B4E50B004C600B00CCE50B00C4E50B00F0
:1075D0004C600B00DCE50B00D4E50B004C600B00AD
:1075E000C8E60B00C0E60B004C600B00B8E70B00D0
:1075F000B0E70B004C600B00C8E70B00C0E70B00C6
:107600004C600B00E0E70B00D8E70B004C600B0070
:10761000F0E70B00E8E70B004C600B0000E80B0004
:10762000F8E70B004C600B0030E80B0028E80B007B
:107630004C600B0040E80B0038E80B004C600B007E
:1076400050E80B0048E80B004C600B005CEA0B00B4
:1076500054EA0B004C600B0074EA0B006CEA0B0060
:107660004C600B0044ED0B003CED0B004C600B003C
:1076700068ED0B0060ED0B004C600B0088ED0B001B
:1076800080ED0B004C600B0098ED0B0090ED0B00B3
:107690004C600B00A8FB0B00A0FB0B004C600B0028
:1076A000B8FB0B00B0FB0B004C600B00EC010C00B6
:1076B000E4010C004C600B00FC010C00F4010C0018
:1076C0004C600B0020040C0018040C004C600B00F4
:1076D000D4040C00CC040C004C600B00E4040C003F
:1076E000DC040C004C600B0060050C0058050C001D
:1076F0004C600B0070050C0068050C004C600B0022
:1077000084090C007C090C004C600B0094090C00EF
:107710008C090C004C600B00A4090C009C090C00A7
:107720004C600B00B4090C00AC090C004C600B0061
:10773000600B0C00580B0C004C600B00700B0C0025
:10774000680B0C004C600B00F40C0C00EC0C0C00F3
:107750004C600B00040D0C00FC0C0C004C600B008A
:10776000140D0C000C0D0C004C600B008C0E0C006A
:10777000840E0C004C600B009C0E0C00940E0C0050
:107780004C600B00AC0E0C00A40E0C004C600B0007
:10779000BC0E0C00B40E0C004C600B00CC0E0C00A8
:1077A000C40E0C004C600B00DC0E0C00D40E0C0060
:1077B0004C600B00A00F0C00980F0C004C600B00ED
:1077C000B00F0C00A80F0C004C600B00C00F0C0099
:1077D000B80F0C004C600B00D00F0C00C80F0C0051
:1077E0004C600B00C4110C00BC110C004C600B0071
:1077F0007C120C0074120C004C600B008C120C00FC
:1078000084120C004C600B009C120C0094120C00B3
:107810004C600B00AC120C00A4120C004C600B006E
:10782000BC120C00B4120C004C600B00CC120C000B
:10783000C4120C004C600B00DC120C00D4120C00C3
:107840004C600B00EC120C00E4120C004C600B00BE
:10785000FC120C00F4120C004C600B000C130C001A
:1078600004130C004C600B001C130C0014130C00D0
:107870004C600B002C130C0024130C004C600B000C
:107880003C130C0034130C004C600B004C130C0028
:1078900044130C004C600B00E8140C00E0140C00C6
:1078A0004C600B0098190C0090190C004C600B00F8
:1078B000F81A0C00F01A0C004C600B00081B0C00AE
:1078C000001B0C004C600B00BC1B0C00B41B0C001C
:1078D0004C600B00CC1B0C00C41B0C004C600B005C
:1078E000901C0C00881C0C004C600B00A01C0C00B1
:1078F000981C0C004C600B00B01C0C00A81C0C0069
:107900004C600B00F41C0C00EC1C0C004C600B00D9
:10791000041D0C00FC1C0C004C600B00141D0C0022
:107920000C1D0C004C600B00241D0C001C1D0C00D9
:107930004C600B00341D0C002C1D0C004C600B0027
:10794000641E0C005C1E0C004C600B00741E0C00CE
:107950006C1E0C0040F8044B40F8045B40F8046BCC
:1079600040F8047B40F8048B40F8049B40F804ABDB
:1079700040F804BB40F804CB40F804DB684670478D
:1079800081F0004102E000BF83F0004330B54FEAD0
:1079900041044FEA430594EA050F08BF90EA020F3D
:1079A0001FBF54EA000C55EA020C7FEA645C7FEAD0
:1079B000655C00F0E2804FEA5454D4EB5555B8BFF3
:1079C0006D420CDD2C4480EA020281EA030382EA64
:1079D000000083EA010180EA020281EA0303362DF6
:1079E00088BF30BD11F0004F4FEA01314FF4801CC9
:1079F0004CEA113102D0404261EB410113F0004FDB
:107A00004FEA03334CEA133302D0524263EB430391
:107A100094EA050F00F0A780A4F10104D5F1200E2F
:107A20000DDB02FA0EFC22FA05F2801841F100018A
:107A300003FA0EF2801843FA05F359410EE0A5F15E
:107A400020050EF1200E012A03FA0EFC28BF4CF08F
:107A5000020C43FA05F3C01851EBE37101F0004545
:107A600007D54FF0000EDCF1000C7EEB00006EEB52
:107A70000101B1F5801F1BD3B1F5001F0CD34908DC
:107A80005FEA30004FEA3C0C04F101044FEA445233
:107A900012F5800F80F09A80BCF1004F08BF5FEABA
:107AA000500C50F1000041EB045141EA050130BD9A
:107AB0005FEA4C0C404141EB0101013C28BFB1F5AC
:107AC000801FE9D291F0000F04BF01460020B1FAF7
:107AD00081F308BF2033A3F10B03B3F120020CDACA
:107AE0000C3208DD02F1140CC2F10C0201FA0CF0A8
:107AF00021FA02F10CE002F11402D8BFC2F1200C0D
:107B000001FA02F120FA0CFCDCBF41EA0C019040C2
:107B1000E41AA2BF01EB0451294330BD6FEA04040B
:107B20001F3C1CDA0C340EDC04F11404C4F12002F6
:107B300020FA04F001FA02F340EA030021FA04F308
:107B400045EA030130BDC4F10C04C4F1200220FA5F
:107B500002F001FA04F340EA0300294630BD21FA9D
:107B600004F0294630BD94F0000F83F4801306BF63
:107B700081F480110134013D4EE77FEA645C18BF57
:107B80007FEA655C29D094EA050F08BF90EA020FEE
:107B900005D054EA000C04BF1946104630BD91EAE6
:107BA000030F1EBF0021002030BD5FEA545C05D1E9
:107BB0004000494128BF41F0004130BD14F5800428
:107BC0003CBF01F5801130BD01F0004545F0FE419C
:107BD00041F470014FF0000030BD7FEA645C1ABFD1
:107BE000194610467FEA655C1CBF0B46024650EA08
:107BF000013406BF52EA033591EA030F41F4002134
:107C000030BD00BF90F0000F04BF0021704730B5B9
:107C10004FF4806404F132044FF000054FF000018E
:107C200050E700BF90F0000F04BF0021704730B54F
:107C30004FF4806404F1320410F0004548BF404224
:107C40004FF000013EE700BF42004FEAE2014FEA79
:107C500031014FEA02701FBF12F07F4393F07F4F54
:107C600081F06051704732F07F4208BF704793F057
:107C70007F4F04BF41F40021704730B54FF460746A
:107C800001F0004521F000411CE700BF50EA01026D
:107C900008BF704730B54FF000050AE050EA010216
:107CA00008BF704730B511F0004502D5404261EB86
:107CB00041014FF4806404F132045FEA915C3FF4C7
:107CC000D8AE4FF003025FEADC0C18BF03325FEA64
:107CD000DC0C18BF033202EBDC02C2F1200300FA15
:107CE00003FC20FA02F001FA03FE40EA0E0021FA3A
:107CF00002F11444BDE600BF4FEA4102B2F1E04395
:107D000024BFB3F5001CDCF1FE5C0DD901F0004C82
:107D10004FEAC0024CEA5070B2F1004F40EB8300D2
:107D200008BF20F00100704711F0804F21D113F1FE
:107D30003872BCBF01F00040704741F480114FEA37
:107D40005252C2F11802C2F1200C10FA0CF320FAC0
:107D500002F018BF40F001004FEAC1234FEAD323DD
:107D600003FA0CFC40EA0C0023FA02F34FEA430347
:107D7000CCE77FEA625307D150EA01331EBF4FF0D0
:107D8000FE4040F44000704701F0004040F0FE40EB
:107D900040F40000704700BF7BB972B90029BEBF34
:107DA00000204FF0004106E008BF00281CBF6FF024
:107DB00000414FF0FF3000F081B9ADF1080C6DE9E2
:107DC00004CE002909DB002B1ADB06F0B7FDDDF835
:107DD00004E0DDE9022304B07047404261EB410159
:107DE000002B1BDB06F0AAFDDDF804E0DDE9022331
:107DF00004B0404261EB4101524263EB43037047E0
:107E0000524263EB430306F099FDDDF804E0DDE93F
:107E1000022304B0404261EB41017047524263EBE0
:107E2000430306F08BFDDDF804E0DDE9022304B036
:107E3000524263EB4303704753B94AB9002908BF64
:107E400000281CBF4FF0FF314FF0FF3000F036B973
:107E5000ADF1080C6DE904CE06F070FDDDF804E02C
:107E6000DDE9022304B0704770B54FF0FF0C4CF40D
:107E7000E06C1CEA11541DBF1CEA135594EA0C0F68
:107E800095EA0C0F00F0DEF82C4481EA030621EAA3
:107E90004C5123EA4C5350EA013518BF52EA0335DE
:107EA00041F4801143F4801338D0A0FB02CE4FF090
:107EB0000005E1FB02E506F00042E0FB03E54FF0C0
:107EC0000006E1FB03569CF0000F18BF4EF0010EB8
:107ED000A4F1FF04B6F5007F64F5407404D25FEAB4
:107EE0004E0E6D4146EB060642EAC62141EA555167
:107EF0004FEAC52040EA5E504FEACE2EB4F1FD0CA9
:107F000088BFBCF5E06F1ED8BEF1004F08BF5FEA26
:107F1000500E50F1000041EB045170BD06F00046D8
:107F200046EA010140EA020081EA0301B4EB5C0485
:107F3000C2BFD4EB0C0541EA045170BD41F480117D
:107F40004FF0000E013C00F3AB8014F1360FDEBFA2
:107F5000002001F0004170BDC4F10004203C35DA7E
:107F60000C341BDC04F11404C4F1200500FA05F301
:107F700020FA04F001FA05F240EA020001F00042A2
:107F800021F0004110EBD37021FA04F642EB060118
:107F90005EEA430E08BF20EAD37070BDC4F10C0442
:107FA000C4F1200500FA04F320FA05F001FA04F206
:107FB00040EA020001F0004110EBD37041F10001F2
:107FC0005EEA430E08BF20EAD37070BDC4F12005FD
:107FD00000FA05F24EEA020E20FA04F301FA05F265
:107FE00043EA020321FA04F001F0004121FA04F20D
:107FF00020EA020000EBD3705EEA430E08BF20EADD
:10800000D37070BD94F0000F0FD101F00046400016
:1080100041EB010111F4801F08BF013CF7D041EA98
:10802000060195F0000F18BF704703F0004652009C
:1080300043EB030313F4801F08BF013DF7D043EA6D
:108040000603704794EA0C0F0CEA135518BF95EA23
:108050000C0F0CD050EA410618BF52EA4306D1D1AA
:1080600081EA030101F000414FF0000070BD50EAC9
:10807000410606BF1046194652EA430619D094EA53
:108080000C0F02D150EA013613D195EA0C0F05D13D
:1080900052EA03361CBF104619460AD181EA030191
:1080A00001F0004141F0FE4141F470014FF0000049
:1080B00070BD41F0FE4141F4780170BD704700BFD2
:1080C0004A0011D212F5001211D20DD56FF4787357
:1080D000B3EB62520ED44FEAC12343F0004343EAAC
:1080E000505323FA02F070474FF00000704750EAF7
:1080F000013002D14FF0FF3070474FF00000704761
:108100009FED197B70B51A4C84ED007B41B30023C1
:10811000DFF868E0101F1D469C4602E001339942DB
:108120000FD050F8042F9607F8D116687645F5D190
:10813000BCF1000F15D10133994215464FF0010CE7
:10814000EFD1BCF1000F0BD095ED017ADFED097A8C
:1081500067EE277A17EE900A05F0DAF9C4E9000114
:1081600070BD05487AF032FD0000000000000000FC
:108170001812012000007A44088B0B0004C50B0084
:1081800090F8743043F0007303F17E43033B102BEF
:1081900005D8DFF83CC05CF823309A4213D310B501
:1081A0009FED097BA0B00C46043004A98DED047B43
:1081B000019266F06DF9019A03AB214604A866F0BE
:1081C0008BF920B010BD70470000000000000000D7
:1081D00034210C00000000002DE9F04F0446A3B04C
:1081E00000250846A160C4E90355A375A282C4F81E
:1081F0008C5084F87C50656012A9914633F0D6FB10
:1082000018B1054673F048F930B9A37D002B40F052
:10821000C58223B0BDE8F08F284633F0B9FC089042
:1082200028B9A37D002BF4D010207AF077FC9FEDC5
:10823000A87B04F118038DED007B129902930122B3
:108240002846984673F0A2F8002840F09E8001234B
:108250000146A56784F87C30404673F013F9002886
:1082600040F02D8282460C900E900B9009900F9555
:1082700019AB042217A9404673F0DEF8002800F07D
:108280008880099B0F9D002B00F019820B9B002B0F
:1082900000F015820E9B002B00F011820C9B002B2E
:1082A00000F00D82284633F0DBFC0D9AA17D91454C
:1082B0004B4628BF13461E469D00002900F01D8234
:1082C00028463CF0A7FB002800F01B82E06056B176
:1082D0004FF0FF31012E016005D00423E268D15038
:1082E00004339D42FAD1A17D75002846002900F093
:1082F00013823CF08FFB002800F0118200212061E6
:108300002A463EF0ADFBA17DB4F88230E37524200F
:10831000002900F01E823CF07DFB0746002F00F094
:108320001C826D4B3B60B4F8825094F88530A17D7F
:1083300006FB05F59D401F35B4F87E30C5F34F159B
:1083400003FB05F5AD002846002900F0FE813CF056
:1083500061FB0346002B00F00D822A4600211846DF
:108360003EF07EFB009094F88530B4F88210012234
:10837000002002FA03F306FB01F1B4F87E2001901D
:1083800038461CF057FC676043E7284633F068FC2A
:108390003BE7199B032B7FF674AF179B0793002BCA
:1083A0003FF46FAF19AB042217A9404673F044F8AD
:1083B00000287FF466AF199B032B7FF662AF179BF3
:1083C000464A934226D0464A934200F08F80454A5F
:1083D000934263D0444A934200F0F580079A0AEB37
:1083E0000203194640469A4673F04CF800287FF481
:1083F00048AF099B002B3FF43BAF0B9B002B4AD0AF
:108400000E9B002B61D00C9A002A40F0C5810B9383
:1084100009932DE716AB232219A9404673F00CF8F7
:1084200000287FF42EAF169B222B7FF62AAF9DF8F3
:108430007E50079B9DF883109DF8822065F307000E
:108440009DF881500AEB030665F30F209DF88430F8
:1084500084F8883062F317400A4403EB4203DBB22E
:1084600084F889300733DB1084F88A30DDF86A300D
:10847000C4F87E3061F31F60BDF87A30C4F8840020
:10848000A4F8823031464046B24672F0FBFF002825
:10849000B3D00F9DFAE6089B0993E9E619AB0422D5
:1084A00016A9404672F0C8FF00287FF4EAAE199B77
:1084B000032B7FF6E6AE169BC4F89C300AF10C0342
:1084C000C4F89430089B0E9388E70B9B0993CFE682
:1084D0000000000000000000D4E20B006865616449
:1084E000636D61706C6F6361676C796619AB0422B0
:1084F00015A9404672F0A0FF00287FF4C2AE199B78
:10850000032B7FF6BEAE159AA37D0A9202EB82057D
:10851000A4F89020AD00002B00F0E38028463CF04A
:1085200079FA002800F0BE800A9BC4F88C0043B1A1
:1085300000252E4616AB102219A9404672F07CFF8A
:1085400010B1089B0B9349E7169B0F2BF9D99DF8A7
:1085500072C0BCF1000F0AD0ACF10203012B06D9A6
:108560000A9B0135ADB2AB422E46E3D8E9E7DDE91F
:10857000191206EB8603D4F88C70BDF86C00BDF8B8
:108580006EE0BDF8706047F823201044D4F88C20CA
:1085900002EB830251445060D4F88C2002EB83023A
:1085A000A2F808E0D4F88C2002EB830282F80AC01B
:1085B000D4F88C2002EB83021161D4F88C2002EBFA
:1085C00083029681CCE7D4F89C30B4F88220C4F8BA
:1085D00098A0012B00F0DB8000250A920D952F4614
:1085E0000C9510E00D9A93423ED0002F40D00C9A8B
:1085F000002A7BD10D9301230C93D4F89C300135D4
:10860000013B9D4237D20DF1470304930DF1460320
:10861000039319AB029316AB019315AB00934FF084
:1086200000038DF846308DF8473013AA14AB21466D
:10863000404667F039FF002300931699199B03FB0E
:1086400001F194F885300DF1460203FB01F140463B
:108650000DF1470367F0E2FE139B002BCDD00A9A81
:108660009342BFD10137C8E70C9B01330C93C4E799
:108670000A930127C1E7B4F882300C983A46002BE0
:1086800039D1002855D1BDF82830A4F8823013B96B
:108690000123A4F88230012A089B0C9338BF0122E1
:1086A0000D929BE694F87C302E460F9D13B1204628
:1086B0001FF07EFAA37D002B73D1C4F88C3094F8A0
:1086C0007C3013B120461FF073FA284633F0C8FA05
:1086D000A37D002B3FF49DAD334840F2CA317AF0C0
:1086E0007DFA1946284665F09BF81AE7B4F88230FF
:1086F0000C983A46EBB10244CDE7284665F090F875
:10870000E1E594F87C3013B120461FF051FAA37DC7
:10871000002B39D1E3607CE565F082F8EBE594F855
:108720007C3013B120461FF043FAA37D63BB236165
:108730006FE50A9B0D9999422ABF0D9B00EB4202FF
:1087400002EB4002C3F34F039FE765F069F803466D
:1087500000E665F065F80746E0E594F87C3013B173
:1087600020461FF025FAA37D002B3FF4DAAD24202C
:108770007AF088F994F87C3013B120461FF018FA8B
:10878000A37D002B3FF445AD28467AF07BF9002A03
:108790003FF47EAF00227EE70F9D83E503487AF029
:1087A00015FA30467AF06EF9988D0B00988E0B0012
:1087B00010B584B004469DF820E09DF828C00393CE
:1087C00008469DF81C1084F8371000216EF307014D
:1087D0006CF30F21BDF818C084F832C0CCF1080C3E
:1087E00084F836C09DF82CC09FED0F7B6CF31741C9
:1087F000E163002121609DF8241084F8331084ED9A
:10880000027B1146CDE9010272F01EFA0198029A2C
:108810000399A0852046E28504B0BDE810402EF003
:1088200035BB00BFAFF30080000000000000000077
:1088300000B513A3D3E9002385B0FFF7ADFA01A972
:1088400075F004FD9DF807309DF806209DF808C0DE
:108850009DF80910BDF804001B0443EA425343EAA3
:10886000CC239DF80A2043EA411343EA5203A0F2C5
:10887000BC7043EA406005B000BD00BFAFF30080AC
:1088800000CA9A3B0000000000B59FED0D7B89B047
:108890000923016802904FF00A0C039302A80023F9
:1088A0008DED007BCDF810C0CDF814D08DF81830C8
:1088B00046F0B0FF0098003818BF012009B000BD95
:1088C0000000000000000000A64A1378002B40F0D2
:1088D0007A822DE9F04F012395B0A34CDFF8A4B2C2
:1088E00004AF13702168A14D2268A1482944C2F544
:1088F00080621AF0BFFA8046002849D002200DF0AD
:108900006BFB23689BF800202D784344012A2360E9
:1089100040F23A81290702D0AA4240F07C83302DF0
:1089200028D80F2D2FD9A5F11003202B2BD8DFE845
:1089300013F005012A00B3002A002A002A002A00A9
:108940002A002A002A002A002A002A002A002A00D7
:108950002A007B002A0048002A002A002A002A0058
:108960002A002A002A002A002A002A002A002A00B7
:108970002A003600502D00F0D681602D00F0A08135
:10898000402D00F0588100232360B8F1000FA9DCCE
:10899000744A002344371370BD46BDE8F08F734B13
:1089A0005B8840F23112B3F57F7FBA85226880F090
:1089B000D181191D8A4280F0C48101238BF80030D7
:1089C000E3E76A4B9B6840F22112B3F57D7FBA85DD
:1089D000226819D20C339A42EFD3644D65486E6811
:1089E000314672F04FFDAA68624805F10C0107F1AB
:1089F0001C0372F069FD5D4BFA699B689342054662
:108A000002D8002800F0BC820023022287F82D2023
:108A100007F12C010093142255481AF093FA564B93
:108A2000186833F01DF92DE0504B5B8840F221129D
:108A3000B3F57B7FBA85226819D203F114018A420B
:108A4000BBD34E49494A4E4D12692A604FF0000986
:108A500001F80390084607F11C0132F0A7FF464ECB
:108A6000306020B172F018FD002840F039820222F7
:108A7000002387F82D203E480093142207F12C0193
:108A80001AF060FA002302208BF8003023600DF00A
:108A90009BFA0DF0A9FA78E72368364840F21113E3
:108AA000BB8372F04BFC314AF86053683B62A0EB29
:108AB000030993687862994528BF99460026C7F84C
:108AC0002890102207F11C012948009633461AF01D
:108AD00039FA264A2748516872F0D4FCB9F1000FE0
:108AE00022D0BD600AE0BCF1000F1BD1CDF800C060
:108AF0001AF028FABB691E44B14513D9A9EB060246
:108B0000142A07F1180328BF142207F12C01194871
:108B100072F092FCBA698446034607F12C011448AE
:108B2000002AE0D1BD68B144FB684B4540F24C815E
:108B300012238BF800300023236026E70B4B5B8861
:108B400040F21112B3F57C7FBA83E946226880F0C7
:108B50001B8103F10C018A4280F0078101238BF80D
:108B6000003012E73F7C0120184C012018480120FA
:108B700028450120480A0120A04601202C48012058
:108B800048770120397C0120302D4DD80F2D40F23F
:108B90002682A5F11003202B00F2248101A151F8B7
:108BA00023F000BF3D8B0200E58D0200998A020090
:108BB000E58D0200E58D0200E58D0200E58D0200E5
:108BC000E58D0200E58D0200E58D0200E58D0200D5
:108BD000E58D0200E58D0200E58D0200E58D0200C5
:108BE000E58D0200298A0200E58D0200C38902009A
:108BF000E58D0200E58D0200E58D0200E58D0200A5
:108C0000E58D0200E58D0200E58D0200E58D020094
:108C1000E58D0200E58D0200E58D0200E58D020084
:108C2000E58D02009F890200502D7CD0602D47D039
:108C3000402D40F0D780A04B5B8840F24112B3F545
:108C40007C7FBA85226880F0B28003F110018A42ED
:108C5000FFF4B3AE591E994A505C2F280BBF002376
:108C600000215354D154944BD3E902018EA3D3E98C
:108C70000023FFF791F89249904A20F00100A0FBF1
:108C8000010172F013FD002840F09180009003462E
:108C900010228C4807F12C011AF054F989481AF077
:108CA00031F8002302208BF8003023600DF08CF99E
:108CB000854B223DEDB2EB40DB077FF566AEE8E683
:108CC0007D4B5A889B88134440F26111B3F57E7F37
:108CD000B985216815DC07339942FFF46EAE7B48F5
:108CE0000025855430F8041C30F8023C0131014461
:108CF000CD5472F00FFD0A2800F07581002800F0B5
:108D000062810222002387F82D206E48009307F12C
:108D10002C011AF017F9002302208BF80030236091
:108D20000DF052F9B5E6206807F098FA01288BF8A3
:108D300000003FF42AAE0023022023600DF044F926
:108D400023E663490022CA54084672F075FC0028E5
:108D500000F055810222002387F82D2007F12C0115
:108D6000009358481AF0EEF89BE75A495A4D0022F2
:108D7000CA54084607F1140132F018FE286018B1F1
:108D800072F08AFB00283BD1022200237A774D48FB
:108D90000093102207F11C011AF0D4F80023CD46ED
:108DA00002208BF8003023600DF00EF9EDE5002372
:108DB000022287F82D2007F12C0100931022414850
:108DC0001AF0C0F86DE77047444872F089FA002342
:108DD00002208BF8003023600DF0F6F8202D7FF490
:108DE000D4AD56E6012A3FF4D0AD00230220236023
:108DF0000DF0EAF8402D3FF6C8AD212DEED957E72A
:108E00009FED2B7B354B2868796902938DED007BB4
:108E1000012272F0BBFAF8600028B5D12F4872F039
:108E20008DFA2549B8604D688B687862461B9E4272
:108E300028BF1E46FB68BE623D621022009307F108
:108E40001C01FB601F481AF07DF82E442348294678
:108E500072F018FBB5421CD2C7E90089D7F80C9014
:108E60001E48721B102A28BF102207F1180307F1B1
:108E70002C0172F0E1FABA691248CDF8009015445D
:108E8000002307F12C011AF05DF8AE42E8D8D7E9CB
:108E90000089BB68AB4240F2FD801223CD468BF8BF
:108EA00000300023236070E500CA9A3B00000000F8
:108EB00000000000000000001848012028480120A0
:108EC00000CA9A3B28450120014000401E4801206D
:108ED0001C48012024480120A0460120480A012006
:108EE000306832F055FE002800F0C8807C4BDFF877
:108EF00000A2D3E90223FA601046BB60194676A3AC
:108F0000D3E90023FEF748FF764AF96920F0010310
:108F1000A3FB0232CAE90032FA6830680092BB68EB
:108F20000193714B0293062272F030FA0346002837
:108F300040F0C2806A492A68D1F80490C9F3080554
:108F4000A2EB0902C5F50075954228BF1546002D14
:108F500072D0DAF800207A63DAF80420BA63C7F82E
:108F60003090FD631422009007F12C01FB605F48F4
:108F700019F0E8FFFB68236022238BF8003004E53A
:108F8000DFF874915A4A1E44D9F800303E639B1BA7
:108F9000B3F5007F28BF4FF40073FB6313687B6356
:108FA0005368BB63142200902B46504807F12C01F4
:108FB00019F0C8FFD9F800309E426FD022232560F7
:108FC0008BF80030E1E400900346022207F12C0107
:108FD000464819F0B7FF454819F094FE9BE6012A70
:108FE0003FF4D3ACA7E6052387F82D300222009585
:108FF0002B4607F12C013D4819F0A4FF8BE60090A9
:109000000346022207F12C01384819F09BFF37482C
:1090100019F078FE45E60023042187F82C2087F814
:109020002D100222009307F12C01304819F08AFF1D
:1090300002200CF0C9FFABE449462B4872F022FA3B
:10904000294872F035FA284872F04AF9306832F04F
:1090500007FEDAF800307B63DAF80430BB63C7F848
:109060003090FD632B460095142207F12C011F4818
:1090700019F068FF1D4819F045FE03E5052387F840
:109080002D3014220090034607F12C01174819F0E7
:1090900059FFF7E4144872F023F97FE6124872F0A2
:1090A00007FA114872F01CF9124B186832F0D8FD1B
:1090B0000E4819F027FEE5E4022387F82D3014222C
:1090C000CDF800904B4607F12C01084819F03AFF03
:1090D000306832F0C5FDD5E400CA9A3B00000000BC
:1090E0001848012000CA9A3B480A0120284501205F
:1090F000300A0120A046012048770120000000002E
:10910000F0B5CDB00BB100241C70529C14B1529D2F
:1091100000242C60539C1CB19FED2B7B84ED007BC5
:1091200004787CB10D46083004A917461E4683F02A
:10913000FCFF044618B99DF82A203AB92870204649
:109140004DB0F0BD022420464DB0F0BD0DF12A0017
:1091500070F00CFA7A1E824228BF02460DF12A01F5
:10916000284603923DF098FA039A04ABAC541A7B5C
:1091700002F0100216B1C2F300113170529911B110
:109180000AB91A680A60539A002AD8D05A891989EC
:1091900002F01F035B000193480AC2F345130093DA
:1091A00000F2BC70D30A01F01F02C1F3431174F046
:1091B00049FF074B539AA0FB0303C2E90003204673
:1091C0004DB0F0BDAFF300800000000000000000D3
:1091D00000CA9A3B0000000070B5CCB01546509C08
:1091E0000AB100222A700BB100221A601CB19FED57
:1091F0001A7B84ED007B803004AA039384F0B5F8D9
:10920000064630BB9DF81C10039B04AA01F0100118
:1092100015B1C1F30010287013B109B911681960B4
:10922000BCB15389118903F01F025200480A019210
:10923000C3F345120092DB0A01F01F0200F2BC707A
:10924000C1F3431174F0FEFE054BA0FB0303C4E918
:10925000000330464CB070BD00000000000000006C
:1092600000CA9A3B000000002DE9F04F87B0044689
:1092700000AF8A469046002540F02CFF07F1080118
:10928000204601223D7267F0ADF897F90800397A5F
:10929000A84234DA01F0E003E02B30D0A02B36D026
:1092A00001F0F003902B00F0A881802B00F0AE813C
:1092B000A1F1C0031F2B00F29D81DFE813F097019D
:1092C0009B01990195015800580058008A008A00B6
:1092D0008A002101CB00E900F600050134014501B7
:1092E000530161016F01800187018E0113011A0191
:1092F00041004100410096009600A300A3004000F9
:1093000040F0010318461C37BD46BDE8F08F01F060
:109310001F02D31D03F038036D46ADEB030D6B4602
:109320003AB169462046C7E9003267F05BF8D7E9F1
:1093300000321846114649F0EDFC0346AD46E1E720
:109340002731C9B2204667F013F90546014607F1F7
:1093500008007EF07DF925B139692A46204667F07C
:1093600041F807F1080049F023FD0346CAE73C3104
:10937000C9B2204667F0FCF805468046014607F171
:1093800008007EF065F9F5B1396920686668796092
:10939000B8F5807F454628BF4FF4807504F10C0373
:1093A0002A46B0470346E0687968002840F05581B6
:1093B000002B00F04E819D4200F24881B8EB05037E
:1093C00029449846E1D107F1080049F033F90346F2
:1093D00098E73931C9B2204667F0CAF852460146CB
:1093E000204679F063FC03468CE72531C9B220465C
:1093F00067F0BEF8434601465246204679F018FC15
:1094000003467FE72331C9B2204667F0B1F8B0F1D7
:10941000005F834680F0238149F09AF90346BBF14F
:10942000000F3FF46FAF00254246514620467B6057
:10943000FFF71AFF4246814651462046FFF714FFC8
:10944000013502464946786846F0C6FCAB457B6864
:10945000EAD157E79FED847B0822B918204687EDB3
:10946000027B66F0BFFFD7E9023210BA19BAFEF7E5
:1094700043FC07EE900AF4EE677AF1EE10FA50D64C
:10948000034623F0030343F00203A3F1FF4339E74C
:109490000023012207F1080120463B7266F0A2FF7B
:1094A0003B7A5B0043F001032CE70023022207F123
:1094B000080120463B8166F095FF3B895BBA9BB271
:1094C0005B0043F001031DE70023042207F10801BC
:1094D0002046BB6066F086FFB86800BA49F030FBF2
:1094E00003460FE752460821204679F0DFFB03468A
:1094F00008E752461021204679F0D8FB034601E7E1
:109500000023042207F108012046BB6066F06AFFD1
:10951000BB681BBA07EE903AF4EE677AF1EE10FAE8
:10952000AFD7534BEEE69FED507B0822B91820468B
:1095300087ED027B66F056FFD7E9021009BA00BA40
:1095400049F020FB0346DDE60023012207F1080174
:1095500020463B7266F046FF97F908305B0043F007
:109560000103CFE60023022207F1080120463B81D8
:1095700066F038FF3B89DBBA5B0043F00103C1E6CC
:109580000023042207F108012046BB6066F02AFF91
:10959000B86800BA49F02EFA0346B3E69FED327B75
:1095A0000822B918204687ED027B66F01BFFD7E939
:1095B000021009BA00BA49F087FA0346A2E65246F9
:1095C0000121204679F072FB03469BE652460221B8
:1095D000204679F06BFB034694E652460421204670
:1095E00079F064FB03468DE63E238BE60E2389E685
:1095F0001E2387E61F4879F0E9FA4346524601F0F8
:109600000F01204679F014FB03467BE601F00F06BC
:10961000304649F09DF8B3460346002E3FF472AE43
:109620004246514620467B60FFF71EFE4246814679
:1096300051462046FFF718FE013502464946786834
:1096400046F0CAFBAB457B68EAD15BE60A4879F095
:10965000BDFA0A48194684F0AEFD79F05FFA084871
:10966000722179F0BBFA00BF00000000000000008A
:1096700002004000708D0B0044780B00CC550B00AD
:1096800048940B00D2B32DE9F0436FF00E0885B07B
:109690000646174601F10F04A8EB010854F80F0C19
:1096A00054F80B1C54F8072C54F8033CEC46ACE877
:1096B0000F003146A4F10F0001F0B4FCA4F1100337
:1096C00006F1EF0213F8011F12F8010FA34281EA1D
:1096D00000011970F6D1EC46BCE80F00103408EB1D
:1096E000040C6745C6F8F000C6F8F410C6F8F82078
:1096F000C6F8FC30D2D805B0BDE8F083704700BF93
:109700002DE9F041044682B36FF00E05164601F1D3
:109710000F0700F1F0086D1A08F1FF31A7F11003EF
:10972000A7F10F0813F8012F11F801CFBB4282EA0D
:109730000C021A70F6D121464046103700F018F995
:10974000EB199E42E8D8D8F80010D8F80420D8F8D1
:109750000830D8F80C00C4F8FC00C4F8F010C4F8C5
:10976000F420C4F8F830BDE8F08100F1F008EAE731
:10977000002A44D070B54C1E84B0064615194FF02F
:10978000100C01E00CF1010CBCF1100F0BD00DEB33
:109790000C0214F8013F1278AC4283EA02032370F2
:1097A000F0D104B070BDD6F8F000D6F8F410D6F8B9
:1097B000F820D6F8FC30EC46ACE80F00314668469D
:1097C00000F0D6F80F2206F5807111F8013DFF2B4D
:1097D0000FD03244013382F8F03014F8013F9DF885
:1097E0000020AC4283EA02032370DAD04FF0010C70
:1097F000CDE70023013A0B70531CE6D1EDE770472B
:1098000003460846194601F00DBC00BF0346084652
:10981000194600F0ADB800BF182A2DE9F04F0546F3
:10982000C0F800217ED0202A76D0102A7ED183462F
:1098300040F20A43A5F80431AC4600200B788CF8BE
:1098400000304B788CF801308B788CF80230CB7874
:109850008CF8033095F80531013098421A4601F131
:1098600004010CF1040CE9D395F804110131B3EBB8
:10987000810F55D20BEB8201501E11F802EC1BF840
:10988000204011F803CC11F8010C2B4FDFF8AC800D
:109890002DE017F80CA018F8099017F80EC017F86B
:1098A00000E0385D8AEA0904A2EB03090BEB8903A7
:1098B0001BF8299084EA09040C7093F80190043194
:1098C0008CEA090C01F803CC93F802908EEA090E99
:1098D00001F802ECDB78584001F8010C95F80431EE
:1098E00001320133B2EB830F1AD295F80531B2FB86
:1098F000F3F903FB192ABAF1000FCAD0D5F80061B9
:10990000202ED1D1BAF1040FCED13C5D17F80CC096
:1099100017F80EE0385CC7E7834640F60E0389E788
:10992000BDE8F08F834640F20C6383E700239B463B
:10993000A0F804311A469DE714200C00081F0C0003
:1099400000B583B0CDE90030FFF766FF009B0198BA
:10995000D3F800C059689A68DB68C0F8FC30C0F8DA
:10996000F0C0C0F8F410C0F8F82003B000BD00BF8C
:109970002DE9F04FD1F80031103B102B85B089460E
:10998000864600F2E980754A22FA03F313F0010FCC
:1099900014BF0D4600250EF10406344600270EEBD9
:1099A000070379191A7811F8010B424003F8012BCB
:1099B0009C42F7D10437102F04F10404EFD10EF1CB
:1099C0001008674FCDF804804FF0010C0EF114021F
:1099D000AB46CA467146002311F82300385C01F8F3
:1099E00023000133042BF7D101318E42F3D19EF8CD
:1099F00005409EF809109EF801309EF80D509EF823
:109A000002008EF801408EF805109EF80A409EF87C
:109A100006108EF809508EF80D309EF80E509EF804
:109A200003308EF802408EF80A009EF80F409EF830
:109A30000B008EF80E109EF807108EF806508EF868
:109A400003408EF80F008EF80B108EF807309AF84E
:109A5000043163456AD0CDE902CB7046047845787D
:109A60008178C37884EA05094FEAD9184D404FEA56
:109A7000D51C08EB480859405C4008EBC8080CEBC3
:109A80004C0C00230CEBCC0C68F307036CF30F2396
:109A90004FEAD11C0CEB4C0C0CEBCC0C89EA010B03
:109AA0006CF317434FEA49094FF0000C6D0069F35E
:109AB000070C490065F30F2C61F3174C0021E509F1
:109AC0006BF3070164006BF30F2105EB450564F3AD
:109AD0001F6C6BF31741046805EBC5056BF31F6141
:109AE00065F31F6383EA0C0361404B4040F8043B7D
:109AF000019B8342B2D1DDE902CB34464FEA0C151B
:109B0000231F0BEB0500197810F8018B81EA08017F
:109B100003F8011B9C42F6D10434A24205F104056E
:109B2000EED10CF1010C5FFA8CFC53E75D464FEA75
:109B30000C1C331F05EB0C00197810F8014B614029
:109B400003F8011B9E42F7D10436B2420CF1040C1B
:109B5000EFD105B0BDE8F08F00251CE70101010041
:109B600014200C00FEE700BF2DE9F04F4FEAA309D7
:109B70005C4FDFF8ACB1DFF8ACA103F0030486461C
:109B80004B4659488BB007EB84171C2B50F8240028
:109B90000090A8BF1C2378680197033323EAE3737E
:109BA00018410790B86818410890F8681841099062
:109BB000B9F11F0F4FF00000C8460690A8BF4FF044
:109BC0001F080BE00DEB8505AC69002B40EA040093
:109BD000B8BF6442013A41F8044B75D05EF8043BCB
:109BE00013EA0B0F23F00045ECD013EA0A0F0BD158
:109BF000019CB9F1000F54F82540BABFC8F1000527
:109C0000AC4044FA08F4E0E7384C23420DD1103D53
:109C1000374C54F82540009D84FB0565A8F10304EA
:109C2000002C47DB45FA04F4CFE76C04B4F1006F75
:109C3000BABF6C0504260026B4F1005FBCBFA400C7
:109C400002362C4DB4F1804FBCBF64000136AC42EB
:109C50003DDD294D294FCDE9045705F1F95505F5AD
:109C6000CE2505F29B150395254F264D02952546D9
:109C700087FB05C5029F3D44274685FB07C7039D1B
:109C80002F44254687FB05C5049F3D4485FB04748E
:109C9000059D2C441C4D55F8265084FB0575EC00A1
:109CA000009D84FB0575194C54F82640A8EB04046C
:109CB000002CB7DA66426FF0004444FA06F7AF4270
:109CC00083DB05FA06F480E70BB0BDE8F08F104D9A
:109CD000104FDFF854C0CDE904570F4D0F4FCDE9B9
:109CE000025CC4E788370C0088380C00C0FFFF7F97
:109CF000C8360C009979825AF0CEC227B477F5FEA7
:109D000063218510A4F633D388360C00A8360C00E6
:109D10008D496C23591858FF28482EB0A9BDA02999
:109D2000FCFFFF7FF0FFFF7F1BAA5759844602F01C
:109D300001007BBB60B3DCF88034DCF88001DCF828
:109D40008012DCF880235B42CCF88034DCF8803869
:109D50004042494252425B42CCF88001CCF880122A
:109D6000DCF88005DCF88016CCF88023CCF880384D
:109D7000DCF88027DCF880304042494252425B42A6
:109D8000CCF88005CCF88016CCF88027CCF8803051
:109D9000002070472DE9F047C3F11F04002847D089
:109DA0004FF00047DF4000200CF18006013F0CF52A
:109DB0001069804656F8802C42FA04FEBEEBE27F22
:109DC00087EAE27E18BF72469A40454646F8802CE4
:109DD00082EAE275A5EBE275DCF88020C2F1000EA4
:109DE0004EFA04F2B2EBEE7F87EAEE7218BF9646A7
:109DF0000EFA03F2CCF88020C64682EAE27EAEEB91
:109E0000E27E0A6845EA0E05284342FA04F5B5EBFE
:109E1000E27F87EAE27518BF2A460CF5807C9A40FB
:109E2000E14541F8042B06F58076C3D1BDE8F08703
:109E30004FF00046DE40013E0CF180050CF5106E3F
:109E4000074655F8802C42FA04F9B9EBE27F86EA1E
:109E5000E27918BF4A469A40B84645F8802C82EA13
:109E6000E278A8EBE278DCF8802042FA04FABAEB58
:109E7000E27F86EAE27A18BF52469A40B946CCF8A9
:109E8000802082EAE279A9EBE2790A6848EA0908C7
:109E900040EA080042FA04F8B8EBE27F86EAE2788A
:109EA00018BF42460CF5807C9A40E64541F8042BE9
:109EB00005F58075C5D1BDE8F08700BF2DE9F041FB
:109EC000436903F5A0430746D3F8C46DD3F8C08DAA
:109ED000EEB1046A0025033414F8023C14F8031CA4
:109EE00014F8012C1B0203EB01431A4429463046A7
:109EF0001BF072FB2946304601351BF05BFBB5F5C4
:109F0000807F04F10304E7D197F825303BBBF96863
:109F10003868B8F8042043189342D7E90134234441
:109F2000B8F80640C8BF111AA34216DA904214DAF4
:109F3000002912DDB8F80C2002FB03F3D8F8082042
:109F400002EB8302BB6986B10244013A194413F85B
:109F5000010B02F8010F8B42F9D1BDE8F08197F8AF
:109F6000241030461BF030FBD1E702EB400297F89B
:109F70002500FC69012809D0194413F8010B34F8B5
:109F8000100022F8020B8B42F7D1E6E797F8245035
:109F9000194413F8010B85421CBF34F810001080DF
:109FA0008B4202F10202F4D1D7E700BF2DE9F04164
:109FB00000F5A04882B098F8AE1D426B01238DF8E1
:109FC0000730036B51BBD11A4C1E40F2F942944248
:109FD00024D833BB044640F2FA4600F1540514E09D
:109FE000636BB3421ADC236C9847616B236C9DF85A
:109FF000072001F5BD511431214428469847636B71
:10A000009DF8072013446363D2B1D4E915739F42CE
:10A010004FF001020DF107012846E1DB02B0BDE877
:10A02000F08100F5BD5213321344551813F8014F57
:10A0300002F8014FAA42F9D10023C0E90C31C9E767
:10A04000012388F8AE3D02B0BDE8F08170B500F59F
:10A05000A042002382B0436582F8B43D82F8AE3D51
:10A06000826D4FF0FF310B2AD8BF5218C0E908317A
:10A07000C8BF0C22036C019200F5DA71044654301B
:10A080009847019A824227D11849052204F5DA70CF
:10A090003CF0ECFA30B11649052204F5DA703CF0D8
:10A0A000E5FA00BB94F8BE31B4F8BA11B4F8BC219B
:10A0B0002160C3F302130133C4E90121E260A3610B
:10A0C0000146626C04F154009047A368B3F5A07F89
:10A0D00007DC012002B070BD06230020E36102B05E
:10A0E00070BD0223F9E70823F7E700BF2C450B00FA
:10A0F00034450B0041F2167C614500F276812DE972
:10A10000F04F00F58D5A0AF1140A00F5ED5700F5ED
:10A110009B460368856A91B00E372E3600F5DA7ECD
:10A120005446A64500F0BD80725C04F8012D37F856
:10A1300011106145F5D95B1B00F17408BAEB0407F7
:10A14000434400F0AE80C16A00F5A5521432039278
:10A1500000293A46054647464FF0000B00F5A04659
:10A16000904640F39A80A86A404500F32E811A1861
:10A1700093420BD2013B04EB000C14F8012B03F8C3
:10A18000012FA445F9D1D5E90A0164462A682B6953
:10A19000AA6202930593A8EB0008039B96F8B40DFE
:10A1A0000B9700280CBFD14699460892D5F804C0F9
:10A1B00096F8B3EDCDF824C00138CDE90C9918BF5D
:10A1C00001208DF83C00D5F81490CDF81890ACEB38
:10A1D00001011EF0400F07910CD00CF1FF3000EB95
:10A1E000D07EB1EB6E0F40F3B58040F00100C0EBC4
:10A1F0004100079096F8AF0D96F8B11D96F8B03D66
:10A2000001934FF0000E00F0010C61F3070EC0F354
:10A2100082006CF30F2E60F3174E63F31F6ECDF8C0
:10A2200038E0D5E9193E0A93BEF1000F23D0079B11
:10A2300002999944AB68022803FB09130EEB8303D0
:10A2400032D0BCF1000F3AD0002A0FDD9DF838C0A3
:10A25000394611F8010B844518BF18700898A1F110
:10A260007402521B904203F10103F2DC96F8B6ED42
:10A27000BEF1010F2CD0AB6C05A89847E96A0139F3
:10A2800011F0030FE96208BF4BF0010BB8F1000FAA
:10A2900003D000293B463FF766AFBBF1000F40F00B
:10A2A0008E8011B0BDE8F08F184601993CF0D8FBC4
:10A2B0009DF839C0089A0346BCF1000FC4D1184676
:10A2C00039463CF0E9F996F8B6EDBEF1010FD2D16E
:10A2D000DDE906329918AA68059BE86896F8B5CDBD
:10A2E00002FB0131AB6E00FB02F2BCF1010F03EB8C
:10A2F00081010C9803EB82032A6850D9002A27DDDC
:10A30000CDE9017403334FF0000C4FF0030911F84D
:10A31000012B02EB42070333C75D03F8067C12FBF7
:10A3200009E70224C75D03F8057C12FB09420CF122
:10A33000010C825C03F8042C2A689445E7DBDDE914
:10A340000174D5E9023203FB02F2AB6E03EB820328
:10A350000B9390E700288646B8BF0CF1020EB1EBD4
:10A36000AE0F07DD20F0030040F00200C0EB8101DA
:10A3700007913FE700288446B8BF00F1070CB1EB16
:10A38000EC0F4FEAC10E07DD20F0070141F0040198
:10A39000AEEB010107912DE7CDF81CE02AE7002A7A
:10A3A000D6DD4FF0000C11F8012B30F8122023F805
:10A3B000022B2A680CF1010C9445F4DBC1E7284616
:10A3C00011B0BDE8F04FFFF7F1BD4746DA199342EF
:10A3D00008D2013BE11914F8012B03F8012FA14227
:10A3E000F9D1A86AC01BA86257E7704710B5D0E939
:10A3F00000431B1B9342B8BF03F1FF3284B012B974
:10A40000104604B010BD04460123009300200390C1
:10A4100003ABE0684DF0F4FE0246039828B92368C8
:10A4200010461344236004B010BD78F077FB00BFE2
:10A4300010B582B0002201AB0446C06801924DF015
:10A4400019FF031E02DB236002B010BD019878F0F3
:10A4500065FB00BF10B545F6B8520C4600213CF034
:10A46000FFFA00F5A04383F8B54D10BD2DE9F04F7C
:10A470000646436C856D87B00F465430002106F5C3
:10A48000DA749847336C4FF48052214606F1540039
:10A49000984796F9BE1196F8BE2100290346A5EB10
:10A4A0000005C0F2F0804FF00D094FF0000E42F2AF
:10A4B0001072CDE901E24FF0020BF2461A46039703
:10A4C0000BF1FF339145049329DA4846171AB7F583
:10A4D000817F034604EB000131DB09782C2942D04F
:10A4E0003B291CD021291AD12344811C5F789878FC
:10A4F000F92F00F0FD800844231802305F7867B11F
:10A5000001460F44791CE75DA2EB010907F2011334
:10A510004B455FDA002FF4D108469042D6DB039F0B
:10A52000D646ABF1020C019BBB60029BC7F800C092
:10A530000120FB60C7F804E007B0BDE8F08F3A46A1
:10A5400020463CF0DDF8336CC7F58052E11906F186
:10A550005400984721463A1809782D1A2C294FF0B3
:10A5600000000346BCD19042D9DA234400F10A0925
:10A5700093F909105B7A002953DB09F1010103F219
:10A580000113571ABB4239DA631809F102091F781F
:10A590007FB14946A946B1F5406F6EDDB9F1000FB4
:10A5A00007EB01034DDCE75C591C002FF6D14D464B
:10A5B000894614F809303B2B04EB090100F0B58003
:10A5C000002D6CD1A2EB09031F2B40F3AE800BF1E1
:10A5D000010B75E74A46214420463CF091F8C9F545
:10A5E000805204EB0901336C06F1540098470021B6
:10A5F00009EB00022D1A002F83D18DE78A426BDC14
:10A60000891A01F1010963184FF48052214600278D
:10A61000059306F15400336C9847059B3A182D1AA0
:10A62000B5E703F00703022199404FF0030011FB47
:10A63000009909F1010103F20113571ABB42DDDA57
:10A64000A2E7551A2A46214420463CF059F8C5F5A0
:10A6500080524A45A8BF4A46336C611906F154003E
:10A660009847E35D2A18A9EB0009791C002B9ED0BE
:10A670000B44591CE75C002F99D00F44791CE75D0F
:10A68000002F88D193E702F007024FF0020909FA80
:10A6900002F94FF003010D2219FB012905E7B36D03
:10A6A000B3F5805F93DD002D91DDA2EB09094A46E9
:10A6B00020463CF025F8C9F58052AA42A8BF2A4698
:10A6C00004EB0901336C06F15400984709EB0002D2
:10A6D0002D1A4FF000097AE721443A4620463CF013
:10A6E0000FF84FF00109E119C7F5805223468FE7B3
:10A6F00004287FF400AF1F795B7947EA0323022B1C
:10A70000B8BF0223019F03EB8303B7EB430F0AEBB0
:10A71000430A4FEA430C02DACDF804C0EBE6029B91
:10A720006345A8BF63460293E5E6DDF810C0039FCA
:10A73000D646F8E6FFF78ABC2DE9F04F8BB0044609
:10A740000491934609B100230B60D4E915735A1E96
:10A75000974227DA04F15402009204F5A041002246
:10A7600081F8B42D81F8AE2D22624FF0FF32626283
:10A7700007F1FF029A42C6BFDB1B03F1FF394FF01E
:10A78000FF0904F5DA750591236C00984A462946BD
:10A790009847814506460ED00623E36100200BB0A2
:10A7A000BDE8F08F636C04F15400002100909847DD
:10A7B000D4E91573D1E7002F00F0978000212B46D4
:10A7C00089461A782C2A22D0DA46B3463B2A00F072
:10A7D000E581212A40F0E78105EB090209F1020831
:10A7E0005278FE2A00F0F980FF2A00F0A980012AA1
:10A7F0006FD0F92A40F0EE8015F80820042A00F006
:10A8000055814146C1462C2AE0D15E46D3462944B3
:10A8100005EB090388785A7802EB00222261087957
:10A82000CA7802EB0022626188794A7902EB002241
:10A830002260087ACA7902EB002262605B7A059A8C
:10A8400082F8B33D1A0609F10A0800F16381059AFE
:10A8500015F8083082F8B23DAA4A0297D35CA3618A
:10A86000002308F10101009F636341F2B478AA4616
:10A87000CDF804B009E03BF00FFF626B0BEB050174
:10A880002A446263002D00F0C382B14201F1010B42
:10A8900080F291811AF80150606BA6EB0B094044DD
:10A8A0004D4520442A460AEB0B01E4DD4A463BF0C5
:10A8B000F3FE616B236C49446163A5EB09094144D4
:10A8C00021444A4638469847636B314609EB0302F8
:10A8D000D7E715F8083008F101089844002BF8D1A3
:10A8E00015F808204146C1468DE7874905222846CC
:10A8F0003BF0BCFE38B18549052228463BF0B6FE48
:10A90000002840F0EE8094F8BE31B4F8BA212260FD
:10A91000A260C3F302120132A2610599B4F8BC210E
:10A920006260E26094F8BF2181F8B02D1A0681F8C8
:10A93000AF0D00F181800D2104F2C113894640E77B
:10A940005B46A34615F8086008F10109A3EB09046A
:10A9500006F11F02A24227DA09EB06080B2E08D0E7
:10A96000002EEFD15C4615F808209B464146C146B3
:10A9700049E7A94466490193324648463BF076FED2
:10A98000019B0028DED199F80B20032ADAD199F82F
:10A990000C20012AD6D199F80E1099F80D2002EB5F
:10A9A0000122CBF82420CDE708F2B5115944224604
:10A9B00028463BF0A5FE04F5DA71DBF8403000983C
:10A9C000594406F1200298474F4423184FF00009DC
:10A9D000B046C3E70123E361E0E64146A1466C5C73
:10A9E0004E1CABEB060804F11F0343450EDA311988
:10A9F000D9F838303E441BB9C9F83860A9F83C4052
:10AA0000002CECD14C466A5C8946FCE601F2B5119B
:10AA10004944424628463BF073FE08F5DA71494442
:10AA2000D9F84030009804F120029847374408EBE9
:10AA3000000B00262146DBE703F0070303F10108C2
:10AA40004FF0030906F5DA7109FA08F9236C00984A
:10AA500021444A469847059B064493F8B50D0128C2
:10AA600042D804F58D514FF0020C12310CFA08FC5B
:10AA70008C44224692F8C23192F8C1E19B084FEA19
:10AA8000DE0E5B0143EACE2392F8C3E1033243EAD0
:10AA9000DE0300B15BBA21F8023F6145EAD1032130
:10AAA00001FA08F10D3189466B188AE62944059BA5
:10AAB000C87883F8AF0D4E790A7902EB062202EBD3
:10AAC00082025200012AD8BF64222262C00744BF1A
:10AAD0008A7983F8B12D09F10809494615F809204A
:10AAE00091E60823E36159E604F58D504A4604F2E5
:10AAF000C11109F10D0914303BF0CEFD494605EBBB
:10AB000009035EE670690C002C450B0034450B0010
:10AB1000DC420B0003F00703013306F5DA71032270
:10AB20009A4001932144236C009802929847059A19
:10AB300092F8B51D029A0129064404F5A55000F2C9
:10AB40007781019A02239340123003EB000E012318
:10AB500003FA02FC04EB090292F8BF3192F8BE81BD
:10AB60009B084FEAD8085B0143EAC82392F8C081EA
:10AB7000033243EAD80301B15BBA20F8023F8645AD
:10AB8000EAD10CF1FF3303EB430309F10D0903EBA9
:10AB90000908059A012382F8B43D58E60723E361CA
:10ABA000C4F864A0FAE5A36DDB1B1F2B3FF712AFBF
:10ABB0000723E361F2E5DDF804B0E369C4F864B0AB
:10ABC000072B3FF4EBAD059B93F8B23D4FF6FF76B4
:10ABD00001339E4004F5BD53143336B203936368CA
:10ABE000E3626FEA66062368A362B31C9BB201931B
:10ABF00004F5ED530E330025721C069304F57653CD
:10AC00001FFA82FA2E33256320460293FFF7CEF90E
:10AC1000BAF1000F14D02B4604F5ED5004F576552B
:10AC200004F59B412D350C302D3141F2187701F898
:10AC3000013F05F8013F0133534520F8027FF6D16B
:10AC4000CAF580535B000993069BCDF800A003EB87
:10AC50004A03F51C08930026A246059B099A93F81F
:10AC6000B28D08984FF6FF7308F1010941F2177190
:10AC700008F1010803FA09F93BF0F2FEDAF83000B6
:10AC8000039BC8F12002B242B8BF00EBE60003EB21
:10AC90000001B8BFCAF830001F5C4878009B07EB82
:10ACA00000278878C97807EB0047B8BF06F0070689
:10ACB0000FFA89F907EB016727FA06F16FEA09092C
:10ACC00009EA010189B28B42464400F08180504676
:10ACD0000791FFF70FFA019B07998B4200F0A680BE
:10ACE0004FF0010B0BFA08FB534644461FFA8BFB4F
:10ACF00007951FFA85FA98462EE0DA4515D2069B8D
:10AD0000029A23F81A10515C02F80A1033F815E081
:10AD100041F217739E4518BF029B0AF5805C16BF6F
:10AD2000595D02F80C1003F80C100AF101031FFA28
:10AD300083FADA450BD30B2C09D8621C4FEA4B0B74
:10AD40004FEA490994B21FFA8BFB49F001092946E1
:10AD50004046FFF7CFF92946D8F82C50002D27DDC3
:10AD6000C4F12005B54217DAD8F83050039B05EB43
:10AD7000E60503EB050CC8F830505F5D9CF8015008
:10AD800007EB05279CF8025007EB05479CF803509A
:10AD900006F0070607EB056727FA06F5009B09EAA8
:10ADA0000505ADB2AB4226442FD0019BAB42A4D1E6
:10ADB0004446049B13B1049A236A1360D4E9150333
:10ADC000013B9842ACBF002001200BB0BDE8F08FE2
:10ADD000B24213DADAF83020039B02EBE60299184C
:10ADE000CAF830209F5C4A7807EB02278A7807EB85
:10ADF0000247CA7806F0070607EB026727FA06F152
:10AE000009EA010189B2464461E7079DC24624E789
:10AE1000059A01238E42DDE901B782F8AE3D7FF746
:10AE2000CCAE0098636C39449847C6E65446C0E7F8
:10AE300005EB0801143001923BF02EFC019A90447E
:10AE4000A7E600BF2DE9F04F0022164689B06C4BF3
:10AE50006C4C6D48CDE9022235460122196841B19A
:10AE6000D4F80413114204D01D60196800910099B0
:10AE70001643043383424FEA4202EFD1614BD3F8C9
:10AE80007C21F1B2002A6ED00022C3F87C21D3F8D5
:10AE90007C3101934FF0A042019BD2F810255B4B0F
:10AEA0000292D3F81035039300297DD10DF1100AD9
:10AEB00000224FF0FF33564DDFF850810492CAF85C
:10AEC00004200693534C07934FF0000B14F9013FF5
:10AED0005F1C31D0C3F3C20E0EF120020DEB020C49
:10AEE00003F007021CF8086CD640F607D9B203F04D
:10AEF0003F0021D5484F3E18890996F9286057F838
:10AF00002660002E5BD003295BD01F2887BF03F08B
:10AF10001F03C64603464FF0A04E1CF818CC0EEB9C
:10AF200083032CFA02FCD3F800271CF0010FC2F3B4
:10AF300001423CD0022A4FD0A542C7D1BBF1000F3D
:10AF40002FD04FF0A0430299D3F81035D8F8102530
:10AF5000994202D10399914223D0CDE90232DDE931
:10AF600004230692AEE7D1B12B4F01250024A300A4
:10AF700003F180432E4203F5C0430BD0D3F81005F4
:10AF800057F82420D3F81015C0F30520C1F3014170
:10AF900002B190470134082C4FEA4505E7D1002E55
:10AFA00084DB09B0BDE8F08F46F00046DCE7032AF9
:10AFB000C2D1032921D0002EBED0B047BCE703295F
:10AFC000BAD11AF80E704FF0010909FA02F947EAEE
:10AFD00009090AF80E9098E70329ECD14FF4403C98
:10AFE000D3F8002722F440320BF1010B42EA0C02A5
:10AFF0005FFA8BFBC3F80027DDE74FF4003CEFE777
:10B0000000610040006000402061004000030050EB
:10B01000C9110120C71101207011012008B50420B9
:10B0200066F0EEF82DE9F04FD1F80031103B102B0F
:10B030008BB0064600F25681AC4A22FA03F313F0B5
:10B04000010F14BF8A464FF0000A91F804C1351D64
:10B050004FEA0C1C06F114092C46231F0CEB0A00C6
:10B060001A7810F8017B7A4003F8012B9C42F7D143
:10B070000434A1450CF1040CEFD191F80431013BEB
:10B0800006F11002DBB20492AC469A00B6469EF876
:10B090000D309EF809609EF805509EF801409EF81C
:10B0A00002109EF80A008EF80D608EF809509EF886
:10B0B0000E609EF806508EF805408EF801309EF81E
:10B0C00007409EF803308EF802008EF80A109EF8B2
:10B0D0000B009EF80F108EF80B108EF806608EF89D
:10B0E0000E508EF803408EF807008EF80F30714630
:10B0F000002311F823007E4C205C01F8230001336B
:10B10000042BF6D101318C45F2D1960065462B1FF8
:10B110000AEB0600197810F8014B614003F8011B97
:10B12000AB42F7D11D1DA94506F10406EFD1002A57
:10B1300000F0D580CDE905A9CDE907C2F346CDF8E9
:10B1400024E09BF803E09BF800A09BF801809BF8AB
:10B1500002904FEADE164FEADA1706EB460606EBD8
:10B16000C60607EB470786EA4E0007EBC70787EAE4
:10B170004A074FEAD815C0F3C01CC7F3C01205EB4D
:10B1800045050CEB4C0C4FEAD91405EBC50502EB59
:10B1900042020CEBCC0C85EA48058CEA400C00908E
:10B1A00004EB44048AEA080002EBC2028AEA090AB4
:10B1B00082EA47028EEA0A06C5F3C01304EBC40410
:10B1C00084EA490488EA0908029689EA00098EEAB5
:10B1D000000603EB4303C2F3C01003EBC30300EB11
:10B1E000400083EA4503C4F3C01100EBC00080EACD
:10B1F00042008EEA08085FFA87FAC3F3C01E574080
:10B2000001EB4101474001EBC1010EEB4E0E81EA1B
:10B21000440101970EEBCE0EEFB28EEA430E8AEA9E
:10B22000090A87EA08075D40C1F3C018DBB283EA68
:10B230000A0308EB4808434008EBC80888EA4108BD
:10B2400003968EEA0303029E5FFA84F988EA030AF2
:10B25000009B89EA06094C40039EC9B27940DFB2DF
:10B260007740D2B27A405FFA8CF787EA090742400A
:10B270007840CCF3C01707EB47078EEA010107EBD4
:10B28000C70787EA4C0783EA0C0688EA0101019B9D
:10B290008EEA020288EA0000794078407A407740DE
:10B2A00059408EEA05058AEA070388EA04048BF808
:10B2B00003306840049B8BF8001062408BF801005B
:10B2C0008BF802200BF1040B9B457FF43AAFDDE9CC
:10B2D00007C2DDE905A9DDF824E0043AD7E60BB0A2
:10B2E000BDE8F08F4FF0000AAFE600BF010101009A
:10B2F000141F0C002DE9F04F89B0129E002800F0B9
:10B3000047820F4609681D469046824680F016F82F
:10B31000B0F10009C0F201823968494439605046F1
:10B3200080F0B0FC021EC0F27682396811443960A8
:10B33000D8F8000009EB020CA0EB0C00C8F80000E4
:10B34000DAF8B817DAF8B037002956D1002B55D102
:10B350000121CAF8B017D8F80010D7F800E0012989
:10B36000CDE903E9AEEB0C0C704622DD01F1FF3BA9
:10B370004FF0000E03E00EF1010EDE4519D0044639
:10B3800010F8019BB9F1FF0FF5D194F8019009F085
:10B39000E009B9F1E00FEED19CF80000FF2800F0C1
:10B3A000C5800EF1030EA1EB0E01012904F103008B
:10B3B000DCDC4FF0FF32DAF8C817DAF8C4C7CAF895
:10B3C000B4270CFB01F2DAF8BC1701FB02F2002AE9
:10B3D00010DDA91E002021F8020FDAF8C847DAF8BC
:10B3E000C42704FB02F2DAF8BC47013304FB02F283
:10B3F0009342F0DB6FF0020095E04BB1DAF8B4470E
:10B4000050467CF0D1FE2044CAF8CC07D8F80000A2
:10B41000002E00F0BA80DAF8D827CAF8CC07002A44
:10B4200040F05D81904240F35A81CAF8DC073E68E3
:10B4300030443860D8F80020DAF8CC17521AC8F82F
:10B440000020DAF8C41700229142079240F34581A8
:10B45000DAF8DC4703924FEAC4080AF2DC77D146F7
:10B460002C46D9F8BC27002A40F3BD80DDF81CA08B
:10B470000597BB460025374604945646DDF80CA0D8
:10B4800020E05BF8043F43452BDC079F01953E44D9
:10B490009B1BCDF800A048467CF092FE0028C7EB2D
:10B4A000C003D9F8BC17A8EB060805F1010504EBA9
:10B4B0000007C0F2D680079E8D423344A8EB0308F4
:10B4C00080F28E8007AA3946CDE900A5434648465A
:10B4D00080F024F8041EC6EBC4063C4407AA2146AB
:10B4E000CFDAD9F8C427D9F8C807D9F8BC17049D12
:10B4F00000FB02F201FB02F2002ACA4611DD002124
:10B50000A81E0E4620F8026FDAF8C437DAF8C847EA
:10B51000DAF8BC2704FB03F3013102FB03F3994281
:10B52000F0DB6FF0070009B0BDE8F08F94F80190F0
:10B530009CF8010081457FF434AF9CF802B0A078FC
:10B540008BEA000003283FF62CAFDDE903E91BF08E
:10B55000020F18BF04F1FF34A4EB0E04DAF8C81789
:10B56000DAF8C4C7CAF8B447002C0CFB01F0FFF6A8
:10B5700028AFDAF8C017A1444A4401FB02F2D20016
:10B5800092FBF0F2CAF8B8273AE7DAF8CC478442DF
:10B5900000F32181DAF8DC17DAF8D8279142C0F2FB
:10B5A000BF80891A0AF11C06314430463BF0A8F8E6
:10B5B000DAF8D807DAF8CC27396830443BF06CF871
:10B5C000DAF8CC17DAF8D8270A44CAF8DC273A6840
:10B5D0000A443A60D8F80020DAF8CC17521A2EE75D
:10B5E0003E46DDE90447039948467DF007FB002805
:10B5F000D9F8BC27C0F2CF80002A55DDDDF80CA0B9
:10B60000002501E095424FDA2A46514648467EF031
:10B6100031F80028D9F8BC2705F10105F2DAD9F88C
:10B62000C417D9F8C80700FB01F101FB02F2002A98
:10B63000CA4611DD0021A01E0D4620F8025FDAF88F
:10B64000C827DAF8C43702FB03F3DAF8BC27013164
:10B6500002FB03F39942F0DB6FF00A0009B0BDE88A
:10B66000F08FD9F8C427D9F8C807049D00FB02F26F
:10B6700001FB02F2002ACA4611DD0021A81E0E4677
:10B6800020F8026FDAF8C437DAF8C847DAF8BC27CE
:10B6900004FB03F3013102FB03F39942F0DB6FF08B
:10B6A000080009B0BDE8F08FD9F8C817039B03FB69
:10B6B00001F102FB01F104EB410148467FF0B6FDC8
:10B6C0000028D9F8C427C0F2C780039B01339342F6
:10B6D000039307F10807FFF6C4AE002023E7DAF86A
:10B6E000C427DAF8C807DAF8BC1700FB02F201FB3E
:10B6F00002F2002A11DD0021A81E0C4620F8024F9C
:10B70000DAF8C827DAF8C43702FB03F3DAF8BC2703
:10B71000013102FB03F39942F0DB6FF0050002E711
:10B720000AF11C002246084439683AF0B5FFDAF8FD
:10B73000CC17DAF8DC270A44CAF8DC273A680A444E
:10B740003A60DAF8CC17D8F80020521AC8F800206E
:10B75000DAF8C817DAF8C42701FB02F2DAF8BC17E6
:10B7600001FB02F2002A10DDA91E304621F8020F6B
:10B77000DAF8C827DAF8C43702FB03F3DAF8BC2793
:10B78000013602FB03F39E42F0DB6FF00100CAE6D4
:10B790006FF00400C7E6D9F8C417D9F8C80700FB52
:10B7A00001F101FB02F2002ACA4611DD0021A01EB0
:10B7B0000C4620F8024FDAF8C827DAF8C43702FB43
:10B7C00003F3DAF8BC27013102FB03F39942F0DB03
:10B7D0006FF00900A7E6DAF8C817DAF8C42701FB0A
:10B7E00002F2DAF8BC1701FB02F2B24210DDA91E28
:10B7F000304621F8020FDAF8C827DAF8C43702FB1E
:10B8000003F3DAF8BC27013602FB03F39E42F0DBB8
:10B810004FF0FF3087E6DAF8C827DAF8C407DAF81D
:10B82000BC1700FB02F201FB02F2002A11DD00212D
:10B83000A81E0C4620F8024FDAF8C827DAF8C437F9
:10B8400002FB03F3DAF8BC27013102FB03F3994250
:10B85000F0DB6FF0060066E6D9F8C807D9F8BC1728
:10B8600000FB02F201FB02F2002ACA4611DD0021B0
:10B87000A01E0C4620F8024FDAF8C827DAF8C437C1
:10B8800002FB03F3DAF8BC27013102FB03F3994210
:10B89000F0DB6FF00B0046E6012913DD821E431E2C
:10B8A000114401E08B420DD09C4613F8012FFF2A72
:10B8B000F8D15A7802F0E002E02AF3D1C0F1010099
:10B8C000604470474FF0FF30704700BF08B17DF013
:10B8D00023BE704788B338B50D46114604467FF045
:10B8E0002DFD013026D0D4F8D037032B22D1D4F847
:10B8F000B8372B60D4F8BC376B60D4F8C027104938
:10B900001023C5E9022394F8D437D4F8D02703EBE9
:10B910004303013A1344D4F8BC2731F9133002FB36
:10B9200003F32B61D4F8D0376B6194F8D437AB6153
:10B93000002038BD6FF0050038BD6FF0040070477F
:10B94000D85F0C007CF0DEBB10B54FF0804386B0B2
:10B95000D3F80443620703D5D3F80821002A62D143
:10B96000A30605D54FF08043D3F81421002A4FD108
:10B97000600605D54FF08043D3F81821002A3BD14B
:10B98000210604D54FF08043D3F81C214ABBE205C1
:10B9900004D54FF08043D3F82021B2B9A30512D5C6
:10B9A0004FF08043D3F824216AB10022C3F8242148
:10B9B000D3F82421214B0592059A1B68022006B07A
:10B9C000BDE81040184706B010BD0022C3F8202182
:10B9D0001A4AD3F82031049301201368049A984737
:10B9E000DCE70020C3F81C01144AD3F81C31039390
:10B9F0001368039A9847CAE70022C3F81821104A2F
:10BA0000D3F81831029301201368029A9847B7E7D8
:10BA10000020C3F814010A4AD3F8143101931368C3
:10BA2000019A9847A4E70022C3F80821054AD3F8F1
:10BA3000083100931368009A984791E754710120E8
:10BA4000507101204C710120064BD3F800213AB10E
:10BA5000054A00205071C3F8000113689168184727
:10BA6000704700BF009002402C7101200248032261
:10BA7000002135F097B900BF00B000400248042211
:10BA8000012135F08FB900BF0010014002480422A7
:10BA9000022135F087B900BF0040024008B50F4AC7
:10BAA0000F4B934208D2013AD21A22F003020D49F9
:10BAB000043218463AF0F0FD0B4A0C4B934208D280
:10BAC000013AD21A22F003020432002118463AF059
:10BAD000C7FF00F0FBF86BF0E5FC00BFAC060120EF
:10BAE00000000120D0710C00547C0120C006012010
:10BAF0000149024876F04CBA6870012000300040DD
:10BB000002494FF0402076F043BA00BF9C700120FC
:10BB10001D4BD3F8182102B9704700B500211B4A0C
:10BB200083B0C3F81811D3F8181192F8203001919E
:10BB3000FF2B01990FD0917F69B9D17FB1B11F2B34
:10BB400086BF134803F01F034FF0A040012101FA04
:10BB500003F3C0F80C35D2E900E100230D48537718
:10BB60001372734603B05DF804EB18471F2B86BFB2
:10BB7000074803F01F034FF0A040012101FA03F32F
:10BB8000C0F80835E7E700BF003002400870012028
:10BB900000030050107001201F4BD3F8182102B988
:10BBA000704700B500211D4A83B0C3F81811D3F8BF
:10BBB000181192F844300191FF2B019911D092F89D
:10BBC000421071B992F84310C1B11F2B86BF1448BF
:10BBD00003F01F034FF0A040012101FA03F3C0F866
:10BBE0000C35D2E909E100230E4882F8413082F891
:10BBF0002C30734603B05DF804EB18471F2B86BF4B
:10BC0000074803F01F034FF0A040012101FA03F39E
:10BC1000C0F80835E5E700BF00F0024008700120D9
:10BC2000000300503470012070B5234C82B002260E
:10BC3000002501A866F034FC05280BD0019B032BDE
:10BC40002CD01ED8022BF4D101A8257066F028FC58
:10BC50000528F3D1194E4FF40C751948ADF8025070
:10BC60000DF1020166F0A8FBE0B9D6F8B440002C53
:10BC7000F3D0D4E90112246811489047002CF8D180
:10BC8000EBE7A3F10902022AD3D80A2B08D0092B2B
:10BC900014BF0120022076F047F8CAE72670C8E7F3
:10BCA0000020F8E70C2801D002B070BD0549064815
:10BCB0004AF084FD02B070BD407C01205C7101201F
:10BCC000D86D0120D4400B003C450B0008B54FF067
:10BCD0008053D3F83021082A1FD0754AD2F8883013
:10BCE00043F47003C2F88830BFF34F8FBFF36F8FF8
:10BCF0004FF01023D3F80C22D20700F1BB80D3F809
:10BD00000022002AC0F29080D3F80432002BC0F247
:10BD10008B80684B684A1A6008BD4FF08040002154
:10BD2000C0F80C11654AC0F81011C0F83815D3F8E6
:10BD30000414C2F82015D3F80814C2F82415D3F857
:10BD40000C14C2F82815D3F81014C2F82C15D3F827
:10BD50001414C2F83015D3F81814C2F83415D3F8F7
:10BD60001C14C2F84015D3F82014C2F84415D3F8B7
:10BD70002414C2F84815D3F82814C2F84C15D3F887
:10BD80002C14C2F85015D3F83014C2F85415D3F857
:10BD90003414C2F86015D3F83814C2F86415D3F817
:10BDA0003C14C2F86815D3F84014C2F86C15D3F8E7
:10BDB0003411D3F844C4C2F870C5F1B151B14FF099
:10BDC0008043D3F80024D10787D56FF00102C3F870
:10BDD000002482E74FF08053394AD3F830314FF4D2
:10BDE0000071082BC2F840167FF477AF4FF0804304
:10BDF000D3F80024D107E8D46FE7A2F5E042DFF8DA
:10BE0000C8C0C2F88CC602F520424FF0FB0CC2F845
:10BE100018C5D0F8E42ED3F8583263F30302C0F803
:10BE2000E42E0029D6D0CAE7264A0123C2F80435F9
:10BE3000D2F80034002BFBD04FF010231221214AFE
:10BE4000C3F80012D2F80034002BFBD04FF01023BF
:10BE500012211C4AC3F80412D2F80034002BFBD084
:10BE600000231849C2F80435D1F80034002BFBD068
:10BE700001F036FB134A0123C2F80435D2F800342E
:10BE8000002BFBD04FF010210E4AD1F80C3223F0DA
:10BE90000103C1F80C32D2F80034002BFBD0002390
:10BEA0000849C2F80435D1F80034002BFBD0DFE795
:10BEB00000ED00E0000001200090D00300C0004031
:10BEC0000090024000E0014048810300014902481F
:10BED00034F0C0BF5070012000900040014902487A
:10BEE00034F0B8BF5C70012000A000400149024856
:10BEF00076F054BBD0700120002000400149024878
:10BF000076F04CBBF470012000800240002078F0F5
:10BF100069BE00BF094BD3F8002172B100B5084AD1
:10BF200083B052689047054B0022C3F80021D3F834
:10BF300000310193019B03B000BD70470000014038
:10BF400024710120022A2DE9F0431ED0444C02EB5B
:10BF5000C20204EB021404F1480601F144058C34DA
:10BF600000F1240750F8043B54F804C956F804EBD8
:10BF70001A468EFB028241F8042B8CFB0323B84245
:10BF800045F80439EED1BDE8F083354B8268D3F82B
:10BF900038C18CFB02428469D3F8205185FB0464CC
:10BFA00022440A60D3F83C71426887FB0242C469AC
:10BFB000D3F8245185FB046422444A600268D3F814
:10BFC000406186FB0242056AD3F8284184FB05E5FF
:10BFD0002A448A600268D3F84491964689FB0E2E63
:10BFE000026AD3F82C4184FB02827244CA60426820
:10BFF000D3F848E18EFB0242C469D3F8305185FB87
:10C00000048422440A618268D3F84C8188FB02428E
:10C01000D3F83451836985FB03431A444A61436969
:10C020008CFB03238B61036987FB0323CB61C3680C
:10C0300086FB03230B62C36889FB03234B620369FE
:10C040008EFB03238B62426988FB02320023C1E925
:10C050000F33C1E90D33CA624B640B63BDE8F08353
:10C0600030670C002DE9F047B0F85E300446002B35
:10C0700071D0434E434D0F46904646F001064FF0B7
:10C08000000A4FF0010994F8622072B30AF00F031E
:10C090004FF40041194101EA0801002313E01F2A6F
:10C0A00086BF02F01F0228464FF0A04009FA02F2B4
:10C0B000C0F8082594F862200133DBB202EB42029B
:10C0C000B3EB420F0FDA2269D25C0029E7D11F2AB5
:10C0D00086BF02F01F0228464FF0A04009FA02F284
:10C0E000C0F80C25E6E7B4F85E30DB1B53450CDAEC
:10C0F00094F834301F2B86BF03F01F032A464FF0FD
:10C10000A04209FA03F3C2F8083594F861301F2BF6
:10C110008ABF2A464FF0A04203F01F0309FA03F337
:10C12000C2F808354020B04794F861301F2B8ABF11
:10C130002A464FF0A04203F01F0309FA03F3C2F8A6
:10C140000C354020B0470AF1010AB4F85E301FFAFE
:10C150008AF2934297D894F834201F2A07D84FF0D8
:10C16000A04101239340C1F80C35BDE8F087054993
:10C1700002F01F0201239340C1F80C35BDE8F0879F
:10C18000906F0C0000030050054B18680368D3F84B
:10C19000402112B10022C3F8402100F03DBF00BF92
:10C1A00020120120002800F05E822DE9F8430446A9
:10C1B0000069002800F01A8294F8613094F8621047
:10C1C0001F2B8CBFDFF82CC34FF0A04C002900F0D0
:10C1D000F2810FFA81F901EB410149000022C54EBD
:10C1E000884615464FF0010E01E08A4213DA835C5F
:10C1F0001F2B88BF374603F01F0398BF4FF0A0479F
:10C2000001320EFA03F3BC45D2B245EA0305ECD085
:10C210000120BDE8F883B5F1807F34BF00230123FE
:10C22000DB0015F47F0F43F0040218BF134615F42A
:10C230007F4FEAB200F0DF81002A00F0B18143F0C5
:10C240000303012202FA03F341F20802134200F051
:10C25000B48109EB4902022302FA03F81A4694F862
:10C260006310B4F85E6084F8603001238B400736B9
:10C2700006F4FF6684F86630DBB216FB03F694F82A
:10C28000653003FB06F694F8683002FB06F6E664B8
:10C2900003B17600012108EB060061F0C1FA60628B
:10C2A000002800F0A38183193246636100213AF02F
:10C2B000D7FB94F8610094F8603094F86260012133
:10C2C00000F01F0201FA02F28B4245EA020500F07B
:10C2D0009781022B00F0C981C4E90625002284F869
:10C2E00064209EB1D4E904359B5C03F01F0301FA7E
:10C2F00003F345F8223094F86230501CC2B203EBCD
:10C300004303B2EB430FEDDB94F8610094F8653022
:10C3100094F8341094F8665001229A40013A4FF490
:10C320007A43B3FBF5F3B3FBF2F3642B38BF64231A
:10C330001F29C4E914338CBF6E4B4FF0A043002279
:10C3400084F86A2003F5A162A26201F01F010122B4
:10C3500002FA01F194F8442003F20C531F2AC4E9B5
:10C360000B318CBF634B4FF0A04302F01F0103F56C
:10C37000A16503F20C5203461F2B4FF0010000FA97
:10C3800001F188BF03F01F03C4E90F2103F5E07337
:10C3900088BF584AA56398BF4FF0A04240F20331CE
:10C3A00042F8231094F861201F2A86BF02F01F0272
:10C3B00050494FF0A04101239340C1F80C3594F847
:10C3C00034301F2B86BF03F01F034A4A4FF0A042B0
:10C3D00003F5E07340F2033142F8231094F834205F
:10C3E0001F2A86BF02F01F0242494FF0A0410123DD
:10C3F0009340C1F80C3594F844301F2B86BF03F0EE
:10C400001F033C4A4FF0A04203F5E07340F20331B2
:10C4100042F8231094F844301F2B86BF354A03F0AE
:10C420001F034FF0A042012606FA03F3C2F80835B5
:10C4300094F862303BB32F49002340F2033722695E
:10C44000D25C1F2A88BF02F01F020D4602F5E0727F
:10C4500098BF4FF0A0454FF0A04045F822702269E8
:10C46000D25C1F2A84BF02F01F02084606FA02F2BD
:10C47000C0F80C2594F862200133DBB202EB4202D3
:10C48000B3EB420FDBDB47F6FF720C212046FFF7D0
:10C49000E9FD40220D212046FFF7E4FD94F86230CB
:10C4A000C3B11449002301252269D25C1F2A084622
:10C4B0008CBF02F01F024FF0A04005FA02F2C0F854
:10C4C0000C2594F862200133DBB202EB4202B3EB9D
:10C4D000420FE9DB94F86320012000FA02F3023BEB
:10C4E00084F86D30002A6FD0024D0021844640F25E
:10C4F000033714E0000300501F2B86BF03F01F0317
:10C500002A464FF0A0420CFA03F3C2F8083594F81B
:10C5100063200131CBB29A424FEA400054D9A66C55
:10C5200006EB01120B01127B1F2A8CBF2A464FF02B
:10C53000A04202F5A162F250A26C1A44167B1F2E93
:10C540008CBF2E464FF0A04606F20C565660A66CE5
:10C550001E44327B02F01F020CFA02F2B260A26C9F
:10C560001A44127B1F2A86BF02F01F022E464FF08C
:10C57000A04602F5E07246F82270A26C94F86D6055
:10C580001A440642137BB7D11F2B86BF03F01F034B
:10C590002A464FF0A0420CFA03F3C2F80C35B6E776
:10C5A00043F00203DBB2012202FA03F313F48B7FA0
:10C5B00003D0134653E60D46894609EB490204238E
:10C5C0004FEAC2081A464AE694F861301F2B10D889
:10C5D0004FF0A04303F5A16203F20C532046C4E9D7
:10C5E000012300F0A7FC0020BDE8F8830220BDE88D
:10C5F000F8833D4BEEE7002A6CD043F00103D1E70E
:10C6000027693978C1F3C101C4E9062584F86410AB
:10C61000002E3FF47BAE3A78606902F01F0203FA05
:10C6200002F2C900CA40027094F8622002EB420292
:10C630005200012A7FF768AE1D46226994F8641003
:10C64000D25C606902F01F0205FA02F2C900CA401A
:10C65000C25494F862200133DBB202EB4202B3EB26
:10C66000420FEADB50E60320704727693B78C4E9B4
:10C670000625C3F3001284F86420002E3FF446AE72
:10C680003B78606903F01F0301FA03F31201D34002
:10C69000038094F8623003EB43035B00012B7FF7C8
:10C6A00033AE0A460D46236994F864109B5C6069BA
:10C6B00003F01F0305FA03F30901CB4020F8123001
:10C6C00094F862300132D2B203EB4303B2EB430F72
:10C6D000E9DB19E6012202FA03F313F48B7F3FF43E
:10C6E000B3AD1346BBE500BF0003005090F86030C7
:10C6F000012B05D0022B01D000F000B900F046BAA2
:10C7000000F000B82DE9F04F8FB090F86830446A1F
:10C7100003910546924633B190F86A30C26CC3F17A
:10C72000010302FB034495F86560062E00F0E080EB
:10C73000C6F10503DBB24FF4006202FA03FC4022AB
:10C7400002FA03F1012202FA03F095F86670002F55
:10C7500000F0CB80B5F85E30D5F814B0CDF82CC021
:10C7600000220492DA1D4FEAD208C3EBC80354FA40
:10C7700083F20AF1FF3300241BB208948E4609931A
:10C78000A94634465146002C00F085800023CDE9AF
:10C790000CE0CDE905230B9DCDF828808246F446B8
:10C7A000079399F967000028B8BF4042013840B2AA
:10C7B000421C55D0059C039B01FB00F607FB06F6C7
:10C7C00010F0010E03EB860607FB01F36ED099F91A
:10C7D0006720002A74DB002900F08480049A164444
:10C7E00006EB43070022CDE9000904EB01080291A2
:10C7F00036F8121037F8120011EA050318BF9BF83B
:10C80000003011EA0C0F1CBF9BF8019043EA0903AA
:10C8100011EA0A0F1CBF9BF802100B4328421CBFF1
:10C820009BF803100B4310EA0C0F1CBF9BF804107D
:10C830000B4310EA0A0F1CBF9BF805100B4304F8CA
:10C84000013B7244444512B2D2D1DDE9000902999C
:10C8500099F86670431E58B2431CACD199F86540F4
:10C86000079B4FEA4C0C002B38D1052C36D94FF0E2
:10C87000010A4FF40065069B059A0A980133069356
:10C88000DBB202EBC002A3420592079389D3DDE934
:10C890000CE0DDF82880089B01330893DBB29F424F
:10C8A00023D9049B03EB410304936CE70029D1D007
:10C8B000049A164406EB43074FF0010E002292E75C
:10C8C00081B1089A013FBF1A01FB07F706EB470742
:10C8D000099A07EB43064FF0FF3E84E76D004FEAED
:10C8E0004A0AC8E7431E58B265E70FB0BDE8F08FAB
:10C8F000102020214FF4004C27E700BF2DE9F04F16
:10C9000095B09246059190F868104569436AC26CEB
:10C910000E9061B1014690F86A0091F86010B2FB88
:10C92000F1F1C0F1010000FB01F103EB81030E986E
:10C9300090F86510B0F85E40062900F02081C1F142
:10C940000501C9B24FF4006088401090402000FA01
:10C9500001F6012000FA01F7184600213AF080F8AC
:10C9600003460E9890F86220002A00F0FD80E11D39
:10C970004FEAD10CC4EBCC01C9B205F1180B03EBA3
:10C9800081050AF1FF339BB20021119390F8669064
:10C9900004910133069331460895CDF834C0B9F1BE
:10C9A000000F00F0D8800E9ACDF83CA0002392F83A
:10C9B000652007930B930B46002A00F0BB80BDF95E
:10C9C00044100C91CDE9123700244946DDF840802F
:10C9D000DDF83890DDF83CC009949A46BE460A94CA
:10C9E00099F9674084EAE473A3EBE473013B5BB21B
:10C9F000581C00F08480089E2746604687EAE7724C
:10CA0000049CA2EBE772D2B204FB023200FB02F2FA
:10CA1000059C01FB02F213F0010504EB820201FB0D
:10CA200000F451D0002F58DB002800F0A5800799B2
:10CA3000571807EB440C0022CDE90290CDE90036EF
:10CA400031462C4606EB800637F812903CF812501F
:10CA500019EA080318BF5BF8183C19EA0A0F1CBF53
:10CA60005BF8140C034319EA0E0F1CBF5BF8100CA3
:10CA7000034315EA080F1CBF5BF80C0C034315EACF
:10CA80000A0F1CBF5BF8080C034315EA0E0F1CBF0E
:10CA90005BF8040C034351F8040B224418438E4204
:10CAA00012B241F8040CCFD1DDE90290DDE9003685
:10CAB000069A99F8661006EB8206013B5BB25A1C97
:10CAC0001AD099F9677099E70028F6D00799571896
:10CAD00007EB440C01250022AEE700284CD00B9D4B
:10CAE0000139491B00FB01F102EB410C0CEB44073F
:10CAF0000C9A4FF0FF359FE799F8652084460A9B12
:10CB00004FEA4A0A002B32D1052A30D94FF0010EE4
:10CB10004FF40068099B08980D9C01330993DBB220
:10CB200000EB4410934208900A93FFF459AFDDE9FB
:10CB3000123789460B9907980F9C01310B91C9B2A6
:10CB400000EB4400894507903FF636AF19460E9B2F
:10CB500093F86220A246049B01330493DBB29A420D
:10CB60000BF1180B3FF61BAF15B0BDE8F08F4FEA85
:10CB700048084FEA4E0ECDE7013B5BB23EE74FF46B
:10CB80000041102720261091E6E600BF2DE9F04F66
:10CB900095B04569059190F868101092466AC26C8C
:10CBA000834659B190F86A009BF86010B2FBF1F12E
:10CBB000C0F1010000FB01F106EB41069BF8651096
:10CBC000BBF85E40062900F01E81C1F10501C9B223
:10CBD0004FF4006000FA01F340200E9300FA01F3D5
:10CBE00001200F9300FA01FA0021304639F038FF96
:10CBF0009BF86220002A00F0FC80E31DDF08C4EBF4
:10CC0000C703DBB206EB4304109B9BF866800894D5
:10CC1000013B1FFA83FC002304930CF10103CDF8C0
:10CC200044B00693644605F10C0B0D97404600286E
:10CC300000F0D680119991F86530002207920B928E
:10CC40001A460B461099D046002A00F0BA80DDE95A
:10CC50000E594FF0000C26B2C246CDF848800C9613
:10CC6000CDF824C01394CDF828C0884693F9677096
:10CC700087EAE771A1EBE77101394CB2611C00F062
:10CC800084800899049A87EAE776A6EBE776F6B2FD
:10CC900002FB064608FB06F6059A00FB06F614F0B2
:10CCA000010C02EB860600FB08F251D0002F5ADB84
:10CCB000B8F1000F00F0A4800798064406EB420785
:10CCC0000022CDE90041CDE9023801EB480E0846CB
:10CCD00036F8121037F8124011EA050318BF3BF876
:10CCE0000C3C11EA090F1CBF3BF80A8C43EA08030D
:10CCF00011EA0A0F1CBF3BF8081C0B432C421CBF57
:10CD00003BF8061C0B4314EA090F1CBF3BF8041C3C
:10CD10000B4314EA0A0F1CBF3BF8021C0B4330F80C
:10CD2000021B62440B43864512B220F8023CCFD16D
:10CD3000DDE90238DDE90041069A93F8660001EB6F
:10CD40004201621E54B2621C1DD093F9677099E7CC
:10CD5000B8F1000FF5D00798064406EB42074FF0F4
:10CD6000010C0022ADE7B8F1000F49D0471E0B9827
:10CD70003F1A08FB07F706EB470707EB42064FF0A1
:10CD8000FF3C0C9A9DE793F865200A994FEA490900
:10CD9000002931D1052A2FD94FF0010A4FF400653F
:10CDA0000999089C0D9E01310991C9B204EB061442
:10CDB000914208940A91FFF459AF4146139CDDF863
:10CDC00048800B9D079E01350B95EDB206EB4106A1
:10CDD000A84207963FF638AF119B93F86220C246EF
:10CDE000049B01330493DBB29A420BF10C0B3FF628
:10CDF0001EAF15B0BDE8F08F6D004FEA4A0ACFE7CD
:10CE0000621E54B23EE74FF400432020CDE90E30BD
:10CE10004FF0100AE8E600BF90B110B500F0AAFA92
:10CE20000446406A08B160F013FCA06C08B160F0E1
:10CE30000FFC206918B160F00BFC0023236110BDCA
:10CE4000704700BF2DE9F04182B09DF82C409DF85D
:10CE500024609DF830709DF834E09DF838C09DF94D
:10CE60003C500194002857D0109C002D08BF01258C
:10CE7000002C51D00446052B28BF0523002D84F833
:10CE8000675084F86520B8BF6D42019A84F861202C
:10CE9000EDB203EB4302052E109884F83470A4F829
:10CEA0005C104FEA420215FB01F137464FF00005D6
:10CEB00028BF05272060A4F85E10D0B284F844E0B3
:10CEC00084F868C084F86230A564656284F8637091
:10CED0000121804660F0A4FC206130B301213801BB
:10CEE00060F09EFC0346A0642069CBB108994246DD
:10CEF00039F0D2FB66B10A9B591E2B46A26C11F881
:10CF0000015F02EB03120133D8B287421573F5D8E3
:10CF1000002002B0BDE8F081032002B0BDE8F0813E
:10CF2000019360F095FB019B2361022002B0BDE8F4
:10CF3000F08100BF00286BD070B590F8662090F8A3
:10CF40006530511E013B82B0012A80F86B3080F8B9
:10CF50006C1088BF90F86C3090F863104FF00002AE
:10CF60008CBF03F1FF33012380F86D3080F86E2011
:10CF7000826500293DD04FF0010C264940F2033470
:10CF8000E64612E01F2B86BF03F01F030D464FF04D
:10CF9000A0450EFA03F3C5F8083590F86350013246
:10CFA000D3B29D424FEA4C0C23D9836C03EB02139E
:10CFB00016011B7B1F2B86BF03F01F030D464FF08E
:10CFC000A04503F5E07345F82340836C90F86D505D
:10CFD000334415EA0C0F1B7BD4D11F2B86BF03F003
:10CFE0001F030D464FF0A0450EFA03F3C5F80C35AC
:10CFF000D3E7019000F030FA0198036801224FF462
:10D000007A715A60DA60C3F840151A6002B070BDD8
:10D01000704700BF000300502DE9F041836B026CA4
:10D020001A60D0E90B321A60836A026B1A600368D7
:10D03000A54F01265E6003685E64D3F84435C26A7A
:10D0400090F86B30016B1160054603F0FF08374321
:10D050003BBB90F863104446F9B195F86C3095F8F5
:10D060006D2053401E424FEA041010D0AA6C95F870
:10D070006CC002EB04131CEA060F996814BF135826
:10D080005B684FF400701960B84795F8631001347D
:10D09000E3B299424FEA4606DFD895F86C3085F83E
:10D0A0006D3095F86B3095F865200133DBB29A420C
:10D0B00085F86B300DD8002285F86B2095F86C3020
:10D0C00095F866100133DBB2994285F86C3040F276
:10D0D00098802A6D2B6802FA08F101225A604020DC
:10D0E000DA60C3F840151A60B847D5E90F321A6004
:10D0F000B5F85E2095F86C1095F865C095F86B3022
:10D1000095F860E007320CFB0133D610D10895F892
:10D110006820C9000EFB03F301FB03F322B195F86D
:10D120006A20E96C01FB02336A6ABEF1010F02EB6F
:10D130000307D5E90640D5E9013100F0C780F2B216
:10D14000561EBEF1020FF6B26CD0002A41D007EB9A
:10D15000461607F12002403652F8207C1F601C6002
:10D1600000BF00BF086052F81C7C1F601C6000BF3D
:10D1700000BF086052F8187C1F601C6000BF00BF31
:10D18000086052F8147C1F601C6000BF00BF08607C
:10D1900052F8107C1F601C6000BF00BF086052F88E
:10D1A0000C7C1F601C6000BF00BF086052F8087C48
:10D1B0001F601C6000BF00BF086052F8047C1F6045
:10D1C0001C6000BF00BF2032B2420860C4D195F895
:10D1D00065C0BCF1010F12D995F86B307BB92A6894
:10D1E000012353642B6DD2F84425C3EBC3031344CE
:10D1F00004336A6DDB08934238BF13462B65BDE8E4
:10D20000F08185F86C2095F86E303BB195F86A3066
:10D21000C3F1010385F86A3085F86E20AB6D0133E8
:10D22000AB6556E7002AD4D007EB061607F11002CB
:10D2300006F1200795F8646003EB460632F810CC3F
:10D24000A6F800C01C6000BF00BF086032F80ECC1A
:10D25000A6F800C01C6000BF00BF086032F80CCC0C
:10D26000A6F800C01C6000BF00BF086032F80ACCFE
:10D27000A6F800C01C6000BF00BF086032F808CCF0
:10D28000A6F800C01C6000BF00BF086032F806CCE2
:10D29000A6F800C01C6000BF00BF086032F804CCD4
:10D2A000A6F800C01C6000BF00BF086032F802CCC6
:10D2B000A6F800C01C6000BF00BF10329742086093
:10D2C000BCD195F865C084E7906F0C00002E80D02B
:10D2D000013EB6B207EBC60607F1080206F11007D9
:10D2E00095F864601E4412F808CC86F800C01C60F3
:10D2F00000BF00BF086012F807CC86F800C01C60B1
:10D3000000BF00BF086012F806CC86F800C01C60A1
:10D3100000BF00BF086012F805CC86F800C01C6092
:10D3200000BF00BF086012F804CC86F800C01C6083
:10D3300000BF00BF086012F803CC86F800C01C6074
:10D3400000BF00BF086012F802CC86F800C01C6065
:10D3500000BF00BF086012F801CC86F800C01C6056
:10D3600000BF00BF083297420860BCD195F865C085
:10D370002FE700BF002860D0436A002B5DD010B4B7
:10D3800090F86E30002BFBD102684FF0010CC2F810
:10D3900004C00268C2F844C0816BD2F84425026C14
:10D3A0000A6090F86220C2B1244903F0FF030269C9
:10D3B000D25C1F2A0C468CBF02F01F024FF0A04423
:10D3C0000CFA02F2C4F80C2590F862200133DBB2AB
:10D3D00002EB4202B3EB420FE9DBB0F85E3023B35D
:10D3E000164C00224FF0010C90F861301F2B2146A3
:10D3F0008CBF03F01F034FF0A0410CFA03F3C1F8F8
:10D40000083500BF00BF90F861301F2B21468CBF4C
:10D4100003F01F034FF0A0410CFA03F3C1F80C35E1
:10D42000B0F85E3001329A42DED3836A026B1A6032
:10D43000D0E90B321A6010BC7047704700030050EF
:10D4400090F8683033B1012380F86E3090F86E3078
:10D45000002BFBD1704700BF1E4A0368934212D0D5
:10D4600002F5805293422ED002F5805293422CD086
:10D4700002F5803293422AD002F58052934208BFCF
:10D48000042201D070470022134B03EBC20100209D
:10D4900091F9041053F832304FF4803C012281425C
:10D4A0005A60C3F80405DA60C3F80805C3F810052C
:10D4B000C3F804C3E6DB4809084B01F01F018A40AA
:10D4C00043F8202070470122DEE70222DCE7032236
:10D4D000DAE700BF00800040986F0C0000E100E038
:10D4E000BFF34F8F0549064BCA6802F4E06213434D
:10D4F000CB60BFF34F8F00BFFDE700BF00ED00E042
:10D500000400FA05014B1868704700BF5000012065
:10D5100007EE900AF5EEC07AF1EE10FA01D400F0B1
:10D5200009B808B580F0004000F004F8404261EB13
:10D53000410108BD70B5FAF787FB0C4B0022044689
:10D540000D46FAF791FCFAF7BBFD0646FAF75AFBCF
:10D55000074B0022FAF788FC02460B462046294674
:10D56000FAF712FAFAF7ACFD314670BD0000F03D53
:10D570000000F04110EE101A21F000430122B3F137
:10D58000FF4FF0EE407A026015D2002B72D000B54A
:10D59000B3F1E45F87B013D20029BEBF4FF0FF3371
:10D5A0000360B1EE400A37F00FF9B1EE407AB0EE09
:10D5B000470A07B000BD20EE007AB0EE470A704778
:10D5C00000295EDBB3F17E5F68D0B3F1804F65D098
:10D5D0004A0000F19F809FEDDD6ADD4A934240F2F0
:10D5E000A382DC4A934240F24A82F0EE005A75EE82
:10D5F000E75A9FEDD67A9FEDD85ADFEDD86ADFED76
:10D60000D84A9FEDD84A65EEA57AE7EE856AA7EE7F
:10D61000A44A9FEDD55ADFEDD54AA6EEA75AE4EE0F
:10D62000274ADFEDD36A9FEDD34AE5EE276AA4EEE1
:10D63000A74A9FEDD15ADFEDD14AA6EEA75AE4EEF4
:10D64000274ADFEDCF6AE5EE276A9FEDCE5AA4EEBA
:10D65000A75A66EEA56AB6EE004AE5EE276AF0EE36
:10D66000667AE5EEC47A37EE877A00299FDA36EEDD
:10D67000477A9CE7DFEDB57AF7EE006A86EEA77A87
:10D680009BE7B3F1964F0CD3DFEDB07AF7EE006A6B
:10D6900086EEA77AB0EE470A07B000BD9FEDAB7AE1
:10D6A00085E7B3F17A5FC0F05982B1EE407A8DED33
:10D6B000020AB0EE470ACDE9041003938DED017A1A
:10D6C0002FF0D8F89DED017ADDED027A059AB4EEDF
:10D6D000407AF1EE10FADDE9033140F09A819FEDD6
:10D6E000AA7A37EE677A17EE100A00F0010007EE0B
:10D6F000100AB8EEC77A8000CDE901310492CDED71
:10D70000037A062800F28A82DFE800F05DDFDF5945
:10D7100059ECEC00B3F1824F80F09B819FED8B6A56
:10D72000DFED9A6ADFED9A5ADFED9A4ABDEEE77AAD
:10D73000B8EEC75A17EE103A77EEC57A9FED965AB3
:10D74000E7EEA65A033BA7EEA45ADFED946ADFED9D
:10D75000944AE5EEA76AE5EE274ADFED925A9FED7F
:10D76000925AE6EEA75AA4EEA75ADFED906ADFEDD3
:10D77000904AE5EEA76AE5EE274ADFED8E5A9FED67
:10D780008E5AE6EEA75AA4EEA75ADFED8C6AE5EEB4
:10D79000A76AF7EE005AE5EE275A66EEA76AF6EE9C
:10D7A000004A86EEA57AA7EEA47A042B3FF65DAF79
:10D7B000DFE813F0C900AC00270118012A01F7EED9
:10D7C000006A36EEC77A9FED7E0ADFED600A27EE2B
:10D7D000000A002000F06AFFDDE90131DDED037A87
:10D7E000049AF1EE406AF5EE406AF1EE10FA3FF469
:10D7F0004BAF27EEA67A9FED720ACDED026AB0EE2E
:10D80000C77A80EE070ACDE903310592CDED017AA2
:10D8100036F0DAFFDDED026ADDED017AF5EEC06A81
:10D82000F1EE10FADDE90331B0EE407A03D5059A46
:10D830004FF0FF301060B3F17E5F3FF4B8AEB3F14C
:10D84000804F3FF4B4AE4800F1EE677AB0EE476A1D
:10D850007FF5C3AEB3F1824FFFF462AFB0EE670A5B
:10D860008DED036A0291CDED017A36F0ADFFDDED6D
:10D87000017A9FED542ADFED542A9FED543ADFEDF3
:10D88000543A9FED544ADFED544A9FED547A029981
:10D890009DED036AF7EE006A86EEA75AF6EE005A8F
:10D8A00077EEE55A65EE057A70EE666AE7EE822A53
:10D8B000A2EEA73AE3EE273AA3EEA74AE4EE274A00
:10D8C000A4EE857AA5EEA67ACFE6F6EE006A36EEED
:10D8D000C77A9FED3B0ADFED1D0A27EE000A00F034
:10D8E00029FB79E7F7EE086A37EE667A9FED340A8E
:10D8F000DFED160A27EE000A00F01CFBDDE901311E
:10D90000DDED037A049AF0EE406A6CE7F7EE006A08
:10D91000B0EE080A37EE800A20EE260AF0EE006A22
:10D9200077EEA67A8DED037A27EE800A8DED026AF6
:10D93000019136F049FF9DED037A01999DED026A50
:10D9400037EE007A91E6B7EE000AE7E70000000044
:10D950006666663F17A6DD3FA283D33767976739B0
:10D96000752C3C384584E238A1549C3A34B6053ACB
:10D970007E02F23BC66E3D3B01F0893D1599A83C05
:10D980003F239E3D661AA53E0000004B67FF053809
:10D99000B435F13ABDD7F536D6EE4B3AE440DA3C31
:10D9A00054BF983CE6DC153E6E0F303E7ACCA63E66
:10D9B000C5D0383F5A245C3E3B2DB23F3F239EBD2D
:10D9C000DB0F4940E8C4D5BAD23D5B3A5C061CBACD
:10D9D000FD0C503A610B36BBABAAAA3D1D7FD63E6B
:10D9E00000000000F7EE006AF1EE045A77EEA55A47
:10D9F00065EEA65AF1EE006A77EEA66A66EEA56AB3
:10DA000086E7F7EE005AF5E7F1EE086A77EEA66AC8
:10DA1000EAE7F6EE006A27EE267ACDE90231B0EEAB
:10DA2000470ACDED047A8DED017A2EF023FF9DEDAE
:10DA3000017A059A37EE407ADDE9023137EE077A4E
:10DA4000F0EE477AFEEECF7A17EE900ADDED047A1B
:10DA500052E6B3F1B94FC0F097808DED020A8DED1B
:10DA6000010A36F0B1FEB7EE007A30EE477ADDED0E
:10DA7000027A1FED256A019927EE277AF5E5724AA9
:10DA8000934240F28480DFED716A9FED717A77EE08
:10DA9000E66A66EEA62A9FED6F4ADFED6F5ADFED6C
:10DAA0006F4A9FED6F5ADFED6F3A9FED6F3A62EE6E
:10DAB000A67AE7EE844AA7EEA55A9FED6C4ADFED01
:10DAC0006C5AA4EEA74AE5EE275ADFED6A4A9FEDAD
:10DAD0006A5AE4EE274AA5EEA75AA7EEA33ADFED6D
:10DAE000675A9FED674ADFED673AA5EE274AE4EEF5
:10DAF000A75AE3EE273ADFED644A9FED645AE4EE5D
:10DB0000265AE3EEA74ADFED626A9FED624AE5EE30
:10DB1000E76AA4EEA75AF0EE667AD2EE857A77EE3F
:10DB2000C47A37EE877AA0E5B0EE670ACDE9023114
:10DB30008DED046ACDED017A36F046FE564A029B21
:10DB4000DDED017A03999DED046A9342B1EE407ACE
:10DB50005CD9F7EE005A75EEE75A4CE59FED4F0A97
:10DB6000DFED3B0A0293CDE9031027EE800A002087
:10DB7000CDED017A00F09AFDDDE90231DDED017AAB
:10DB8000049AF0EE406A2EE69FED316A66E6B7EE43
:10DB9000007A77EEC77A9FED2E7A9FED415ADFED3E
:10DBA000416ADFED415ADFED414AE7EE856AE7EE73
:10DBB000A54A9FED3F5ADFED3F5AA6EEA75AE4EE85
:10DBC000A75ADFED3D6ADFED3D4AE5EE276AE5EE57
:10DBD000A74A9FED3B5ADFED3B5AA6EEA75AE4EE6B
:10DBE000A75ADFED396AE5EE276AB7EE005AA5EECF
:10DBF000A75A66EEA76AFEEE004AC6EE855AF0EE18
:10DC0000656AE7EEA46A36EE877A2EE52F4A9342DC
:10DC1000C3D9DFED2F6A77EEE66A3AE7F0EE006AE5
:10DC200037EE667A9FED1D0ADFED090A27EE000A3E
:10DC3000002000F03BFDDDE90131049ADDED037ABF
:10DC4000F1EE406ACFE500BF1FA69D3FC316BB3F64
:10DC50000000000027F9A3B9F7E9AF3967F8663A81
:10DC600085300DBA6B7BA53976F4B7BAFE7771BBF8
:10DC70009916143B3D37933CFEFC28BC3C2117BE53
:10DC8000155A843D07E7C73B474D06BD5EB9F73ED1
:10DC9000521CE631CDCDF83D1F4A3B3FDB0F4940DA
:10DCA0005E3C5B3C78756A3EDBD5523BAF72D53D3E
:10DCB000B24B7A3FDFEF443FE73ABA3F2D39084095
:10DCC000F400223FBE2E1D403F239EBD07336D3E14
:10DCD0000C5BEC3E10B510EE104A884A24F000436D
:10DCE000934288B0014662D9854A934222D824F0F3
:10DCF0000043002CDFED837A834A23F00F0340F3C7
:10DD0000E380934230EE670A09BFDFED807A9FED32
:10DD1000807A9FED807A30EE670A70EE477A30EEB7
:10DD2000670AC0ED007A30EE470A80ED010A012053
:10DD300008B010BD784A934240D89FED787A9FEDA5
:10DD4000716AB0EEC00AF6EE007AE0EE077A9FED57
:10DD5000707AFDEEE77AF8EEE76A17EE900AA6EE23
:10DD6000C60A1F2866EE877A30EE677A6BDCDFF82A
:10DD7000C0C100F1FF3E24F000425CF82EC022F04A
:10DD8000FF0262455FD081ED007A30EE470A002C39
:10DD900030EE670A81ED010ACADAB1EE477AB1EED8
:10DDA000400A81ED007A81ED010A4042C0E700237C
:10DDB00080ED000A4360002008B010BDB3F1FF4FB2
:10DDC00072D2DA15863AA3EBC25307EE903ABDEE53
:10DDD000E77ADFED536AB8EEC77A77EEC77A8DED52
:10DDE000057A67EEA67ABDEEE77AB8EEC77A77EEE7
:10DDF000C77A8DED067A67EEA67AF5EE407AF1EEF7
:10DE000010FACDED077A5DD1B5EE407AF1EE10FA59
:10DE100056D10123434801900220009005A80391A8
:10DE200000F00AF9002C039982DA91ED007AD1ED25
:10DE3000017AB1EE477AF1EE677A81ED007AC1EDB1
:10DE4000017A404274E717EE102AC2F3C752C2EBC0
:10DE5000D352082A97DD9FED2D7ADFED2E5AB0EED2
:10DE6000406AA6EEC76A70EE467AE6EEC77AD6EE4C
:10DE7000A57A36EE677A17EE102AC2F3C752C2EBC4
:10DE8000E353192B17DD9FED287ADFED285AB0EE0A
:10DE9000460AA6EEC70A76EE407AE6EEC77AD6EED6
:10DEA000A57A30EE677A6EE730EE400A80ED010A1F
:10DEB00080ED000A7FE7B0EE460A81ED007A64E764
:10DEC0000223A7E70323A5E7934230EE270A09BF01
:10DED0009FED0E7ADFED0E7ADFED0E7A30EE070A57
:10DEE00030EE277A30EE470A80ED007A70EE277A1E
:10DEF000C0ED017A4FF0FF301AE700BFD80F493F5D
:10DF0000E3CB1640800FC93FD00FC93F00443537DF
:10DF10004344353708A3852E800F494384F9223FB7
:10DF200000008043F8220C0000A3852E32318D249E
:10DF300078220C0010EE103A23F00043B3F1485F52
:10DF40002CD2FDEEC07A17EE903A002B60D060EE36
:10DF5000007A9FED317A9FED315ADFED315A9FED16
:10DF6000316ADFED316AA7EE875A9FED307AE7EE2E
:10DF7000855AA7EEA56AA7EE867AE7EE876A66EE6F
:10DF8000A76A60EEC00AB6EE007AE7EEA60AB7EE20
:10DF9000000AD7EE870A30EE600A704760EE007A1A
:10DFA0009FED1D7A9FED1D5ADFED1D5A9FED1D6AF5
:10DFB000DFED1D6A1E4AA7EE875A93429FED1B7A3A
:10DFC000E5EE275AA5EEA76AA6EE277AE7EE276ABE
:10DFD00066EEA76AD5D9174A934214D803F17F4356
:10DFE00007EE103AB7EE006A36EE476A60EEC00AF6
:10DFF000F6EE005A97EEA57AE7EEA60A37EE607ABB
:10E0000036EE470A7047B6EE076AB5EE027AEDE7DC
:10E01000B7EE000A704700BF4ED747ADF6740F3118
:10E020007CF293B4010DD037ABAA2A3D610BB6BA8E
:10E030009999993E0000483F2DE9F04F2DED048B52
:10E04000DBB01C4696460493689ACD4B1EF1040F34
:10E0500053F8225081468B4604F1FF38C0F24682C5
:10E06000BEF1030348BF0EF10403DB100393013339
:10E07000DB000693069B15EB0800AEEB030218D4F9
:10E08000039B9FEDC37A699C0130A3EB08031844FE
:10E090001EA9002BA4BFE65C07EE906A03F1010302
:10E0A000ACBFF8EE677AF0EE477A8342E1EC017A92
:10E0B000EFD1002DC0F2D98204981EAC04EB80048D
:10E0C000002346AF8100464605EB000CB8F1000F77
:10E0D00080F2AC810136664547F8043B04F1040444
:10E0E000F4D109ABCDE907BE0DF1280A03EB850396
:10E0F0009FEDA49ADFEDA48A059309EB01040AEBD6
:10E10000850746AE019510460DEB8503002D93ED76
:10E11000460A4FEA850B16DD06EB0B03524660EE0E
:10E12000097AB0EE407AFDEEE77A73ED016AF8EE17
:10E13000E77AB342A7EEE87A37EEA60ABDEEC77AD1
:10E14000A2EC017AEBD1029063F014FFB0EE408AAA
:10E15000B4EE000A28EE000A2EF08CFBF2EE007AF4
:10E16000A0EE678A02980028FDEEC89AF8EEE97AD8
:10E1700038EE678A69DD691EC0F108035AF821E0AC
:10E180004EFA03FC0CFA03F3AEEB030EC0F10702E8
:10E1900019EE903A4EFA02F26344002A09EE903AE0
:10E1A0004AF821E000F3D980B5EE408AF1EE10FA8A
:10E1B0005CD1019B9D420CDD0AEB0B0300219446D0
:10E1C00053F8042DBB4241EA0201F9D1002940F085
:10E1D0004381019B013B05F1010C5AF82330002BD0
:10E1E00040F02281059B012153F8042D0131002AC2
:10E1F000FAD02944699B039A03EB020E049BAE44B8
:10E200001D441EAB03EB850547AB9B441EF8013F45
:10E2100007EE903AF8EE677AB8F1000FE5EC017A74
:10E22000DFED5B7A09DB2A464B46F3EC016A32EDFF
:10E23000017AA342E6EE877AF7D10CF1010C8C4506
:10E24000EBEC017AE2DD0D465EE700F0D680F6EEFB
:10E25000007AB4EEE78AF1EE10FA80F24C81B5EE66
:10E26000408AF1EE10FA4FF00002A2D0DDE907BEBD
:10E27000069B0295B0EE480A019D0190A3EB0E00AB
:10E28000914663F077FE9FED407AB4EEC70AF1EE57
:10E2900010FADDE90123C0F2AF81DFED3A7A60EEDA
:10E2A000277A5C1CFDEEE77A0832F8EEE77AA7EEF3
:10E2B000C70AFDEEE77ABDEEC00A10EE101A4AF862
:10E2C000231017EE903A4AF824301046B7EE000AB1
:10E2D00063F050FE002CB0EE407AC0F2B8810AF133
:10E2E000040347A9DFED276A03EB840301EB8401F4
:10E2F000A20046AF73ED017AF8EEE77A534567EE78
:10E30000877A27EE267A61ED017AF3D10DF1C80EF6
:10E310001744F44626460020002DC0F2B480DFF8F2
:10E320006C80DFED1B7A3946002307E0F8EC016AC8
:10E33000B1EC017A9D42E6EE877A03DB834203F17A
:10E340000103F3DD013E711CCCED007A00F0A680E4
:10E350000CF1040C0130043FE1E70133002D09EE1C
:10E36000903A40F36A8151464FF0000E51F8043B59
:10E37000002B3CD0C3F5807341F8043C0FE000BF94
:10E380006C220C000000803B0000804340220C0007
:10E39000000000000B68C3F1FF0341F8043B0EF1DD
:10E3A000010E7545F6DC4FF0010E00280BDD01284B
:10E3B00000F09480022806D1691E5AF8213003F03B
:10E3C0003F0C4AF821C0022A7FF4EEAEB7EE000AF5
:10E3D00030EE488ABEF1000F3FF4E6AE099202909B
:10E3E00063F0C8FD0298099A38EE408ADCE60EF127
:10E3F000010E7545BADC9E46D7E76B1E5AF82320FE
:10E400001212002A7FF7D0AE19EE903A002D03F1D8
:10E41000010309EE903AA6DC022A7FF4C5AEF7EEBE
:10E42000007A37EEC88ABFE66146E3E609EB0100F1
:10E430005FED297AA2464B46F3EC016A3AED017A88
:10E440008342E6EE877AF7D101366645E7EC017A3A
:10E4500004F10404ECD144E66C1E59465AF8243009
:10E46000019DDDF81CB0E146A0F10802002B7FF40D
:10E470002CAF0B4609A90B4453F8041D013C083A84
:10E480000029F9D021E70023013E4CF8043B731C1E
:10E4900000F10100A7F104077FF43EAF689B022B57
:10E4A0005FDC002B38DC10D10EF104035FED487AFD
:10E4B000134433ED017A734577EE877AF9D1B9F1D8
:10E4C000000F40F0B780CBED007A19EE903A03F0E0
:10E4D00007005BB0BDEC048BBDE8F08F691E5AF8F5
:10E4E000213003F07F0C4AF821C06CE70823069323
:10E4F00000230393BEE519EE903A002D03F10103CA
:10E5000009EE903AC8BF02223FF72DAFF7EE007A2E
:10E5100037EEC88A022247E60EF10401DDED327AB9
:10E520001FED657A0A4472ED016A724537EE267A6C
:10E53000F9D1B9F1000F74D177EEC77A8BED007A7B
:10E5400064B10123B1EC017A01339C4277EE877A02
:10E55000F8DAB9F1000F01D0F1EE677ACBED017A6C
:10E56000B3E7689B032BB0D1002C00F08D800EEB3D
:10E57000020090ED007A0346014671ED017AF0EE5B
:10E58000476A37EE277A714577EEC77A81ED007AD0
:10E5900077EEA67AC1ED017AEFD1012C74D090ED1F
:10E5A000007A0EF1040173ED017AF0EE476A37EE5E
:10E5B000277A994277EEC77A83ED007A77EEA67ACA
:10E5C000C3ED017AEFD15FED8E7A8B180EF1080E54
:10E5D00033ED017A9E4577EE877AF9D1DDED326A27
:10E5E0009DED337AB9F1000F0ED1CBED006A8BEDC2
:10E5F000017ACBED027A68E7BDEEC00A1C4610EE48
:10E60000101A4AF8231060E6F1EE666AB1EE477A16
:10E61000F1EE677ACBED006A8BED017ACBED027AF1
:10E6200053E7F1EE476A77EEC77ACBED006A002C2C
:10E6300087D191E7F1EE677A45E7012818D00228E3
:10E640007FF4EAAE0EF03F034AF82130E4E6689B1F
:10E65000022B15DC002B1ADC7FF437AF5FEDB47AA8
:10E66000B9F1000F3FF42FAFE4E7049B990038E5C0
:10E670000EF07F03022A4AF821307FF495ADCEE6F2
:10E68000689B032B7FF421AF5FEDBF7AA6E7DDED3A
:10E69000327AB9F1000F04D04FF00043CBF80030CC
:10E6A0005AE70023CBF8003058E700BF10EE103ACD
:10E6B00023F00043B3F1485F04D2FDEEC07A17EEB9
:10E6C000903A5BB360EE007A9FED157ADFED155A54
:10E6D0009FED156ADFED156AE7EE875A9FED147A14
:10E6E000A5EEA76A20EE275AE6EE276AA6EEA77ADD
:10E6F00030B9DFED106AE7EE876AA6EE850A70474B
:10E7000027EE457AF6EE006AA0EEA67ADFED0A6AF9
:10E71000D7EE270AE5EE260A30EE600A704700BF02
:10E72000D3C92E2F342FD7B21BEF3836010D50B975
:10E730008988083CABAA2ABEABAA2A3E10EE103A42
:10E7400023F00042B2F1465FF0EE407A10D2BDEE07
:10E75000C07A17EE101A01BB431C134300F0A080CF
:10E76000012800F09C80BFEE007A87EE270A7047F0
:10E770004F498A4211D39FED4F7ADFED4F6A002B4C
:10E78000BCBFF1EE600AF1EE407A77EE677A36EEC2
:10E79000E07ADFED4A0A77EE277A67EEA76ADFEDC7
:10E7A000484ADFED485A9FED485A9FED486A404974
:10E7B00026EEA67A8A42E7EE245AA7EE056ADFED36
:10E7C000444A9FED445AE5EE874AA6EE075ADFED2C
:10E7D000425A9FED426AE4EE875AA5EE076ADFEDE2
:10E7E000404A9FED405AE5EE874AA6EE075A9FED54
:10E7F0003E6ADFED3E5AA4EE876AE5EE075AB0EEB8
:10E80000467AA5EEA67A27EEA65AB0EE606AA7EE83
:10E81000056ADFED374AE6EE260AE5EE240A37EE12
:10E82000A00A1ED201283AD0BFEE007AC7EE006AD5
:10E8300010EE103A6FF30B0306EE103A16EE903A14
:10E8400076EE677A6FF30B0300EE103A70EEE70A8C
:10E85000F7EE007AE6EE007AE0EE807AA7EEA60AFE
:10E86000704707EE100AF8EEC76A20EE007A30EE25
:10E87000260A9B1787EE006A03F00203C3F1010327
:10E88000F0EE005A36EE606A07EE103A77EEC67A7E
:10E89000B8EEC77AE7EEE56A26EE870A704770475A
:10E8A000F0EEC07AB7EE007A87EE270A704700BF15
:10E8B00040A12C3FDA0F493F6821223300000000BD
:10E8C0005FAE9BB745F4A3388453D9377AC09538E7
:10E8D000C8261A3AB937813916696B3B48DEBE3A09
:10E8E000A427B33C1F37113C8988083ED10D5D3DFC
:10E8F000ABAAAA3E42084B0802F0553203F055334A
:10E90000801AC91A8A08830801F0333100F03330C5
:10E9100002F0333203F033330344881803EB13134C
:10E9200000EB101003F00F3300F00F30184400EB31
:10E93000002000EB0040000E704700BF2DE9F047BB
:10E9400082B00646DDF828E00846B4460D46002BA6
:10E950004ED18A4214466DD9B2FA82F242B1C2F166
:10E960002003954026FA03F394401D4306FA02FC67
:10E97000260CA7B2B5FBF6F14FEA1C4306FB115576
:10E9800043EA054301FB07F0984209D9E31801F176
:10E99000FF3580F00381984240F200810239234420
:10E9A0001B1A1FFA8CFCB3FBF6F006FB10334CEA83
:10E9B000034C00FB07F363450AD914EB0C0C00F180
:10E9C000FF3580F0ED80634540F2EA80A4440238D0
:10E9D00040EA0140ACEB030C0021BEF1000F04D073
:10E9E0002CFA02F30022CEE9003202B0BDE8F08733
:10E9F0008B4209D9BEF1000F01D0CEE900610021A0
:10EA0000084602B0BDE8F087B3FA83F11746002943
:10EA10004DD1834202D3B24200F20F81B6EB070C14
:10EA200060EB030301201D46BEF1000FDDD0CEE9EF
:10EA300000C5DAE7002A00F098801A46B4FA84F399
:10EA4000002B40F0AF800B1B270CA6B20121B3FBBB
:10EA5000F7F54FEA1C4007FB153340EA034306FB7A
:10EA600005F8984507D9E31805F1FF3002D298451B
:10EA700000F2E8800546A3EB08031FFA8CFCB3FB09
:10EA8000F7F007FB10334CEA034C06FB00F3634539
:10EA900008D914EB0C0C00F1FF3602D2634500F2EA
:10EAA000CE803046ACEB030C40EA054095E7C1F15F
:10EAB00020058B4022FA05FC4CEA030C00FA01F415
:10EAC00026FA05F3E84002FA01F943EA04084FEA9E
:10EAD0001C4206FA01FAB0FBF2F71FFA8CF602FBB1
:10EAE00017004FEA184444EA004407FB06F0A0422E
:10EAF0000AD91CEB040407F1FF3380F09C80A0428C
:10EB000040F29980023F6444241A1FFA88F3B4FB50
:10EB1000F2F002FB104443EA044300FB06F69E4277
:10EB200009D91CEB030300F1FF3480F082809E4280
:10EB30007FD90238634440EA0740A0FB09749B1B5D
:10EB4000A3423E46A04664D361D0BEF1000F0AD076
:10EB5000BAEB060263EB080303FA05F5CA40154356
:10EB6000CB40CEE9005300213FE7730843EAC1736D
:10EB70004A08190C41EA02414FEAC67C9BB2B2FB3B
:10EB8000F4F02646A04627461F2243EA0143B1FB84
:10EB9000F4F1A3EB080341EA004158E72946FFE6F8
:10EBA000284615E71A46C3F120019C4026FA01F3D6
:10EBB00020FA01F190400343270C06FA02FCB1FB56
:10EBC000F7F0A6B207FB1015190C41EA054100FB4E
:10EBD00006F58D423BD9611801D28D4220D8491BE0
:10EBE0000138B1FBF7F5019505FB06F8019D9BB2D5
:10EBF00007FB151143EA0143434526D2E31805F10B
:10EC0000FF31C6D24345C4D2A91E2344C1E7BA4549
:10EC10009BD2B7EB090664EB0C040138A04694E7DD
:10EC2000651B29440238B1FBF7F5019505FB06F891
:10EC3000DCE720467FE71F4666E70846F4E6A44483
:10EC400002382FE7023D234415E70199A1E7491B4C
:10EC5000B1FBF7F5019505FB06F8C7E770B590F82D
:10EC60002A30DC0657D4054640F21C500E4647F0C9
:10EC7000B3FD044688B1436830469847A368012134
:10EC80009B6906469847002847D1A36805F108010B
:10EC900030469B68BDE8704018472349304640F035
:10ECA000A7FD0446C0B190F85030D90635D443F0E2
:10ECB000100305F1080180F8503029F04DFD95F85A
:10ECC0002A3013F00C0F204618BF0121BDE8704018
:10ECD00008BF002129F030BD1449304640F088FDBE
:10ECE0000446E8B190F82A309A0716D443F002039C
:10ECF00005F1080180F82A3028F034FD95F82A3013
:10ED000013F00C0F204618BF0121BDE8704008BF6A
:10ED1000002128F0D7BC0EF051FD054873F056FFD6
:10ED2000044873F053FF00BF18E70B00E4E40B0046
:10ED3000248D0B00148D0B0010B5144684B01A609E
:10ED400030B1104600215EF06BFD98B104B010BDEB
:10ED5000084603A9019364F0F5FE019B20B90398CE
:10ED6000002801DD1860EDE7186800215EF058FD0D
:10ED70000028EBD1014620465EF052FD0028E5D187
:10ED8000092062F03DFA00BF12F0FEBD2DE9F84FF8
:10ED9000834608462A4940F02BFDD0F808A0BAF176
:10EDA000020F4AD9D0F80C80DBF8040001224FEAA8
:10EDB0008A012FF0DFFA00240746CBF80440ABF8B5
:10EDC0000840254658F825001E4940F2075238F001
:10EDD00079FE58F8256040F207527068022138F039
:10EDE000EFFDB06840F2A26138F0C0FE40F2A263CD
:10EDF00047F6FF721449814638F0D2FDF0684FF4AF
:10EE0000D56138F0B3FE01344FF4D5630E4947F6AF
:10EE1000FF720646A4B238F0C3FD07EB85035445E4
:10EE200027F825905E802546CCD34FEA4A0ACBF8D6
:10EE30000470ABF808A0BDE8F88F044873F0B2FE88
:10EE4000D45B0B00C4670B000080FFFFB48A0B008B
:10EE50002DE9F0472DED028B1C4696B0C368BDF836
:10EE60008470BDF88C600546B0EE408A8A46002B5F
:10EE700000F0D18041688B4200F014818E4B1878ED
:10EE80004FF00008FF2885F8458013D0019263F009
:10EE90009DFA2946814689480AF004FA39F00803A8
:10EEA000019AC5F80C8085F84480484602D00EF0DF
:10EEB000DBFB019A1F2F66D9BAF1000F40F0A48046
:10EEC000002E40F0D68025964FF00A09002A00F067
:10EED0008F8040F20123ADF83830002C00F099808B
:10EEE000631C0DF13808ADF83A30404600230F930B
:10EEF00063F08EFA0346002B3FD1DFED717A9FED70
:10EF0000716A259A099228EE277A229A0D93C7EE04
:10EF1000067A9E4208BF1A4622920692209A0492CE
:10EF2000694A089302FB04F4684A0B93A2FB042489
:10EF30000122640BF6EE006A77EEA67A8DF8352092
:10EF4000FCEEE77A082241461846ADF81470ADF899
:10EF50001C608DF820900C93CDED0A7AADF82C4012
:10EF600001930CF0F9F800285BD1534808AA04A9D2
:10EF700063F028FA0346002861D0184616B0BDECAD
:10EF8000028BBDE8F0871F2E3BD8BAF1000F75D079
:10EF9000259B002B00F08C801B799DF80810F0EE6B
:10EFA0000C7A03F07F03B4EEE78A63F34701F1EED6
:10EFB00010FA259B8DF8081066D807EE904A9FED51
:10EFC000447AF8EE677AF4EEC77AF1EE10FA5BD87D
:10EFD000D3F80530CDF80930259BB3F80930ADF8EA
:10EFE0000D3002AB25934FF00209002A7FF471AF78
:10EFF0000DF138084046CDE90E2263F009FA0346C8
:10F0000079E7BAF1000F34D0002325934FF00609B9
:10F010005CE7234665E71F2F80F845303FF64CAF8D
:10F02000B1E7C2B20199404663F0E0F90346002817
:10F030009BD0184616B0BDEC028BBDE8F0871E4C85
:10F040001E492A4605F128000AF002F921789DF9A7
:10F050009020012063F0E6F9034600288DD1207846
:10F06000012163F0B1F90346002886D1209AEA60B5
:10F0700083E7CDF894A04FF0080927E7A6B1CDF8B3
:10F0800094A04FF0040921E7D3F80530CDF80930FA
:10F09000259BB3F80930ADF80D3002AB25934FF046
:10F0A000030913E7112368E725964FF005090DE7DB
:10F0B0004FF001090AE700BFA7060120C1170300AE
:10F0C0000024744900401C4440420F005917B7D136
:10F0D0006666A63F38B5DFED117A416020EE270A5B
:10F0E0000446BCEEC00A049D80ED020A11461A4691
:10F0F0009DF8143084F820300C3062F0DFFA35B11E
:10F10000224628460649BDE838400AF0A1B8214603
:10F110000348BDE838400AF067B800BF00007A44F1
:10F12000E1D40300F0B583B0416017464A68044655
:10F1300090790A9A84F82C0022858D7D05F030069E
:10F1400005F0060500283DD14FF6FF72E284002E3F
:10F1500044D1089BE36194F82C20099B236200238F
:10F1600084F82D3084F82A30A3840B9BDAB1002B6D
:10F170003BD02349224618460AF06AF85EB116F0E1
:10F18000040118BF012160681ABF84F82B10002207
:10F19000012213F0ADF925B1AA060ED5022384F899
:10F1A0002B3003B0F0BD2BB31649224618460AF0A7
:10F1B0004FF8002DF5D06B07F0D5012384F82B30E4
:10F1C00003B0F0BD4A680193D0680AF0EDFE324604
:10F1D0002E46019BE0841546002EBAD01A463946C9
:10F1E00004F1080062F06AFAB3E70548214609F025
:10F1F000FBFFC3E70348214609F0F6FFD9E700BF4C
:10F2000015BE08008DBE08002DE9F0414FF6FF76CF
:10F2100082B003610023154681608371C360C271AF
:10F2200004468680084601A90BF07AFB681C221D63
:10F2300001A9C0B263F014F9074618B1384602B00C
:10F24000BDE8F0810F4AA5881388DFF84080AB4203
:10F2500028BF2B4613800C4A1388AB4238BF2B467D
:10F260001380044638F81400B0422A46294601D0DB
:10F2700063F0FAF84434B4F5AA7FF3D1384602B00B
:10F28000BDE8F081A4060120B4790120A80A01207C
:10F290002DE9F04F89B081461D4640689DF84880B1
:10F2A0008A46164658F048FC002D4FD088F00108D9
:10F2B000DFF8ACB04FEA4818002701E02D1B45D01D
:10F2C000B5F5806F2C46424628BF4FF4806403A9F1
:10F2D0004846CDE90667CDE904478DF80C708DF8F6
:10F2E0000DA001F03BFE58452644E7D00190D9F827
:10F2F000040058F003FC184A019B934219D00BD923
:10F30000164A934210D0013A23F00203934218D0D8
:10F31000002009B0BDE8F08F043A93420ED16FF09F
:10F32000730009B0BDE8F08F6FF0120009B0BDE8BE
:10F33000F08F6FF00F0009B0BDE8F08F03329342F9
:10F34000E6D16FF0040009B0BDE8F08FD9F80400F1
:10F3500058F0D4FBDCE700BF0B00AD0B0100AE0B97
:10F360000000AD0B2DE9F04F85B0804601920C46B0
:10F37000002A40F03D8201F10C06D4F800A03AF0DA
:10F38000A9FE98F800204046002A77D04FF00009E7
:10F390005746CB46292A5BD05E2A00F2EB81232A0E
:10F3A0003FD9243A3A2A3CD8DFE812F0A6013B00C4
:10F3B0003B003B005B013B001C01FA003B003B00B3
:10F3C000DB013B003B003B003B003B003B003B00C4
:10F3D0003B003B003B003B003B003B003B003B0055
:10F3E0003B00B0013B003B003B003B003B003B00CF
:10F3F0003B003B003B003B003B003B003B003B0035
:10F400003B003B003B003B003B003B003B003B0024
:10F410003B003B003B003B003B00B10074003B0065
:10F420006B002768002E00F091827A1C2260012276
:10F43000F2552268511C216098F80010B1544546DD
:10F440006268013262606A7805F10108002AA1D180
:10F450004046BBF1000F0DD02268A2EB0B02013A2F
:10F4600051B2914218BF49F001095FFA89F90EB112
:10F4700006F80B20B9F1000F40F0B68105B0BDE8E9
:10F48000F08F2268571C2760002ED8D05021B1542D
:10F490002768D4E798F80120002A00F0A5812768A2
:10F4A00042F02001642908F1010507F1010000F094
:10F4B000FD8142F02402772A00F0F881002E00F04E
:10F4C000488201222060F255226898F80110531CEE
:10F4D000A1F1610023603244152800F2F481DFE8D5
:10F4E00010F076027302F201F201F2016D02F201F4
:10F4F000F201F201F201F201F201F2017002F201F5
:10F50000F201F2016702F2016A02F201F10198F8D8
:10F51000012027685E2A07F1010300F0F28108F15B
:10F520000105002E00F01B8203222360F2552268A1
:10F530000132226062680132626098F801205D2A1F
:10F5400000F048824FF0000E5C2A00F06581002A2E
:10F5500000F04A81294648782D2800F0BC812068B7
:10F56000002E00F0C181451C256032542268501CD9
:10F5700020600878B0544A785D2A01F101050EF147
:10F58000010EE1D14FFA8EF2724518BF49F0010920
:10F590005FFA89F9002E3FF456AF06F803E052E710
:10F5A0002268BA4200F0208198F801103F2900F04B
:10F5B000C881002E00F0DE8145466221B1542268E8
:10F5C000BF1A0132023FB75479B2B94218BF49F0AD
:10F5D000010922685FFA89F9971C62682760013285
:10F5E000626030E72268BA4200F0FE8008F101054F
:10F5F000002E00F04181B81CD21BF119304437F0C5
:10F600007FF82268023260212260B15420683A1AE1
:10F610003044023A427020680230206098F80100BD
:10F620004FFA82FC944518BF49F001093F280CBFEE
:10F6300062226122F255226807F10101A2EB070262
:10F64000A2F10202725450B218BF45462768904298
:10F6500018BF49F001095FFA89F9626802326260F5
:10F66000F1E698F8012027683F2A00F06081A2683F
:10F67000531C5A0051B2914218BF49F00109A360CE
:10F680005FFA89F9002E00F06781791C21607E21E4
:10F69000F1552168481C2060725462680132626032
:10F6A00001220292019A039308F101002146FFF71B
:10F6B00059FE0546002800F097800278292A40F07C
:10F6C0009380029B002B3FF4BEAE039B5A00013295
:10F6D00051B2914218BF49F001095FFA89F92168D6
:10F6E000002E00F05681481C20607E207054216856
:10F6F000481C20607254A3E62268571C2760002E25
:10F700003FF49DAE5121B154276898E62268BA4271
:10F710006AD008F10105002E00F09C80B81CD21BB5
:10F72000F119304436F0ECFF22680232226098F87A
:10F7300001203F2A0CBF62226122F255226807F1A4
:10F740000101A2EB0702A2F10202725450B218BFEB
:10F750004546904218BF49F0010927685FFA89F9C8
:10F760006EE627687A1C2260002E3FF468AE022203
:10F77000F25564E67C2A7FF454AE2268BBF1000F98
:10F7800038D0A2EB0B01013948B2884218BF49F0CA
:10F7900001098EB306F80B10226806EB0A050AF180
:10F7A00002002946A2EB0A02304436F0A9FF236882
:10F7B000F1186020033323608870D4F800B0612210
:10F7C0000BF10101216006F80A202268A2EB0A026F
:10F7D000023A51B26A70914218BF49F00109276894
:10F7E0005FFA89F9454638E7002005B0BDE8F08F9B
:10F7F0000026C2E5002ED0D1171D02F1030BA7EBA6
:10F800000A02023A51B2914218BF49F00109276039
:10F810005FFA89F9454620E76A7842F020006428BB
:10F8200005F101016BD042F02400772867D0A2F1E6
:10F83000610015280CD8DFE800F0AAA80B0B0B5EBE
:10F840000B0B0B0B0B0B0B5C0B0B0B5A0B480B60D6
:10F850000D467CE602322260D11B174698F8012043
:10F8600002393F2A18BF45464AB28A4218BF49F0BA
:10F8700001095FFA89F9E3E5111DC81BBA1A043AB8
:10F88000023821600F464FFA80FC51B2844508BF10
:10F89000914214BF0122002249EA02025FFA82F972
:10F8A00098F801203F2A18BF4546D6E6002E50D0D2
:10F8B00005222060F2552268511C216098F8011041
:10F8C000B154BDE50B211170BAE548782D284FF0F1
:10F8D00009027FF444AE88785D283FF440AE20688A
:10F8E0000231002E7FF43FAE0230206043E60D224D
:10F8F00031E60A222FE60C222DE60B222BE600220F
:10F900002DE6002E48D004222360F25522680132F1
:10F91000226062680132626098F802205D2A08F174
:10F92000020508BF4FF0000E7FF40CAE32E698F8E7
:10F9300002203A2A7FF49BAE002308F102080293CA
:10F94000B0E608F101054EB3612137E6BA1C22602A
:10F9500075E5BA1C226073E5BA1C22609DE66268F8
:10F9600001326260BA1C226098F801205D2A7FF49F
:10F97000E9AD68E5BF1A023F79B2B94218BF49F054
:10F98000010945465FFA89F926E60822E3E50722E0
:10F99000E1E50231216053E51A46B8E7B91A0239A8
:10F9A00048B2884218BF49F001095FFA89F913E6A5
:10F9B0000D21117044E50921117041E50C211170F0
:10F9C0003EE50A2111703BE50821117038E5072159
:10F9D000117035E54FF0000EDFE500BF08B502F00D
:10F9E000C1F908B1012008BD02F0B2FB70B902F004
:10F9F000E3FB68B9074B1868C20705D4C303F1D409
:10FA0000800C00F0040008BD052008BD022008BDE0
:10FA1000032008BDA4750120034B53F8203013B117
:10FA20009A6801329A60704714260120114B53F8EE
:10FA30002000F0B1017942791F298ABF0E4B4FF0A7
:10FA4000A04301F01F01D3F810351F2A23FA01F358
:10FA50008ABF09494FF0A04102F01F02D1F81015EA
:10FA600003F00103D1405B0001F00101194366F08E
:10FA700033BA70473C3C0120000300502DE9F04FA1
:10FA8000ABB0044603910020214646F0A5FE0028B5
:10FA900000F03083012120463DF044FB4268CDE96F
:10FAA0000C4200230E938DF86030082104A877F0F3
:10FAB000B9FD0023CDE90A33DDE90C040EAB0122C8
:10FAC00018A9A0470E9B002B40F02C83002800F0C3
:10FAD0006C819DF86090DFF8F082DFF8F0B20026CC
:10FAE0003446B2464D46002D00F066810EAB0C98B0
:10FAF0000D9F012218A9B8470E9B002B40F01283DE
:10FB000008B98DF860007D2D00F256815A2D40F223
:10FB10005F815B3D222D00F24F81DFE815F036005A
:10FB20004D0123004D014D014D014D014D014D0190
:10FB30004D014D01F6004D014D014D014D014D01AD
:10FB40004D014D01B2004D014D014D014D014D01E1
:10FB50006B004D014D014D014D014D014D01540012
:10FB60004D012300002C00F027810A9B002B00F0A0
:10FB7000DC82013B0B9A0A9352F82340204641F065
:10FB8000F7F982469DF86050ADE70021084643F042
:10FB900015F8054694B18A4B9A451DD0002E00F009
:10FBA0000B8131462A46204640F016F90B9B002671
:10FBB000CBB1214608A842F091FB284641F0D8F984
:10FBC0002C468246DEE7002042F0C2FD0546002CAE
:10FBD000F4D07B4B9A45E1D12946204642F07EFB8A
:10FBE0000B9B002BE5D1012108A842F0BBFB0B9B2E
:10FBF0001C60E2E79DF86030722B40F0DD800EABB8
:10FC00000D9D0C98012218A9A8470E9B002B40F0CF
:10FC10008982002800F0CD809DF86030752B40F07F
:10FC2000CB800EAB0D9D0C98012218A9A8470E9B06
:10FC3000002B40F07782002800F0BB809DF86030F8
:10FC4000652B40F0B9800EAB0D9D0C98012218A9D0
:10FC5000A8470E9B002B40F0658208B98DF8600024
:10FC6000002C00F01C82564B9A4500F02D82002E8D
:10FC700000F005823E223146204640F0ADF80026D5
:10FC800080E79DF86030752B40F096800EAB0D9D9F
:10FC90000C98012218A9A8470E9B002B40F0428225
:10FCA000002800F086809DF860306C2B40F0848046
:10FCB0000EAB0D9D0C98012218A9A8470E9B002B96
:10FCC00040F03082002874D09DF860306C2B73D1E6
:10FCD0000EAB0D9D0C98012218A9A8470E9B002B76
:10FCE00040F0208208B98DF86000002C00F0CF8130
:10FCF000334B9A4500F0E381002E00F0C2810E22C2
:10FD00003146204640F068F8B9E79DF86030612B35
:10FD100052D10EAB0D9D0C98012218A9A8470E9B3D
:10FD2000002B40F0FF81002843D09DF860306C2B01
:10FD300042D10EAB0D9D0C98012218A9A8470E9B2D
:10FD4000002B40F0EF81002833D09DF86030732BFA
:10FD500032D10EAB0D9D0C98012218A9A8470E9B1D
:10FD6000002B40F0DF8120B39DF86030652B23D15C
:10FD70000EAB0D9D0C98012218A9A8470E9B002BD5
:10FD800040F0D08108B98DF86000002C00F08F8120
:10FD90000B4B9A4500F09D81002E00F06E811E22D3
:10FDA0003146204640F018F869E78DF8600081463A
:10FDB00091E600238DF86030024872F007FF00BF23
:10FDC000D45B0B0040770B000020FF030110000400
:10FDD0003A2DF1D81F2D40F24A81A5F12002D2B26E
:10FDE0000123934013EA080F40F0AB8013EA0B03A2
:10FDF0007FF4C8AE222DDFD19DF860100593354603
:10FE00000029D9D022297BD05C2913D004A877F00F
:10FE100097FA0EAB0D9E0C98012218A9B0470E9BC5
:10FE2000002B40F07F8110B19DF86010E8E78DF85D
:10FE30006000C1E70EAB0D9E0C98012218A9B047D7
:10FE40000E9B002B40F06E8118B98DF860000146C2
:10FE5000DCE79DF86010A1F16203132BD6D801A254
:10FE600052F823F0C5FE02000DFE02000DFE020056
:10FE70000DFE0200C1FE02000DFE02000DFE02009A
:10FE80000DFE02000DFE02000DFE02000DFE02003E
:10FE90000DFE0200BDFE02000DFE02000DFE02007E
:10FEA0000DFE0200B9FE02000DFE0200B5FE0200CA
:10FEB000C9FE02000921A9E70D21A7E70A21A5E74C
:10FEC0000C21A3E70821A1E74FF0000904260EAB9F
:10FED0000C980D9F012218A9B8470E9B002B40F0EB
:10FEE0002181002840F0A3808DF86000C923013EE5
:10FEF00043EA0919EBD1494604A877F04BFA88E7A1
:10FF00000EAB0C982E4601220D9D18A9A8470E9BFA
:10FF1000002B40F0078108B98DF86000DDE905107D
:10FF200042F0F8FE0246002C51D0834B9A4500F077
:10FF30009780002E00F08780314620463FF04CFF2E
:10FF40009DE6002305939946294604A877F0F8F921
:10FF50009DF86050452D15D82A2D15D9A5F12B03F4
:10FF60001A2B11D8DFE803F014101423101010100E
:10FF70001010101010101010101010101010101081
:10FF800010102300652D12D0284672F0D9FC88B1DC
:10FF90000EAB0C980D9F012218A9B8470E9B002BA1
:10FFA00040F0C0800028CFD18DF86000CCE74FF042
:10FFB0000109EDE70346DDE90510B9F1000F44D072
:10FFC0001A46009345F0A0FF0246002CADD19146A1
:10FFD00040F0CEFF039BDBB99DF8600072F0D8FCC7
:10FFE00088B10EABDDE90C04012218A9A0470E9BD5
:10FFF000002B40F097800028EED18DF8600072F061
:020000023000CC
:10000000C7FC0028EDD19DF86030002B7FF4D4AE02
:10001000B9F1000F3FF4D0AE0A9B002B7FF4CCAEB9
:1000200004A877F07FFA48462BB0BDE8F08F9DF822
:10003000602042F02002A2F13003DBB2092B84BF22
:10004000573AD3B253E716469CE50A224B4646F090
:100050008DF80246002CBAD0374B9A457FF469AF31
:100060001146204642F03AF9DFF8CCA08AE50A2D85
:1000700009D8082D3FF686AD9EE61E2682E53E266F
:1000800080E50E267EE50D2D3FF47CAD94E60E2036
:1000900040F06EFF039B4BBB4FF00E099CE73E20E8
:1000A00040F066FF039BCBB94FF03E0994E71E205A
:1000B00040F05EFF039BABB94FF01E098CE70E21A9
:1000C000204642F00BF9CFE73E21204642F006F9E8
:1000D000CAE71E21204642F001F9C5E70A9B4FF00E
:1000E0003E099AE70A9B4FF01E0996E70A9B4FF0DC
:1000F0000E0992E70FAA20467E2100260027CDE9AF
:1001000016673EF0AFFA0D4A0D4B129201214022C4
:10011000CDE913120CAC1AA912AACDE90C43159122
:100120001192C2E4184672F0F9FC039BA146002B21
:100130007FF476AF50E700BFD45B0B00604F0B003D
:10014000CD1E06000288112A0B4608D0362A0BD194
:1001500019B181889A89914208D0012070474FF6E1
:10016000FF71012299811A740020704700B5C2887E
:1001700083B0DA81C289009300F11001586882428D
:1001800028BF02461868019236F086FADDE900328F
:10019000012101209A60197403B000BDC207034613
:1001A00020D400B510F0030283B00BD1114A0168CE
:1001B00091421AD0184640F0DBFE5E22C1880E48FC
:1001C00072F0F8FC022AF5D10C4A0240062AF1D05E
:1001D00040F0DAFDFCEEC07ACDED017A9DF8040026
:1001E00003B000BDC0F34700704740F09BFEC0B2B3
:1001F000F6E700BFAC5A0B0050830B00070080FFEE
:1002000070B588B014460DF11E030DF11F02CDE943
:1002100000320E460DF11D0307AA214604460EF0DA
:1002200053F99DF81C209DF81D300B49059220467E
:1002300004939DF81E409DF81F503FF0D9FA03909B
:100240003FF0D4F9CDE90045DDE9043203983146A9
:100250005CF0F0FB08B070BDCCC10B002DE9F04F95
:100260000446E1B0674812F08FFD031E029321DBC4
:10027000654F7B88B3F57F7F80F0B2801A1DA24264
:100280001CD85A1E3C1D6148A15C614D2F290BBF33
:1002900000230022A354E25407A92BF087FB286017
:1002A00010B16BF0F9F868B940F2513302983B8015
:1002B00062F032FE002061B0BDE8F08F012061B035
:1002C000BDE8F08F582200210AA836F0C9FB286843
:1002D00007990AAA6BF0A0F80023C7E90133FB6075
:1002E00040F25113054644F8043C00287ED120AE6C
:1002F000CDE9000003464FF4807231460AA8F8F7B2
:10030000FFFE002878D18246044608E0CDE900448B
:1003100031460AA8F8F7F4FE0AF1010A28B9317843
:1003200000234FF480720029F0D10AA86BF09EF8E8
:10033000C7F808A0BAF1000F42D04FF000090DF144
:10034000200B06AB00934FF480720DF11703CDF82C
:1003500004B031460AA8F8F7D3FEDBF800209DF878
:1003600017303A61099AC7F804907A61002B34D1AA
:10037000069AFB603046BA6169F0F8F80546788065
:10038000029862F0C9FDBDB10024A046CDF80C90E2
:10039000A5EB0409B9F1040F28BF4FF00409311986
:1003A0001848CDF8008000234A464C4412F0CAFD9C
:1003B000A542EDD8DDF80C9009F10109D145C0D175
:1003C0000AA86AF0B1FF0023BA6802987B807A60BD
:1003D000FB60BB6162F0A0FD6CE701230022C8E76F
:1003E00040F251233B8062F097FD63E703230298BC
:1003F0007B7062F091FD5DE70AA86BF037F8BD6095
:10040000DEE700BF28450120184801201C480120D4
:10041000A046012038B52B4A2B4B04460121106819
:100420001D6857F05BFA294A02F1200C52F8043F8C
:1004300013B11979A14202D06245F7D138BDDA79FA
:100440001ABB5A699969AA1A411AC2EB02420A44B4
:100450004FF6FF718A4228BF0A46D9891C8AA4B286
:1004600014FA81F19C89B1FBF4FC04FB1C119C681B
:1004700024F811201A8A998992B28A4218D21A8ACB
:1004800001321A825D61986138BD1F2C88BF104A05
:10049000597994BF4FF0A04204F01F04D2F8102500
:1004A000E24002F001029142ECD00022DA71E9E769
:1004B000DA8992B20132B2FBF1F401FB1422DA8143
:1004C000E0E700BF3C770120747501200C0A012091
:1004D000000300502DE9F04110F8017C0578A7F1E8
:1004E0000306B6FA86F67609CDB18846841C06E086
:1004F00000F01CF880B9013D04F102040FD014F89B
:10050000013C41462046002BF2D098F8002093424F
:10051000F1D823789342EED33046BDE8F081FE1E39
:1005200018BF01263046BDE8F08100BF03780A7885
:1005300043F020016429C3F340101DD0732910D06B
:1005400022F02001413919290AD9A2F130010929E3
:1005500006D96FEA531303F001035F2A18BF184648
:100560007047202AFCD06FEA5313093A03F00103C5
:10057000042A88BF184670476FEA5313303A03F0D5
:100580000103092A88BF1846704700BF2DE9F04FC4
:1005900095B0814600F15804D0E9140300AF5B68C0
:1005A00021469847D9F8583033B109F10803184665
:1005B0003B6226F0BDFC18B95437BD46BDE8F08F4C
:1005C00099F84810002940F0A381D9F808000028C4
:1005D00000F01C8126F00AFE8346002800F01681F8
:1005E000B9F838305A2B6D4600F08F81B3F5877F0C
:1005F00000F08B81B9F836200732D210D31D23F0DA
:100600000703ADEB030D0021684636F029FAD9F84F
:100610005430D9F850005B6821469847EA464FF0BD
:1006200001087D60C7F82C90386AC7F80CD007F134
:100630003802594626F086FB002800F0D680FB6A77
:1006400093F83A10072915D893F8443093B1B7F9C5
:100650003C200823B3FBF1F31A44013A92FBF3F276
:1006600012FB03F2BA87B7F9382092FBF3F202FBD0
:1006700003F33B8707F1380025F06CFBFB6A7863D6
:1006800007F1380093F83A402023B3FBF4F425F047
:1006900083FB054607F1380025F07EFBB0EBC41F55
:1006A0004FEAC41600F2B980C5F34A1301339B0028
:1006B0007B610733ADF5007D23F00703C7F828D031
:1006C00007F13800ADEB030DC7F810D025F042FB61
:1006D0004FF400720123C7E90623844600253D63D9
:1006E000C7F808B0C7F824C07A6A786B398F3E69BA
:1006F000A7F844100023521B92B2FB647B8F9042F8
:1007000003EB050188BF7A6AA7F8461098BF1B184B
:10071000B7F93C10A7F848108CBF9B185B197A6991
:10072000A7F84A300021304636F09AF9BC6ABA6917
:100730000021204636F094F923463246386A07F104
:10074000440126F043FBB7F94620B7F94A3094B28A
:100750009C423CDAF96AB7F9440091F83A30B1F8B2
:100760007660B1F87410D7F828B006FB021113FBBD
:1007700000F2002AB8BF073201EBE201B7F94820C6
:10078000121A03FB02F2FB6A002A9B6DB8BF073204
:1007900001340B444FEAE209A4B2601EC0F3CC025C
:1007A00000F007001AF8021008FA00F008430AF8EF
:1007B0000200594618464A4635F06EFFB7F94A100E
:1007C000A14200EB0603CB4404F10104E5DC05F093
:1007D000DBFC73F0F5FA7A6B3B6B1544FA69013375
:1007E0009A423B6380D1D7F808B0DBF808B0D7F85D
:1007F0000CD0BBF1000F7FF417AFD7F82C907D68B9
:10080000D9E9140351469B689847AD46386A26F0EB
:10081000EDFA5437BD46BDE8F08F07F1380025F0FA
:1008200075FBFA6AB6FBF0F692F83A30002E57D014
:10083000B1B2072B79630CD892F844204AB9796B8E
:100840000822B2FBF3F2B1FBF2F302FB03F39BB21B
:100850007B6307F1380025F07DFA7D6BB0FBF5F383
:1008600007F138009EB225F075FA721CB0FBF5F363
:1008700003FB150392B29BB2002B14BF1146314605
:10088000F96107F1380025F041FB7B6B10FB03F3A6
:100890009BB2B3FBF4F204FB12340CB1013292B2FE
:1008A00092005B09BA6101339A00BB697A61073330
:1008B00023F00703ADEB030DD31DDB086A46A2EB63
:1008C000C303C7F828D007F138009D46C7F810D0F9
:1008D00025F040FAFB698446002B7FF4FFAE84E7E5
:1008E000072B06D8FA6A92F8442012B901227A63DB
:1008F000A5E707F1380025F02DFAF86107F1380077
:1009000025F028FA01237B63BBE7B9F8342073E6AE
:100910000023C9F8303009F1280B61E62DE9F04FCA
:1009200000F1080B93B0814602AF584626F000FB59
:1009300018B94437BD46BDE8F08F99F84810002932
:1009400040F04C81D9F80800002800F0D68026F04D
:100950004DFC8446002800F0D08009F1B2037B6092
:10096000C7F81CB0C7F808C0B968F86907F12802D1
:100970006D4626F0E7F9002800F0B68007F1280060
:1009800025F0E8F9044607F1280099F83A8025F0A7
:1009900003FA99F8822083B2002A00F0B780C4F3EA
:1009A000CF027A614FF40072BA6108245B09013307
:1009B0009A00BB693A61073323F00703ADEB030DDF
:1009C000D31D23F0070302AEADEB030D02AB07F11D
:1009D0002800FB6025F0BEF97B698646002B00F0FD
:1009E00003814FF0000A3D60D04609F1500B3546B7
:1009F000C7F820E049E025F0CFF999F83A60F60809
:100A000016FB00F6B3B27B62D7E9036200213046E1
:100A100036F026F8BA690021284636F021F8324629
:100A2000FE692B4607F13401304626F0CFF95846CF
:100A300007F13402314626F015F8584625F068FFD4
:100A4000002861D099F8801041B90123D9F85000ED
:100A500000931A46D9F860607B68B0477B6AD9F882
:100A60005000009300222B460121D9F86060B04766
:100A7000584625F0E5FF05F087FB73F0A1F97B6987
:100A800008F101084345A2442AD0798D3B8DBB86ED
:100A90000AEB0102FA863A6AB7F92C603E87A2EBAC
:100AA0000A02002392B2A242FB6301EB0403534407
:100AB00099F83A203CBF3B6ACB18072A07F134006B
:100AC0007B8798D807F1340025F066F999F83A3019
:100AD0000822B2FBF3F3B0FBF3F6B3B27B6293E709
:100AE0003D68584625F0B0FFBB689B68BB60AD46CB
:100AF000002B7FF439AFD7F81CB0584626F076F9B2
:100B00004437BD46BDE8F08F3D68EDE707F12800AA
:100B10007B6225F041F92026B6FBF8F6B0EBC61F44
:100B20007B6A4FEAC61818D85B0901339B003B610A
:100B30000733ADF5007D23F0070302AEADEB030DE7
:100B400002AB07F12800FB6025F004F901234FF404
:100B50000072C7E90532864643E707F1280025F011
:100B6000D5F999F83A20B8FBF0F000283FD0072AD1
:100B700084B20AD899F844303BB90823B3FBF2F2A7
:100B8000B4FBF2F302FB03F39CB207F1280025F05B
:100B9000E1F8B0FBF4F307F1280099B2796125F090
:100BA000D9F87969B0FBF4F34A1C03FB140392B241
:100BB0009BB2002B18BF1146796107F1280025F080
:100BC000A5F910FB04F39BB2B3FBF6F206FB123659
:100BD0000EB1013292B29200BA61E7E60023C9F881
:100BE000303009F1280CB8E609F1500B79E7072AF3
:100BF00002D899F8443053B107F1280025F0AAF83B
:100C0000786107F1280025F0A5F80124D5E7012433
:100C1000B3E700BF2DE9F043884690F82A1011F0A1
:100C2000100785B06BD14368DB68044653F8281081
:100C300040F21C5045F0D0FD064600285DD06368A8
:100C4000DB6853F8280073689847B36801A95B68AC
:100C500081469847B36839469B6805464846984799
:100C6000B36839469B694846984763682549DB68FD
:100C700053F828003EF0BCFD064668B190F85030AD
:100C800023F0100301A980F8503027F0A3F90021C8
:100C90000546304627F060FD63681B49DB6853F862
:100CA00028003EF0A5FD064668B190F82A3023F0F2
:100CB000020301A980F82A3026F042FA00210546F5
:100CC000304626F04FFD7DB194F82A30DB070ED573
:100CD00004F1180201A9104625F0CAF894F82A3048
:100CE00043F0010384F82A3005B0BDE8F08304F135
:100CF000180101A824F0F0FFF0E70546B5E70CF075
:100D00005DFD00BF18E70B00E4E40B0070B586B092
:100D100005460191164619F0DFF890B9019840F0A8
:100D2000ADF80622044603A930463CF085F903AA33
:100D30002146284619F0E6F8002804DB0E2006B00C
:100D400070BD5EF043FF404271F0E8FE70B586B0C2
:100D500005460191164619F0BFF890B9019840F088
:100D60008DF80522044603A930463CF065F903AA34
:100D70002146284619F022F9002804DB0E2006B08F
:100D800070BD5EF023FF404271F0C8FE242B2DE9B8
:100D9000F047884601D8012B06D1FCF7B3FB162398
:100DA00003600020BDE8F087344E0D46294615F853
:100DB000014B375D17F00807F8D12D2C10D12C7896
:100DC00001278D1C33F0100115D1302C0DD129785D
:100DD00001F0DF01582908D16C78023510230AE0B0
:100DE0002B2C04BF2C788D1CECE7002BF6D1302C7B
:100DF00014BF0A23082307F1004E0EF1FF3E002125
:100E0000BEFBF3F90E4603FB19EAA4F1300CBCF16A
:100E1000090F10D86446A3421EDDB1F1FF3F07D091
:100E2000B14516D301D1A24513DB06FB03460121D0
:100E300015F8014BE9E7A4F1410CBCF1190F01D8F9
:100E4000373CE8E7A4F1610CBCF1190F04D8573C1A
:100E5000E1E74FF0FF31EBE74B1C05D122230360A4
:100E6000764632B930469DE707B17642002AF9D07E
:100E700009B105F1FF38C2F80080F3E7CD700C002E
:100E80002DE9F043344E86460D46284615F8014BB1
:100E9000375D17F00807F8D12D2C10D12C780127D9
:100EA000851C33F0100015D1302C0DD1287800F0BE
:100EB000DF00582808D16C78023510230AE02B2C6B
:100EC00004BF2C78851CECE7002BF6D1302C14BF26
:100ED0000A2308234FF0FF380026B8FBF3F803FB82
:100EE00008F96FEA09093046A4F1300CBCF1090F8A
:100EF00010D86446A3421EDDB6F1FF3F07D08045FF
:100F000016D301D1A14513DB00FB0340012615F8E0
:100F1000014BE9E7A4F1410CBCF1190F01D8373CB2
:100F2000E8E7A4F1610CBCF1190F04D8573CE1E7E4
:100F30004FF0FF36EBE7731C06D12223CEF80030CA
:100F4000304632B9BDE8F08307B14042002AF9D0FB
:100F500006B1691E1160F5E7CD700C00F0B583B0E5
:100F600004460D4601926AF08BF96368019A0746C0
:100F70000120587260680E46294656F0DFFE134B7A
:100F8000984204D0636800225A7203B0F0BD17F58E
:100F90007A7546F1000605E06AF072F9854276EB53
:100FA00001010CD363685A7A002AF5D19B7A042B8D
:100FB00096BF074A074852F8230003B0F0BD6368A4
:100FC000054800225A7203B0F0BD00BF0000AD0B0F
:100FD000C8B10B000100AD0B0700AD0BF8B54368BD
:100FE0009A6852B3054600240BE073689847B368CB
:100FF00005F108019B6898476B689A680134944230
:101000001BD2DB6840F21C5053F8241045F0E4FB7F
:101010006B68DB680646A70053F82400002EE4D175
:101020000D493EF0E5FB48B105F1080127F094FBBE
:101030006B689A6801349442E3D3F8BD6B68074942
:10104000DB68D8593EF0D4FB0028D5D005F1080163
:1010500026F088FBD0E700BF18E70B00E4E40B00A4
:1010600090F950302149B0F90C2000B5002B836A6B
:10107000B4BFB0F812C0B0F810C0002B08BF0B46C8
:101080009444997B92B2C1B193F9051011FB02F21D
:1010900059880A4412B2A0F8462093F90510B3F813
:1010A00002E011FB0CE31BB29A42D2BFA0F84A3017
:1010B000A0F84A20A0F8463000BD93F9041011FBB7
:1010C00002F219880A4412B2A0F8442093F90410DD
:1010D000B3F800E011FB0CE31BB29A42D2BFA0F8B8
:1010E0004830A0F84820A0F8443000BD1C0301207F
:1010F00090F950302149B0F90E2000B5002B836AD9
:10110000B4BFB0F810C0B0F812C0002B08BF0B4637
:101110009444997B92B2C1B193F9041011FB02F28D
:1011200019880A4412B2A0F8442093F90410B3F8C5
:1011300000E011FB0CE31BB29A42D2BFA0F848308A
:10114000A0F84820A0F8443000BD93F9051011FB29
:1011500002F259880A4412B2A0F8462093F9051009
:10116000B3F802E011FB0CE31BB29A42D2BFA0F825
:101170004A30A0F84A20A0F8463000BD1C030120E8
:1011800010EE102A22F00043B3F17E5F05D34BD15D
:10119000002A71DB9FED5C0A7047B3F17C5F05D2DA
:1011A000B3F14A5F47D89FED590A704700B5002A4E
:1011B00083B0F7EE007A62DB77EEC07AB6EE007AA3
:1011C00067EE877AF5EE407AF1EE10FA00F185804D
:1011D000B1EEE76ADFED4E6A9FED4E5A9FED4E7A13
:1011E0009FED4E4AA7EEA65A16EE103A6FF30B0388
:1011F000A7EE857A06EE903AF0EE674AF7EE005ACF
:10120000E7EE845AE6EEE64A36EE865A67EE277A2D
:1012100084EE850A87EEA57AA7EE060A30EE260A46
:1012200030EE000A03B000BD70EE407A9FED367AD2
:1012300087EE270A704760EE006A9FED356ADFEDA2
:10124000357A9FED357AE6EE867A9FED346AA6EE22
:10125000A77AF7EE005AE6EE865A27EE267ADFEDF9
:101260002B7AC7EE256A9FED2E7AA0EE667A30EED5
:10127000470A37EEC00A70479FED2A0A704730EEE2
:10128000270AF6EE007A60EE277AF5EE407AF1EE64
:1012900010FA2DD4F1EEE75A9FED1D6A9FED1D7AED
:1012A000DFED1D6A9FED1D5A9FED180AA7EE867AA5
:1012B000B7EE006AE7EE876AA7EE856A66EEA77A60
:1012C000C7EE866ADFED187AE6EEA57A77EEA57AA4
:1012D00030EE670A30EE000AA4E7B0EE670ACDED03
:1012E000017A65F0D7FFDDED017AB0EE406A71E773
:1012F000B0EE670ACDED017A65F0CCFFDDED017A45
:10130000F0EE405AC8E700BF00000000DA0FC93F06
:101310006BD30DBCBA132FBD75AA2A3EAEE534BF00
:101320006821A233DA0F49406821A2B300B510EE5C
:10133000103A5A0083B0F0EE407A26D523F00043ED
:10134000B3F18B4F07D333F03FFADFED267A30EE5F
:10135000270A03B000BDBFEE000AA7EEA70A77EE8A
:10136000A76AB5EE400AF1EE10FA24D4B1EEC07AC5
:1013700077EE877AB7EE007A87EE270A36EEC00A54
:1013800003B05DF804EB33F01FBAB7EE007A70EEED
:10139000477A37EEA77AA7EEA77AB5EE407AF1EE54
:1013A00010FA15D4B1EEC70A37EE800A03B05DF823
:1013B00004EB33F053B9CDED017ACDED006A65F061
:1013C00069FFDDED017ADDED006AB0EE407ACFE72E
:1013D000B0EE470ACDED007A65F05CFFDDED007AF6
:1013E000E2E700BF1872313F30B5084687B01146BA
:1013F0001A460F4B0DF10C0CCDE9003C032336F0DF
:1014000073FA0C49039C0C2041F0A6F89DF81020BB
:10141000214605460CF006FE9DF8143013B9284607
:1014200007B030BD28460CF021FE284607B030BD7D
:1014300010C00B0088C00B0000B583B001900CF009
:10144000F5FD019803B000BD08B508680CF03AFE40
:101450000E2008BD10B58EB003AB51F8044B0193BC
:10146000184B00930138032336F096F9606840F278
:101470003D5106AA3DF0F6F8227A049B039C09949C
:10148000520042F001020892059A6FF000415B00A1
:1014900040F6261043F001038A420A900B930ED0C7
:1014A000520040F2E64342F00102CDE90C32022143
:1014B00006AA022038F002F90E200EB010BD01215C
:1014C000F6E700BF28C00B0010B58EB003AB51F893
:1014D000044B0193184B00930138032336F05CF959
:1014E00060684FF4D46106AA3DF0BCF8227A049BF0
:1014F000039C0994520042F001020892059A6FF091
:1015000000415B0040F6261043F001038A420A9036
:101510000B930ED0520040F2E64342F00102CDE9B7
:101520000C32022106AA022038F0C8F80E200EB0B4
:1015300010BD0121F6E700BF70C00B0030B597B0B9
:1015400002AB51F8044B01932F4B00930138062353
:1015500036F022F9606840F2A16108AA3DF082F8F5
:10156000049B227A029C0B945B0043F0010352001F
:101570000E93059B42F001026FF0004144F61660A5
:101580000A928B42039A0D900C9234D05B0044F681
:10159000E65143F001030922CDE90F134FF00B0E82
:1015A0004FF00A0C14460321069B0DEB82000DEB55
:1015B0008C0C5B0043F00103079A44F2B6250562E8
:1015C000CCF820306FF000439A420DD00DEB8E0E18
:1015D0000DEB8404520042F00102013144F28623F3
:1015E000CEF82030C9B2E26208AA032038F066F8CB
:1015F0000E2017B030BD07224FF0090E4FF0080C37
:1016000014460221D0E700BF40C00B0010B50846C9
:101610008EB011461A46174B0DF11C0CCDE9003C5B
:10162000072336F061F9DDE90740134940F219322A
:1016300036F0B2FA08980E2803D00022012113F0E8
:101640009FFA0E49182040F087FF9DF834209DF83E
:1016500030300590CDE902329DF82C200A9B2146BE
:10166000CDE900329DF82430089A0CF03BFD059836
:101670000EB010BD14C10B0098E00B004CC10B0064
:101680000CF042BD08B508680CF08EFD0E2008BDB8
:10169000F0B5054685B001F134000E4604F0D8FCE3
:1016A0002B88102B2FD0112B2AD10022A888424C36
:1016B000134634F81210814202F1440203D0013380
:1016C000052BF6D1042303EB031304EBC3013B48C2
:1016D0000193009107F0E6FD019B00994FF6FF7220
:1016E00024F83320CB6D00220E2B81F85A2002D033
:1016F0005A602A7A1A720023B361012005B0F0BD46
:10170000002005B0F0BD00222B4C13464FF6FF70B1
:1017100034F81210814202F1440203D00133052B48
:10172000F6D1042303EB0312D700A888E05304EB9F
:10173000C202002082F85A00A2F876000E20D0657E
:10174000E87B009219010B44022804EBC30314BF89
:1017500096F845000120D87007F108004FF000020C
:101760004FF6FF71204483F87820A3F8581083F8CF
:10177000792009F095FC07F16000009A0F49204498
:1017800007F066FD0023B3612869696907F16C03FE
:10179000234403C302A860F037FEBDF808302A8A4C
:1017A0009A4202D86A8A9A4203D2A88802A960F0B3
:1017B00013FE0023F360A0E7A80A0120C91C05005E
:1017C00038B50388102B0C4618D0262B2ED11A4B77
:1017D0001878FF2810D060F0F9FD2146054617481B
:1017E00007F060FD0023E36084F8443035F008031F
:1017F000284601D00BF038FF012038BD8188002237
:10180000032060F00FFE0C4B1878FF280ED060F01C
:10181000DDFD21460546094807F044FD0023E3604D
:1018200084F8443035F00803284601D1002038BD43
:101830000BF01AFFFAE700BFA7060120C11703004B
:1018400030B587B0044615460846052269463BF088
:10185000F3FB03A9062228463BF0EEFB0199049A0C
:10186000204674F065FADDE90012039834F014FFA5
:101870002046DDE903120DF015F80E2007B030BD4B
:1018800030B587B0044615460846052269463BF048
:10189000D3FB03A9062228463BF0CEFB0199049A0C
:1018A000204674F045FADDE90012039834F0F4FEA6
:1018B0002046DDE903120DF007F80E2007B030BD19
:1018C00090F80C01400040F0010070472DE9F04114
:1018D00008468CB011461A46254B07ACCDE90034BA
:1018E000052336F001F80522079804A93BF0A4FB74
:1018F000059EA6F11002102A37D81E4BD340DB07F5
:1019000033D5089D022D20DD062D20D10998049F96
:1019100020B104A901223BF08FFBE8B980460A9868
:10192000C0B13FF0FFFA044613494FF48A7040F00B
:1019300013FECDE9005443463246394603900CF07D
:101940008FFF03980CB0BDE8F081002DDEDC0B4862
:1019500071F0D0F80446E7E7059840F26F121021C5
:1019600036F02EF8DDF81080D9E7054871F02EF931
:1019700000C30B000101010038C30B00E8890B0014
:10198000408D0B0070B551F8043B88B01D4603AB89
:101990000193184B00930138022335F0FDFE052218
:1019A000039805A93BF048FB069CA4F11002102AFD
:1019B0001CD8114BD340DB0718D5DDE9040620B154
:1019C00005A901223BF038FB40B9034628462246D0
:1019D00031460CF08BFF0E2008B070BD069840F227
:1019E0006F12102135F0ECFF059BEFE7034871F013
:1019F000EDF800BF28C30B0001010100408D0B0072
:101A000010B5044608463FF039FA022807DD0628DB
:101A100007D1014620460CF085FF0E2010BD00289E
:101A2000F7DC014871F066F8E8890B0030B5114B1E
:101A300087B005ADCDE900350446012300200D46F1
:101A400035F0AAFE2946204674F0C2FA059840F007
:101A5000FFFB421004D0084840F2115171F052F8D7
:101A60002946204604AB03920DF012F8039903486F
:101A70007CF0A1FBE8C30B006C950B0044530B00FA
:101A800010B90E231846704730B50D4683B0044692
:101A900074F09EFA294620460CF066FF0022019061
:101AA00046F6760104483CF06FFF019B00B14360AD
:101AB000184603B030BD00BF6C000120E0B130B566
:101AC0000F4BDFF840C01C780439002201E090423F
:101AD0000FD051F8043F9D0702F10102F7D11D68B4
:101AE0006545F4D15D6895F804E0A645EFD1184648
:101AF00030BD0E23184630BD0E231846704700BF78
:101B0000747C0120A8C40B0010B5084688B01146AB
:101B10001A46104B0DF1100CCDE9003C042335F0B2
:101B2000E3FE049840F2FD4174F00EFA0A490446BF
:101B30000C2040F011FD9DF81C2000929DF81830FB
:101B40009DF81420039021460CF05CFF039808B028
:101B500010BD00BF88C40B00A8C40B0008B50CF072
:101B600065FF002808BF0E2008BD00BF08B50CF0B7
:101B70005FFF00280CBF1E203E2008BD08B5054BA6
:101B80001A7802B108BD1FF0C7FF024B01221A707C
:101B900008BD00BF3B7C01200E4A0F49506810B5BC
:101BA0000E4C0023C008C4E9001310D00C49D268C1
:101BB00091F800E002F1040C01E0834207D05CF8E8
:101BC00033201179714503F10103F6D162600348B6
:101BD00010BD00BFE8B20B00A8C40B00A84601204E
:101BE000747C01202DE9F041184F194E0024012585
:101BF000D6E90001D7E90032A4F1200CC4F1200895
:101C000005FA0CFC25FA08F803430A434CEA080CD1
:101C100005FA04F10B4002EA0C021343E0B207D0CC
:101C20005FF002FB204654F013FD204654F048FEBE
:101C30000134402CDCD1074900220023C7E90023EE
:101C4000C6E90023C1E90023BDE8F0815811012055
:101C500068110120F0110120002975D02DE9F04F05
:101C60003A4B1C685E683A4B87B0D3E90098394B11
:101C7000009400251C680194043ACDE90255CDE991
:101C800004505F68344C02EB81014FF0FF3C4FF091
:101C9000010E01E091422CD052F8043F9807F9D18F
:101CA0001868A042F6D1586893F808B090F804C0BC
:101CB000ACF12000CCF1200A2EFA0AFA0EFA00F05C
:101CC00040EA0A000EFA0CFABBF1000F2FD049EAE5
:101CD0000A0948EA0008CDF808B05B7A002BD9D091
:101CE000019D049345EA0A059142019547EA0007E0
:101CF000D2D1DDE904501DB1164B019AC3E900278A
:101D0000039B1BB1114B009AC3E90026029B13B140
:101D10000F4BC3E90098BCF1FF3F05D078B10F49E4
:101D20000F4A00230B60137007B0BDE8F08F009DD1
:101D300045EA0A050095012506430395CDE707B05E
:101D4000BDE8F04F1FF0E8BE704700BF68110120EA
:101D500058110120F0110120A8C40B00A475012026
:101D60003B7C0120054B1B78012B01D000207047E4
:101D7000034B1878FF3818BF01207047757C01208D
:101D8000747C012008B500F009F8FFF72BFF00F084
:101D9000D3F9BDE8084000F00BBA00BF10B5124CF3
:101DA000124A23686FF3172393421CD04FF48072BA
:101DB00000210F4834F054FE0E490F4B00220A70E8
:101DC0001A704FF080404FF44031130103F180430B
:101DD0000132082AC3F80419F7D1044B4FF47C12DE
:101DE000C0F88429236010BD707C0120AF0000ADD5
:101DF000787C0120757C0120747C0120002A75D03C
:101E000070B514468A0788B005460B4603D1464A8A
:101E10000968914230D028462E6801930CF066FE86
:101E2000019A0146002330463BF040F9042C064657
:101E300015D020463FF022F84223FF22002104461D
:101E400035F0AEFD012305AA314628468DF8144031
:101E50000CF050FE002846D00E2008B070BD0146A0
:101E60000123284605AA0CF031FE9DF8140040001D
:101E700040F0010008B070BD01930CF037FE0199ED
:101E800002AA45F043FC002844D0DDE90232042CCC
:101E9000A2EB03062FD0A3072AD12368234A93423B
:101EA00008D0234A934205D0224A934202D0224AC4
:101EB00093421DD1052205A920463BF0BDF8069BA3
:101EC000B3422DD19DF81C10059C0022402035F016
:101ED00099FE012821D102993346224628460CF06A
:101EE00009FE0028B8D1154870F03CFE1046704736
:101EF000134870F0FFFD304632F05AFD0299044657
:101F00000246334628460CF0E1FD2146304640F0BB
:101F10005DFBA2E70B4870F0EDFD0B4870F056FE3C
:101F20000A4870F053FE00BF34630B00E44E0B0010
:101F3000604F0B00184F0B0000660B0040870B0032
:101F4000AC840B00E0790B005C920B0090890B00D5
:101F500010B5044608460CF0C9FD042C09D0052C28
:101F600001D0002010BD064B03EA400040F0010004
:101F700010BD80B200280CBF1E203E2010BD00BF47
:101F8000FEFF0100F0B1DFF84CC00439002351F826
:101F9000042F12F0030F03F1010311D110B41468E0
:101FA00064450AD0984210D051F8042F940703F1E9
:101FB0000103F7D114686445F4D1104610BC704792
:101FC0009842E4D10E22104670470E22104610BCF3
:101FD000704700BF04C50B0038B5084BD3E9004576
:101FE00054EA050305D019F069FD201A65EB0101DB
:101FF00038BD4FF0FF30014638BD00BF1812012038
:1020000010B52DED028B08468AB011461A46324BA8
:1020100005ACCDE90034022335F066FCDDE90504AA
:10202000B0F10E0218BF0122B4F10E0318BF012354
:102030009A424BD00E2846D03EF0A6FEB0EE408A23
:1020400019F03CFD70F054FB9FED247A0E2CC0EE8D
:10205000077A25D040F2AF310698CDED037A35F0FE
:1020600085FD04465FF062FC07A967F097FB9DF8C9
:1020700022009DF821109DF820309DF81F20CDE909
:1020800000109DF81E10BDF81C006CF0B1F8231A6A
:1020900008EE103ADDED037AB8EEC88A38EE278AEA
:1020A000B4EEE78AF1EE10FA13D40D49082040F09F
:1020B00053FAB0EE480A04460CF02EFD20460AB052
:1020C000BDEC028B10BD9FED078AB9E7064870F0A2
:1020D0007DFD064870F07AFDF4C40B0000007A44E0
:1020E00004C50B000000000028890B004C880B0081
:1020F00008B50CF015FDB4EE400AF1EE10FA08D662
:1021000010EE103A23F0030040F00200A0F1FF406F
:1021100008BD014808BD00BF02004000704700BF75
:102120000349044A0A6000234B600846704700BF19
:10213000A846012004C50B0008B501205BF074FA25
:10214000024B00200021C3E9000108BD1812012044
:10215000034B1878A0F10200B0FA80F040097047F4
:10216000757C012010B5084686B011461A460C4B06
:102170000DF1140CCDE9003C012335F0B5FB0598B9
:1021800040F2FD4173F0E0FE06490446082040F0AD
:10219000E3F9214603900CF0C7FC039806B010BD8C
:1021A00040C50B0048C50B00406870470E207047C3
:1021B000704700BF704700BF0020704738B5094C1A
:1021C000094D23680BB1AB4208D14FF4BA7200211C
:1021D000044834F045FC2560024838BD034870F0DF
:1021E000C1FC00BFC04C0120A8600B0018880B0088
:1021F00010B5094B094C1B68A34203D013B1084822
:1022000070F0B0FCB4220021064834F029FC054BE4
:1022100043F8044C181F10BDD00D0120A8600B001E
:1022200010880B00D40D0120164B0122002186B02E
:10223000C3F80025C3F81011D3F8101101910199CA
:10224000DA60D3F81021002AFBD00022C3F8102155
:10225000D3F8101105910599C3F80421D3F804119E
:1022600004910499C3F80821D3F808110391039944
:10227000C3F80C21D3F80C1102910299C3F8002580
:1022800006B070470070004008B50CF089FC0E20C5
:1022900008BD00BF10B582B0084611464FF00212CB
:1022A000019335F03FFA019B18680CF02DFD0649AB
:1022B0000446082040F058F9214601900CF050FCEB
:1022C000019802B010BD00BF84C50B0010B50446D4
:1022D0000CF086FCC8B920460CF088FCB5EEC00AAC
:1022E000F1EE10FA0DD9B4EE400AF1EE10FA0AD66A
:1022F00010EE103A23F0030040F00200A0F1FF407E
:1023000010BD0E2010BD024810BD5DF05FFC00BF87
:102310000200400010B504460CF062FC30B92046C3
:102320000CF06AFC400040F0010010BD5DF04EFC76
:1023300008B50CF0F5FC0E2008BD00BF10B582B04A
:10234000084611464FF00212019335F0EBF9019B5C
:1023500040F2FD41186873F0F7FD06490446042079
:1023600040F002F9214601900CF0D2FC019802B035
:1023700010BD00BFF8C50B0030B583B004460D4654
:102380000CF0D0FC80B9019028463EF077FD019911
:10239000A2234FF6FF7235F003FB81B220460CF00A
:1023A000C3FC0E2003B030BD5DF010FC2DE9F04FF2
:1023B0002DED088B804B8FB009ACCDE9003405239F
:1023C00035F0EAF90021099850F062FC0021074637
:1023D0000A9850F05DFC054600210B9850F058FC1F
:1023E000EB790290012B40F0E380C379012B40F0A0
:1023F000DF80AA68012A40F2DB808368012B40F26B
:10240000D7809A4240F0D4806621B86852F084FFA9
:10241000EC6929798146204650F080FDAB68A869B7
:102420002979013B00FB0340F0EE408A50F076FD35
:102430000C98029B0E28DC69B0EE40AA00F0A28046
:102440003EF0A2FC0D980E28B0EE409A00F0A48059
:102450003EF09AFCF0EE409ABB68C3B3EB6904937C
:10246000029BD7F81CA0DB69D9F81C6003934FF0DE
:102470000008BB46CDF81C900EE0B4EEC0AAF1EE09
:1024800010FA2AD5F0EE697AE6EC017ADBF808203A
:1024900008F10108424518D950469BF8041050F045
:1024A0003DFDDBF81820F4EEC08AF1EE10FAB0EE34
:1024B000408A9244E1DDF0EE497AE6EC017ADBF8FD
:1024C000082008F101084245E6D8DDF81C9048468E
:1024D0000FB0BDEC088BBDE8F08FAC68013C012C5F
:1024E00027464FF000091ED9CDE905862E46049DEA
:1024F00004E0A7EB0804012CC14610D9B06931797A
:10250000640804EB090800FB085050F007FDB4EE26
:10251000C80AF1EE10FAECDB012C4746EED835463E
:10252000DDF81480069E049CA869297900FB094007
:1025300050F0F4FCA869297900FB0740F0EE40BA9E
:1025400050F0ECFC029C039BA069217900FB093050
:10255000F0EE40AA50F0E2FCA069039A217900FB5A
:102560000720B0EE40BA50F0D9FC38EE6B8A30EE5E
:102570004B0A7AEEEBAA28EE008AC8EE2A7A77EEAA
:102580008B7A81E72046197950F0C8FC0D980E2807
:10259000B0EE409A7FF45CAF029A9068936911792B
:1025A000013803FB004050F0B9FCF0EE409A53E7CD
:1025B000024870F00BFB00BFA42A0C00647D0B00E6
:1025C0002DE9F0472DED068B5D4B88B005ACCDE9CC
:1025D0000034032335F0E0F80598002150F058FB53
:1025E0008368012B75D9C579012D044640F0A5807B
:1025F000007950F031FC07460698E6690E286ED047
:10260000002150F045FBC579012D814640F09280B4
:10261000A26883689A4240F08D80007950F01CFCDB
:1026200080463046D9F81CA0B847A36903935046AA
:10263000B0EE408AC047A368012BF0EE408A74D9FF
:10264000039B9FED40AA1E44D9F818309A443046A7
:10265000B847A3695046B0EE489A1E44B0EE408A8F
:10266000C047F0EE689A38EE099A70EE699AF0EE7B
:102670004A6A07EE905AD9EE896AA368D9F81820F9
:10268000B8EE677A0135C6EE877AAB429244F0EE37
:10269000408A3AEE27AADAD8F6EE007A2AEE27AA7E
:1026A000013B07EE903AF8EE677A67EE8A7AF4EE2D
:1026B000677AF1EE10FA3BD617EE903A23F003005A
:1026C00040F00200A0F1FF4008B0BDEC068BBDE871
:1026D000F0871D4808B0BDEC068BBDE8F087079871
:1026E000DFED188A3EF050FB3046B0EE40AAB84706
:1026F000A368012B16D92A462179E069B0EE408AF9
:1027000050F0C8FB07EE905A30EE088AB8EE677AB0
:1027100038EE688AA368C8EE077A0135AB4278EED6
:10272000A78AE8D82AEE28AAB6E79FED06AAB7E757
:102730000648C9E7064870F049FA064870F046FABC
:102740008C2A0C0000000000020080800200400083
:10275000A4760B0098760B001E280ED03E280CD0D5
:1027600010F001030AD110F0030209D10168094AEF
:10277000914208BF0123184670470123184670474D
:10278000022AFBD16FF3D600831F18BF012318461E
:10279000704700BFAC5A0B0010B54268FF2A82B0E8
:1027A00004460B460ED9D4E90221207935F0DEFF2C
:1027B000D4E901320E200132A3F58073C4E901325D
:1027C00002B010BD019100220179402035F01AFAC3
:1027D0000246D4E90210083102FB01F1009232F006
:1027E0002DF9009AA168D4F804C0E06001FB022131
:1027F0000844082161F31F2CC2EBC202C4F804C0D4
:10280000002134F02DF9019BCDE700BF2DE9F04305
:1028100013468BB005460C46242820D8DFE800F08C
:1028200024242424241F1F1F1F1F1F1F1F1FA61F18
:10283000131F1F1F1F1F1F1F1F1F1F671F131F1F78
:102840001F1F1F1FB30013F0010240F0B18013F0EF
:10285000030104D1B24A1868904200F0A980002414
:1028600020460BB0BDE8F08309790393002201F004
:102870007F01402035F0C6F9E368AA4A21681E4668
:10288000A36899462379914298460746039B00F036
:10289000F3801846012207A93AF0CEFB002800F089
:1028A000828008F07F03012B099A00F0EB805A2BFD
:1028B00094BF20330020012A00F0C1805A2A00F37F
:1028C00017812032934240F0B08023F00203642B42
:1028D00000F0AB80089B009309FB07F2079B314691
:1028E000284644F03DFE00285DD03E24B8E78D4DDB
:1028F0000A68AA42B3D009790393002201F07F014C
:10290000402035F07FF9A268E36802FB00F82279E5
:1029100002F07F062268AA421F46039B00F0BB809C
:10292000184607A905223AF087FB002231464020CD
:1029300035F068F9A168089B05463046B3FBF5F30E
:102940001944039300F02AFA044639464246C06807
:1029500033F0A2FEE068039B079903FB05F24044B5
:1029600033F09AFE20460BB0BDE8F0836D4A09684B
:1029700091423FF474AF1946204600F047F92046D3
:102980000BB0BDE8F0831846012204A903933AF086
:1029900053FB039B00283FD014F0030203D1624B8A
:1029A000216899424FD01E2420460BB0BDE8F08329
:1029B00018463EF063FA2179002201F07F0181463A
:1029C000402035F01FF9E3682668A168227998460F
:1029D000544B9E4201FB00F700F08480102D60D024
:1029E00009FB01F102F07F0000F0D8F9C36804464A
:1029F000002F3FF435AFB9F1000F3FF431AF09F1CB
:102A0000FF35414618463A4633F046FE013D691C03
:102A100000EB0703F5D123E7DA0706D413F003022E
:102A200006D13F4A1B689342BDD1002070F062F886
:102A3000022AB8D16FF3D603062BF6D1B3E7622B87
:102A40003FF448AFF1E72179364D01F07F01402096
:102A500035F0D8F80246D4E9023003FB02F12368CE
:102A6000AB4256D00124DDE90423009429F028FB71
:102A700000287FF43AAF96E76268C2F3172200FBA2
:102A8000026606E7012A3FF425AF5A2A3DDC422AB6
:102A90003FF420AFC9E76268C2F3172200FB027758
:102AA0003EE711464020002235F0ACF8A36809FB50
:102AB00003F300FB03F1E06831F0C0FFA368E060BE
:102AC00009FB03F3A360636803F0FF036360B9F1DC
:102AD000000F3FF4C5AE09F1FF39C319002F3FF4D1
:102AE000BFAE88E76368C3F3172300FB038875E76D
:102AF00093429AD123F00203642B96D0022D3FF427
:102B0000E9AE00287FF4E6AE8FE7622A3FF4E2AE3A
:102B10008BE76368C3F3172302FB0300A2E700BF40
:102B2000AC5A0B00184F0B00604F0B00F0B501289A
:102B300085B007460E463FD08B0736D030463FF073
:102B400097FB002857D045102946384600F026F953
:102B50000021044630463AF005FB06463AF0CAFD2D
:102B600068B17DB100252A460346E168384635F054
:102B7000FDFD304601353AF0BDFD0028F3D1204679
:102B800005B0F0BD01462046FFF706FE30463AF09C
:102B9000B1FD0028F3D001462046FFF7FDFD304689
:102BA0003AF0A8FD0028EDD1E9E70B68144A9342FA
:102BB00002D0144A9342C1D1012201A930463AF011
:102BC0003BFA0028BAD039460022402035F01AF8E6
:102BD000029BB3FBF0F100FB01F5AB420DD138468F
:102BE00000F0DCF8019904462A46C06833F054FD31
:102BF000204605B0F0BD0546A6E703486FF0E6FFA6
:102C000000660B00604F0B00A4830B0070B50E46EE
:102C100086B00446012203A930463AF00DFA002896
:102C20003AD021790022402034F0ECFF6268049B06
:102C3000B3FBF0F3B3EB122F0546C2F31721E068A4
:102C400013D8C91A61F31F226260A2680399019325
:102C500002FB050003FB05F233F01EFDA268019B99
:102C60000E201A44A26006B070BDA16801931944F9
:102C700005FB01F131F0E2FE6268E06002F0FF0264
:102C80006260B442019BE0D1052203A920463AF0DC
:102C9000D3F9E068019BD8E7014630463AF062FA82
:102CA000054601E0FFF778FD28463AF023FD01468E
:102CB00020460029F6D10E2006B070BD70B50D4635
:102CC0000179044601F07F0116464020002234F0CD
:102CD00099FFE2682A60A36800FB03F36B60237925
:102CE00003F07F03AB602168094B994201D00020BB
:102CF00070BD94F90430002B03DBB30701D501202C
:102D000070BD6368C3F3172300FB03222A60EEE75C
:102D1000184F0B004268C36891688B4284460BD2FF
:102D20001079D168DCF808201A44013300F07F00E4
:102D3000CCF80C3035F0BAB900207047084A0023AF
:102D4000C1E90233C1E90020064B02689A4201D072
:102D5000084670474368C3F317238B6008467047E3
:102D6000AC4E0B00184F0B0038B50C461D461146F3
:102D70002046094A34F0D6FC286841F0E3FC012CD7
:102D8000007804D06968BDE83840FFF7CFBEBDE8E1
:102D90003840002100F002B8040002007828F8B59D
:102DA0001CD005460E4600220146402034F02AFF82
:102DB000012D0CBF0B490C49074610203FF0CCFBFE
:102DC00005714368866003F0FF030446436006FB19
:102DD00007F031F027FEE0602046F8BD03486FF0B1
:102DE000F5FE00BF604F0B00E44E0B0014840B0097
:102DF00070B50D79012D0C4606462FD01F492A4685
:102E000043F0DCFCA3682BB930461D49BDE8704097
:102E100043F032BC1B49304643F02EFCA3689BB103
:102E2000002501E043F028FC2A46E168207935F0CE
:102E30003DF901220146304640F05AF9A368124993
:102E40000135AB423046EDD81049304643F014FC12
:102E500030460B49BDE8704043F00EBC0C4943F0CE
:102E60000BFCD4E9022130462B4645F023F93046CD
:102E70000349BDE8704043F0FFBB00BF00390B00C1
:102E8000283A0B000C390B0010390B0014390B00D9
:102E9000F4380B002DE9F04788B0002A35D011F046
:102EA000030304468C46806815461E4603D1904BAA
:102EB0000A689A422ED062460146002320683AF002
:102EC000F5F88C4B216894F804C09942024609D069
:102ED000042D0FD1E1680CF07F0008B0BDE8F04789
:102EE00035F0E4B86368042D00EB1322F2D01CF037
:102EF000800F0AD02B46E1680CF07F0035F036FCDD
:102F00000E25284608B0BDE8F0870025284608B001
:102F1000BDE8F08702AA44F0F9FB002800F0E28047
:102F20002179042D01F07F0132464FF0400078D026
:102F300034F068FE15F0030280464BD12968887B87
:102F400030B101EB800003696B48834200F0AD8033
:102F50006A4A91423ED1B8F1010F40F0C680052285
:102F600005A928463AF068F8DDE9059761484FF071
:102F7000000ADDE902212668E3688D1A8642A7EB84
:102F800005052AD0002D34DD6068B5EB102F65D81B
:102F9000D019A26801932A44121A08FB013108FBD8
:102FA00002F208FB003033F0ABFBDDE9013009EB46
:102FB0000A0108FB07F200FB083033F0A1FB63684D
:102FC000C5EB132262F31F23A26863602A44A26048
:102FD0000E2596E74A486FF08DFD94F904100029FC
:102FE00093DA002D40F081806168C1F3172108FB5E
:102FF000013308FB023009EB0A0108FB07F20193D9
:1030000033F07EFB0399A2680298019B521A384460
:1030100008FB02F208FB013108FB003033F070FBC3
:10302000CDE734F0EFFD334B2168029A9942064612
:1030300029D1B2F1807F51DA10203FF08DFA054698
:1030400094E80F0085E80F00029A02EB112363F366
:103050001F216960039B9B1AAB6052E7A268019332
:103060002A4408FB02F1184631F0E8FC6268E0608F
:1030700065F31F226260019B9945DDE90221034649
:1030800008BF814684E703992079891AFFF786FEF5
:10309000DDE902130546E0685B1A06FB03F206FB56
:1030A0000101E86833F0F8FA2BE72979402001F0B4
:1030B0007F0134F0A7FD404517D1AB680D482A6861
:1030C0001F46EB688242994602D04FF0000A50E753
:1030D0006A68C2F3172208FB02FA4AE709490A485C
:1030E0007BF069F809486FF005FD09486FF06EFD47
:1030F00034630B00184F0B00952E030000660B0085
:10310000AC840B00C87B0B005C560B00E0790B0015
:10311000787C0B00042808D0052801D000207047D7
:103120008868400040F0010070478B68002B0CBF9E
:103130001E203E20704700BF10EE102A22F00043F0
:10314000B3F17E5FF0EE407A07D30FD070EE407A95
:103150009FED3B7A87EE270A7047B3F17C5F27D259
:10316000A3F50003B3F1645F07D270479FED357A92
:103170009FED350AA7EE870A704760EE006A9FED63
:10318000336ADFED335A9FED337A9FED335AE6EE23
:10319000865AB7EE006AA6EEA57AA6EE856A27EEF5
:1031A000267AC7EE066AE0EE267AB0EE670A704726
:1031B000B7EE007AF0EEC07A77EE677A00B5B6EE39
:1031C000007A67EE877A83B0F5EE407AF1EE10FA76
:1031D00028D4F1EEE76A002ADFED1C5A9FED1C6A45
:1031E0009FED1C7A9FED1C5A9FED160AA7EEA56A6B
:1031F000F7EE005AA7EE867AE7EE855A67EE277A51
:10320000B0EE005A87EEA57ADFED147AE7EE266A73
:10321000E6EE857A30EE670A01DB03B000BDB1EE61
:10322000400AFAE78DED010AB0EE670ACDED007AAB
:1032300064F030F8019ADDED007AF0EE406ACAE7FA
:1032400000000000DA0FC93F000080036BD30DBC03
:10325000BA132FBD75AA2A3EAEE534BF6821A2B3CA
:1032600000B585B08DED010A019B23F00042B2F15B
:103270008B4F00EE102A4FEAD37127D25B000ED499
:10328000B2F1665F2BD2DFED1F7A70EE277ACDEDBB
:10329000037A039B09B1B1EE400A05B000BDB7EE59
:1032A000007AF0EE476AE0EE006A0191B0EE006A43
:1032B000F1EEE67A77EE807AC7EE276AE0EE066AEC
:1032C000B0EE660A31F080FA0199E3E7019131F03E
:1032D0007BFADFED0D7A019930EE270ADAE720EE6E
:1032E000007AF7EE006A37EE266A0191F1EEC67AAF
:1032F00077EEA67AC7EE276A36EE800A31F0AEF98D
:103300000199C7E70000807B1872313F08B55AF079
:10331000AFFA044B02689A4200D108BD0D205DF05F
:103320006FFF00BFEF29780100B585B04FF4007C36
:1033300001A903AB02AACDF80CC02BF023FB024875
:1033400003996FF04BFC00BF30950B00F4EE400A80
:10335000F1EE10FAF0EE407A53D610EE901AB1F179
:103360007E5F49D010EE102A8B0F03F0020343EA70
:10337000D27332F0004208D1022B3FD09FED397A50
:10338000032B08BFB0EE470A704731F000412ED042
:10339000B1F1FF4F21D001F15060904227D3B2F13B
:1033A000FF4F24D000B5980783B030D502F15062AA
:1033B0008A4251D387EEA00A0193B0EEC00A00F012
:1033C00063F8019B022B3ED19FED277ADFED277A30
:1033D00030EE070A37EEC00A25E0B2F1FF4F03F1E5
:1033E000FF3328D0022B20D99FED210A7047DB073D
:1033F0000AD49FED200A704700F046B89FED1B0AE3
:10340000704730EE800A70479FED1B0A704787EEC9
:10341000A00A0193B0EEC00A00F036F8019B012B20
:1034200001D1B1EE400A03B000BD144A02EB8303A0
:1034300093ED000A7047022B11D8114A02EB830367
:1034400093ED000A70479FED087ADFED087A30EEC1
:10345000070A30EE670AE6E79FED050AB2E79FED3F
:10346000090A7047DB0F49C02EBDBB33DB0F494053
:1034700000000000DB0FC93FDB0FC9BFC0230C00F9
:10348000CC230C00DB0F493F10EE102A22F0004342
:10349000B3F1994F4FEAD27109D3B4EE400AF1EE7D
:1034A00010FA0ED6002943D09FED4A0A70474A48C9
:1034B000834207D8B3F1665F3DD212F0FF4F00F0B0
:1034C00081807047454A9342B0EEC00A4ED9444AC3
:1034D00093426ED8F7EE087AF7EE006AE0EE276ABC
:1034E00070EE677A9FED3F7A9FED3F0A87EEA66AFE
:1034F00026EE065ADFED3D7ADFED3D4A9FED3D4A6F
:10350000DFED3D5A65EE056AE6EEA74ADFED3B7A50
:10351000E6EE847AE6EEA45A67EEA67AE5EE257A20
:1035200097EE867A77EE467A30EE670A89BB704767
:103530009FED330A704720EE006ADFED2C7ADFED55
:103540002C5A9FED2C5ADFED2C6A26EE067AE7EE18
:10355000275ADFED2A7AE7EE057AE7EE256A67EE6D
:10356000877AE6EE267AA7EEC00A7047A2F5D00267
:10357000934211D8F0EE007AFFEE006AE0EE276A7F
:1035800070EE277A9FED1F7A9FED1F0A86EEA76ADD
:10359000AEE7B1EE400A7047F7EE007A70EE676A68
:1035A00030EE270A9FED197A86EE806A9FED180AA1
:1035B0009EE7FFEE007A87EE806A9FED167A9FED18
:1035C000100A95E760EE007A82B0CDED017A019B9A
:1035D00002B07047DA0FC9BFFFFFDF3EFFFF973F22
:1035E000FFFF1B40B40F14335E987B3F25AC7C3D3E
:1035F0000DF5113E4712DABDA9AAAA3E98CA4CBEE3
:10360000DA0FC93F6937AC313863ED3E68212233A8
:10361000DA0F493F6821A23300B585B08DED010A6C
:10362000019B23F00042B2F17C5F00EE102A4FEACA
:10363000D37124D2B2F13E5F0CD213F0FF4F04D10C
:1036400060EE007ACDED037A039B09B1B1EE400A3A
:1036500005B000BD30EE007AF7EE007A77EEC07A62
:1036600067EE006A019186EEA70A30EE070A30F095
:10367000F5FFF6EE007A20EE270A0199E5E7F7EE6E
:10368000007A77EEC07A019180EE277A37EE070A4A
:1036900030F0E4FFF6EE007A20EE270A0199D4E735
:1036A000014B18682AF03ABBC046012010B5D1F88A
:1036B00000C001280C46134600F1FF3188BF221DCF
:1036C000604698BF002260F05BFD206810BD00BF1F
:1036D00010B5044C206831F069F9034A00231360E7
:1036E000236010BDC0460120C846012000B583B04C
:1036F000019001A860F0B0FD0E2003B000BD00BF36
:1037000008B50BF08FFB0E2008BD00BF70B5084652
:103710008EB011461A461F4B08ACCDE90034062383
:1037200034F0E2F89DF83440089840F2DF213CB3D1
:1037300072F042FC40F294610646099872F03CFC3B
:1037400002460A98079240F2553172F0FDFB40F2B2
:103750007A4106900B9872F00FFC0F49054628201D
:103760003EF002FF02949DF830400095DDE90632FC
:103770003146019405900BF0D9FA05980EB070BD52
:1037800072F0E2FB40F294610646099872F0DCFBAD
:103790000246D6E7D0C60B0010C70B0010B5044692
:1037A0000BF08EFB38B920460BF092FB00280CBFC3
:1037B0001E203E2010BD5CF009FA00BF10B5044683
:1037C0000BF07EFB38B920460BF088FB00280CBFBD
:1037D0001E203E2010BD5CF0F9F900BF10B5044674
:1037E0000BF06EFB40B920460BF078FB30B1204661
:1037F0000BF088FB0E2010BD5CF0E8F901486FF07B
:10380000B1F900BF7C8B0B0030B50C6887B0054662
:103810002046CDE902210BF053FBDDE9022188B9F6
:1038200004AB0193084B0093681E0223043133F06C
:10383000B3FF20469DF8142004990BF06BFB0E207B
:1038400007B030BD5CF0C2F900C70B0010B50446EC
:103850000BF036FB50B920460BF03AFB08B90E20AE
:1038600010BD20460BF05CFC0E2010BD5CF0AEF9E4
:1038700010B504460BF024FB20B920460BF058FC91
:103880000E2010BD5CF0A2F908B50BF0A9FC0E20CB
:1038900008BD00BF2DE9F0472DED028B08468CB026
:1038A00011461A46304B05ACCDE90034072334F0FD
:1038B0001BF84FF44871059872F046FB4FF45671AF
:1038C0008046069872F040FB40F2925281460121F8
:1038D000079834F059F8089D082D824601D0102D24
:1038E0003DD10A9CA4F10801F72933D8630731D1EF
:1038F0000B989DF82460EDB2E4B240B33DF044FA79
:10390000B0EE408A40F2F452B0EE480A01210020A5
:1039100034F000F8154908203EF026FE53464A468A
:103920004146CDE90164009507460BF011FCDFED3F
:10393000107A28EE278AFCEEC87A17EE900A39F042
:1039400063FC38460CB0BDEC028BBDE8F0879FED00
:10395000098AD7E7084840F2E6416FF03FF9064888
:103960004FF438716FF03AF9C8C70B0000C80B006C
:1039700000007A44AE47E13D9C940B0010B504462C
:103980000BF042FC30B920460BF048FC400040F000
:10399000010010BD5CF01AF9F0B585B006460D4681
:1039A00017460BF031FC00283BD1044640F263413E
:1039B000384634F0DBF8214640F26342074634F0E3
:1039C00017F828463EF066FB044678BB062201A99C
:1039D000284639F031FB22469DF80C10029C40200D
:1039E00034F010F9B4FBF0F4BC421CD330460BF0B9
:1039F00013FC039B482B0FD010281AD0422B01D068
:103A0000012B09D101993A4630460BF00BFC4000DE
:103A100040F0010005B0F0BD0828F3D106486FF072
:103A2000D5F85CF0D3F805486FF0D0F804486FF093
:103A300061F804486FF0CAF8FC800B00BC8F0B00E3
:103A4000EC900B00E4800B0090F82C20012A5CD154
:103A500090F82D30002B58D090F82E30002B54D0F9
:103A600090F82B30002B50D0036A002B4DD030B58E
:103A7000044683B000926DF049FD94F82B30009A13
:103A8000591E8A40D2B2216A002818BF134603FB90
:103A900001F1CDE900136DF039FD236A009900288A
:103AA00014BF4FF4FA524FF47A721D46B1FBF2F292
:103AB00000926DF02BFD94F82D10009A019B0028C8
:103AC00094F82E0002F1010201FB00F012FB00F25B
:103AD000218A92B214BF4FF4FA5E4FF47A7E91427B
:103AE00014D303FB05F1A2EB000CB1FBFEF30EFBBC
:103AF00013111FFA8CFC89B100216CF30F016CF3D8
:103B00001F416162228503B030BD70474FF0E02352
:103B1000D3F8F03DDB07F6D500BEF4E7ACEB0000D0
:103B2000A084A4F826C02285EDE700BF2DE9F04F60
:103B3000012989B00646154605D0022918D0012072
:103B400009B0BDE8F08F127812F060010F4637D14E
:103B50006B780A2B53D00B2B7FD0012BEFD04FF07B
:103B6000E023D3F8F03DDB0700D500BE0020E7E7F7
:103B7000137803F0E002202AE1D103F01F03012BA8
:103B800000F00581022BEAD1AB880DF11F01D8B2FC
:103B9000DFB200F0A5FB0028E8D09DF81F303BB94C
:103BA000A24B1C465B681BB1DB79002B00F08F81B8
:103BB00071F01AFB2946024630466CF0B9FEBFE7A9
:103BC0002029CCD1AB8802F01F010129D8B200F026
:103BD00005810229C3D10DF11F0100F081FB0028EE
:103BE000C4D095F90030002BC0F2968171F0FCFA38
:103BF00040230246294630466CF0C6FFA0E78B4BB7
:103C0000A98858681C46C9B2002899D09A89002A08
:103C1000ACD0024404E003781844131A002BA5DD4D
:103C20004378042BF7D183788B42F4D100238DF8AD
:103C30001F30A37C8B4202D1E37C8DF81F30A37E22
:103C40008B4204BFE37E8DF81F300DF11F0201236C
:103C5000294630466CF098FF72E77449AB884A6891
:103C60000C46DBB2002A81D0888900283FF47EAF61
:103C7000104405E011780A44811A00297FF776AFD5
:103C800051780429F6D191789942F3D1A27C6988C0
:103C90009A42884600F0F780A27E9A4200F00681A0
:103CA000A289616801EB020CA268ACEB0201002959
:103CB00065DD5FFA88FE05E011780A44ACEB02018D
:103CC00000295CDD51780429F6D191789942F3D12D
:103CD000D1787145F0D111798946002948D04FF04B
:103CE000000163F307016EF30F21CDE9033E02915A
:103CF0009046E246934604E098F80030B94598446F
:103D000033D9AAEB0803002B2FDD98F80130052BDF
:103D1000F2D14146304671F08FF900283FF41FAFD1
:103D2000636898F802101BB1DB79002B00F0EA8081
:103D300098F80330D80615D4CB0940F00C81039BCA
:103D4000A376049BA175E376B8F804300022C3F390
:103D50000A0323830092A26C304671F00DFA00280A
:103D60003FF404AF7B1CDFB2C6E7B9457FF4FEAE7B
:103D7000294630466CF062FD00283FF4F7AE2B4830
:103D8000FFF762FE294630466CF0E8FED7E6AB88C6
:103D9000D8B21B0A4CD1254B1C465B68002B3FF464
:103DA000E5AEA18900293FF4E1AE194405E01A7897
:103DB0001344CA1A002A7FF7D9AE5A78042AF6D1DA
:103DC0009A788242F3D100238DF81F3071F00CFAFB
:103DD0002946024630466CF0ADFDB1E6190A41D1E4
:103DE000124B1C465B68002B3FF4C0AEA189002932
:103DF0003FF4BCAE03EB010C06E019780B44ACEBCE
:103E0000030100297FF7B2AE59780429F5D19978DA
:103E10008142F2D1002312068DF81F307FF5E6AE05
:103E2000294630466CF09CFC8AE600BF281201202F
:103E3000D9B20DF11F0200F029FA00283FF496AE26
:103E40009DF81F3033B96F4B1C465B6813B1DB79AB
:103E5000202B66D071F0C8F92946024630466CF036
:103E60003DFD6DE60DF11F0200F010FA00283FF451
:103E70007DAE95F90030002BBFF6B8AE294630462E
:103E80006CF0EEFB5CE660480293002262826CF00C
:103E900005FA294630466CF0FFFC00283FF466AE78
:103EA0000022029BA27362622285F5E657480293C4
:103EB000002262836CF0F2F9294630466CF0ECFC8B
:103EC00000283FF453AE0022029BA275E8E6A37BD4
:103ED000BB427FF46DAE6B881B0A012B7FF468AE8A
:103EE0006B78012B7FF464AE71F07EF99DF81F3082
:103EF0000268502101FB034022F07F420262FFF77B
:103F0000A3FD55E698F80330CA0903F00C031FD14E
:103F1000002B3FF427AF12E7294630466CF01EFC19
:103F20000EE694F82A308B4294D16B881B0A012B41
:103F300090D16B78012B8DD171F056F99DF81F301F
:103F40000268502101FB03400262FFF77DFD81E71B
:103F5000002B3FF407AFBDF80830A1736382B8F8B7
:103F60000430C3F30A032382B4F840305B08A38211
:103F70009BF80030059300200BEB03026CF038FC3B
:103F80000128059B0CD05078242822D000230093D0
:103F9000E26C304671F0F0F800287FF4E3AEE5E51E
:103FA0001BF8033013445A78242AEFD19A78022A56
:103FB000ECD1DA7884F82C20012AE7D11A7984F838
:103FC0002D205A7984F82E209B6823F07F432362AA
:103FD000DCE790780128D9D1907A84F82D005079C7
:103FE00084F82C001BF803301A445378242BCDD1CD
:103FF0009378022BCAD1D378012B04BF137984F8AC
:104000002E30C3E72812012064120120581201202B
:104010000020704710B50D4C0C485022002132F0A2
:104020001FFD0B4901234FF4446204F13C006CF086
:1040300039F90848E064012307494FF4446204F168
:1040400030006CF02FF9054BA36410BD281201203D
:10405000484E0120486C0120885A01200C6D012037
:104060004B79012B02D18B79012B01D000207047B5
:10407000CB7913F0DF0FF9D12DE9F0410B7801EB8B
:10408000020E0B44734582B0844609D21878184456
:10409000864509D35C78042C06D003467345F5D3D6
:1040A000002002B0BDE8F081AEEB03000828F7DD88
:1040B00058790128F4D19B79022BF1D10B79012B8E
:1040C0002DD82CD0CB781D46002BE9D1634B5B68F3
:1040D0002BBB624B596083F800C00B78D21A002AC0
:1040E00040F3B6800B44092009E00B2A1FD01A7850
:1040F0001344AEEB03040244002C90B217DD5A784F
:10410000042AF2D15A79012A11D19A79022A0ED1C0
:10411000524A9268002AEAD1504A9360E7E74FF08A
:10412000E023D3F8F03DDD07BAD500BEB8E74B4B2E
:10413000988138B3084400260B4600274FF000084A
:1041400007E093F800E07344A0EB030EBEF1000F0C
:1041500027DD93F801E0BEF1050FF2D1CA79AAB1CB
:10416000DA78D406EDD493F802E05FEADE1265D186
:104170009A88C2F30A0297423C4638BF14467646F4
:104180002746DEE7354A012313778AE793F802E0F2
:10419000DA785FEADE1402F00C024DD1002AD0D0AA
:1041A000E6E763467DBB26B13A463146184670F0D5
:1041B00067FF2A4B98890028E4D0596801EB000C6E
:1041C0000B460BE021B191F807E0BEF1200F23D0A0
:1041D0001A781344ACEB0302002AD3DD5A78052A7F
:1041E000F0D1DA7802F0030EBEF1010FF0D193F8AE
:1041F00002E05FEADE1EEBD0D206E9D4174C9A79D2
:1042000084F82B20E4E7424629466046CDF804C0F6
:1042100070F036FF019BC6E7242AD9D19A78032A89
:10422000D6D1B3F804E040F201129645D0D10B4C40
:104230001A7A84F82A20CBE7002A82D09A88C2F31F
:104240000A029045444638BF14467546A04678E7B2
:10425000024A09239381C8186DE700BF2812012084
:1042600010B530220021054832F0FAFB04486CF00A
:1042700015F8BDE8104003486CF010B82812012072
:104280006412012058120120704700BF10B5134C72
:1042900063680BB9184610BD93F802C08646F44512
:1042A0004FF00000F7D11878D4F808C01C5C18440F
:1042B0002044ACEB0003002B06DC0CE00378184430
:1042C000ACEB0003002B06DDC3788B42F6D1002354
:1042D0001370012010BD002010BD00BF2812012066
:1042E0000E4B5A68C2B1B3F80CC09B689444ACEB57
:1042F0000302002A06DC0FE01A781344ACEB030239
:10430000002A09DD5A78052AF6D19A788242F3D13B
:1043100000230B70012070470020704728120120F5
:10432000002070472DE9F04F514CA27B8A4283B0A8
:1043300080461F4625D0A37D8B420BD1A16C002364
:10434000BAB204F130006CF077F838B9012003B04C
:10435000BDE8F08F002003B0BDE8F08F0122238B71
:104360000092A26CA17D404670F006FF0028EDD0BF
:10437000E27EA37D0092B9B2002240466CF05CFA66
:10438000E4E7E37C002BE1D0B4F84430B4F84620F5
:10439000B4F84010208A92B29BB29342B6BFC2EBEF
:1043A00041029A1AD21892B2E38C8A4228BF0A4676
:1043B000002B38D0B1EB830F35DBA18C8A4236D38A
:1043C000258DA68ADFF8B0E0A5EB030C1FFA8CFC64
:1043D000AA46B346DEF80050A6EB0C06B242A94648
:1043E00027DA002D33D1884228BF08460A23024627
:1043F000CEF80030E16C1F48002315466BF0F8FF43
:1044000001230093E26CA17B2B46404670F0B4FE82
:1044100000289BD0E27CA37B0092B9B200224046E8
:104420006CF08AFA92E7824228BF0246E2E7002255
:10443000E0E7DC44624513DD4DB98245524628BFB2
:1044400002468B42D6D00A23CEF80030D2E79842FB
:1044500028BF184609F1FF330246CEF80030C9E7FD
:10446000002DF4D1984228BF18460246C2E700BF8B
:1044700028120120641201201448012008B50AF016
:1044800027FF0E2008BD00BF70B590F80FE0D0F8F0
:1044900008C0BEF1000F13D0049CC4F800C0D0F8CF
:1044A00010C081B390F80DE0007BB2FBFEF10EFB73
:1044B0001121C008C9B201FB00C11960002070BD04
:1044C000049C4FEA5C0CC4F800C0856890F814E0C6
:1044D00004694FEA550C0EFB0CFC41B904EB0C02CD
:1044E0001A60037DC3F101030375002070BD457B95
:1044F000017BB2FBF5F605FB1622C908D2B212FB0E
:1045000001C2A218ECE7C3F800C0002070BD00BFD4
:1045100010B508468EB011461A462B4B0AACCDE9B1
:104520000034042333F0E0F90A98052207A938F093
:1045300083FD099B622B2FD0682B2AD0422B2ED0D3
:1045400030DC012B08BF002430D19DF834204AB95B
:104550000B9A089903FB02F25200B1FBF2F002FB46
:10456000101159BB1949059318203DF0FDFF9DF826
:10457000342003920C9A02929DF82C200192059B04
:10458000089A0799009404900AF08EFE04980EB0E1
:1045900010BD01240223D8E701242346D5E70024D7
:1045A0000123D2E723F02003482B04D0084840F22F
:1045B000FF216EF013FB00240223C6E7054840F2FA
:1045C000FF216EF00BFB00BFA4C80B00C4C80B009A
:1045D000B8940B00FC8C0B00704700BF08B50AF0C4
:1045E000A9FF0E2008BD00BFF0B50446C56B87B01B
:1045F0001F46E9B1012A164677D0E26AA36BE2B9F9
:10460000AB4274D0218D01350D44ED1AEB075AD51C
:1046100023693B600C9A63691360002E5AD1E36BE7
:104620000133E363E06A003818BF012007B0F0BD32
:10463000E26AA36B0E46002AE2D0AB42218DE2D1A2
:10464000236B9A4228BF1A46CB074CBFA169216948
:1046500039600123009300230593606B039205AB3F
:1046600043F0CEFD059B002B47D1039A824244D1F3
:10467000E36A9B1AE36283B912F003010DD0C1F122
:1046800004018818217B08293AD0102905D13A68FD
:1046900020F001010A4422F8023C0C9B1860218D95
:1046A000A36BCA0701F1010189B205F1010503F10C
:1046B00001030D44A5EB03054CBFE0616061A363FA
:1046C000EB072185A4D4A3693B600C9AE3691360CE
:1046D000002EA4D0012EA5D1236C227B01332364AC
:1046E0003B6803EBD2033B609CE7056C85E70C9BC2
:1046F0003A6010461A6007B0F0BD022007B0F0BD66
:10470000013A431E4FF0800C396801F803C0013BA9
:104710009A42F9D1C1E700BF70B51E460D4686B07A
:10472000114628461F4A32F0FDFF34681E4B2340D5
:10473000062B26D0A10720D0012D2BD9062203A9B4
:10474000706838F079FC40F2FF234FF480620498DF
:10475000039D082133F058F9420703461DD1134940
:10476000019344203DF000FF019B2A462146064666
:104770000AF0B2FD304606B070BD0D4B22689A4279
:10478000DAD121460B4845F2863234F067FF012D1D
:104790000446D3D800231D46E1E7074808216EF000
:1047A0001DFA00BF040002000F0080FF40C90B008B
:1047B00050660B00F8990B00C4910B0009B1012A57
:1047C00012D010B5D0E90831044682B0406BE362E4
:1047D000002201AB43F04EFD013006D00023C4E9B6
:1047E0000E33236402B010BD704701986EF096F945
:1047F00008B50AF0D5FE0E2008BD00BF2DE9F04F28
:104800002DED068B824693B01E462298DAF82430AE
:10481000E1B1012A154600F04E84DAF81820026052
:10482000DAF820109AF81C20994229D082B9DAF8D7
:10483000103033608DB9DAF824300133CAF82430EF
:10484000012013B0BDEC068BBDE8F08F0D46E4E708
:10485000DAF814303360002DEDD0012DF0D1DAF804
:1048600028309AF80C200133CAF828303368012028
:1048700003EBD203336013B0BDEC068BBDE8F08FC1
:10488000DAE90437002A18BF1F4637609AF81C304F
:1048900083F001038AF81C30DAF818304FEA930BE2
:1048A0009AF82C30002B00F00A8400249FED96AA81
:1048B000DFED969A9FED969ADFED968A0D9710950B
:1048C000119605945F460AF13005564655F804BF27
:1048D000DBF808200392002A00F0DC80002F00F0B3
:1048E000D7800D9B04930BF11003CDE90737CDE979
:1048F0000945DBF81420029742BB9BF80D304BB9F9
:104900009BF80C30002B00F0D083DBF80800114638
:1049100001F0FAFADBF80800002800F053810BF1EF
:104920001403002200931146079B01F04DFA022860
:1049300000F0A683DBF81420A0F10100B0FA80F0AB
:10494000400992088BF80D00CBF81420039B717B73
:10495000587BDBF810A088424FEA012340F03781F2
:104960000298834228BF0346934228BF13469846C5
:104970007068B8FBF1F189B25FF0A6FBF7EE000AB0
:104980000BF11800B0EE4A0A67F006F8F0EE690A7B
:10499000B0EE408A0BF11C00B0EE490A67F01EF839
:1049A00028EE288A727BBCEEC88A022A18EE103ADA
:1049B0009FB240F00A81030400F1FD80C0F5FF4082
:1049C0007F3080B24FF4004307FB00F007FB03F396
:1049D000C013DF13039B597B059BDBE90845002BC4
:1049E00040F09A80337B102B40F07E81B37B002B0C
:1049F00000F0D7818A4240F0D382B8F1000F00F076
:104A00000481049BAAF10402DDF814A0CDF818A0DB
:104A1000A3F1040E4FEA880C02EB8809A04252F879
:104A2000041F63D1AF4261D1230433FB01F34FEA8A
:104A3000054A3AFB11F123F3CF3321F3CF31C3EA17
:104A400001434A454EF8043FE8D1039B727B5B7BF0
:104A50009A4240F0C880029BDBF81420A3EB0803C5
:104A60000293049B63440493DBF81030A2EB08022A
:104A70006344CBF81030029BCBF81420CBE9080735
:104A8000002B7FF439AFDDE908740A9D96F82C30CD
:104A9000012205920134A3423FF718AF059B109DF8
:104AA000BB46B2460D9F119E002B00F008839AF87A
:104AB0000E30ABB99AF80C30102B00F04785BBF1E3
:104AC000000F0DD00BF1FF3307EB83034FF0803164
:104AD000043F57F8042F82FA41F29F423A60F8D11E
:104AE000DAF820300133CAF82030A3E6B1F5803F70
:104AF0005ED38BB2002B5BD0069B1BB14B4013F0F7
:104B0000802F55D106918FE70000000000FE7F3F07
:104B100000FE7FBF00000047337B102B77D196F853
:104B20000EC0BCF1000F00F07E818A4240F0C481CB
:104B3000B8F1000F69D0AAF10402049B4FF0000AFB
:104B4000A04202EB8809A3F1040E52F8041FCDF82D
:104B500018A04FEA880C1BD1AF4219D1230433FBB4
:104B600001F34FEA054A3AFB11F123F3CF3321F366
:104B7000CF31C3EA01435EF8041F93FA11F34A45AB
:104B8000CEF800303FF461AFA04252F8041FE3D0EA
:104B9000B1F5803F09D38BB23BB1069B1BB14B40B3
:104BA00013F0802F01D10691D8E73D460446D5E7A2
:104BB0003D46044638E700F5FF407F3083B24FF4AE
:104BC000004001E7DBF81420C0E6384602E74FEA70
:104BD0004208029A934228BF1346984528BF984638
:104BE000C6E64FEA880C049BDBF814106344049378
:104BF000029BA3EB08030293DBF810304FEA58083E
:104C000003EB8803A1EB080233E7C44623E78A429B
:104C10004FEA480340F00383002B00F02E82049AF1
:104C20000693AAF1020C0021A2F1020A0B918E4612
:104C3000624632F802CF96F80E904FEA0C414FEAE6
:104C40000C2C01F07F411FFA8CFC41EA0C01B9F1F8
:104C5000000F03D14FF0802391FA43F1A0422FD1EE
:104C6000AF422DD14FEA044C3CFB01FC4FEA054911
:104C700039FB11F92CF3CF3129F3CF39C1EA0941BE
:104C80003AF8029F4FEA094C4FEA09291FFA89F9BD
:104C90000CF07F4C4CEA090C91FA1CF14FEA114CD4
:104CA000069B0EF1010E0CF47F4CC1F307214CEA78
:104CB00001017345AAF80010BBD14FEA880CC4E685
:104CC000B1F5803F0BD31FFA81FCBCF1000F06D079
:104CD0000B9B3BB181EA030C1CF0802F02D03D46B8
:104CE0000446BFE70B91BDE78A4240F00B825FEAC2
:104CF000480300F0C28104990693A1F102090599C5
:104D00000B91AAF102028A4632F802CF96F80EE021
:104D10004FEA0C414FEA0C2C01F07F411FFA8CFC4A
:104D200041EA0C01BEF1000F03D14FF0802391FA4C
:104D300043F1A04221D1AF421FD14FEA044C3CFBCA
:104D400001FC4FEA054E3EFB11FE2CF3CF312EF352
:104D5000CF3CC1EA0C414FEA114C069B0AF1010A13
:104D60000CF47F4CC1F307214CEA01019A4529F864
:104D7000021FC9D14FEA880C67E6B1F5803F0BD31B
:104D80001FFA81FCBCF1000F06D00B9B3BB181EAFE
:104D9000030C1CF0802F02D03D460446CDE70B915A
:104DA000CBE78A4240F05483B8F1000F3FF42DAFB7
:104DB000049ACDF818B0AAF10403A2F1040E059AE2
:104DC0000B924FEA880C03EB880A4FF0802953F8C6
:104DD000042F92FA49F2A04215D1AF4213D1210417
:104DE00031FB02F14FEA054B3BFB12F221F3CF31CD
:104DF00022F3CF32C1EA024153454EF8041FE6D1F7
:104E0000DDF818B021E6B2F5803F07D391B229B1A1
:104E10000B9931B1514011F0802F02D03D4604462C
:104E2000DDE70B92DBE78A4240F09682B8F1000F93
:104E30003FF4EBAEAAF10403049ACDF82CC003EBC7
:104E4000880AA2F1040E53F8041FCDF818B04FEAF7
:104E5000880C4FF0802991FA49F1A0421CD1AF4251
:104E60001AD1220432FB01F24FEA054B3BFB11F150
:104E700022F3CF3221F3CF31C2EA01425EF8041FA0
:104E800092FA11F25345CEF80020B9D053F8041F1E
:104E900091FA49F1A042E2D0B1F5803F07D38AB23E
:104EA0002AB10B9A32B14A4012F0802F02D03D460F
:104EB0000446D6E70B91D4E7B8F1010F7FF691AE27
:104EC00004994FEA5803AAF1040C01EBC30E8A4679
:104ED00000210C91CDE90EB60104069139040B9125
:104EE0005CF8042FA04293B243EA024348D1AF4298
:104EF00046D121044FEA054931FB03FB39FB13F38B
:104F00002BF3CF3B23F3CF33CBEA0343DAF8006034
:104F100093FA16F3CAF80030130C1B04A04243EABC
:104F200012431AD1AF4218D131FB03F139FB13F30D
:104F300021F3CF3123F3CF33C1EA0342DAF804304F
:104F400092FA13F2CAF804200AF1080AF245C7D10E
:104F5000DDE90EB64FEA880C77E5B3F5803F07D35D
:104F60009AB22AB10C9A4AB15A4012F0802F05D059
:104F70000699DDF82C903D460446D5E70C93D3E71F
:104F8000B3F5803F07D399B229B10C9931B159409B
:104F900011F0802F02D03D460446AAE70C93A8E703
:104FA000B8F1010F7FF61DAE0499CDF838B04FEA85
:104FB000580301EBC303AAF104098A4605990C9131
:104FC0000104069139040B919B4659F8042FA04225
:104FD00093B243EA024340D1AF423ED121044FEAAB
:104FE000054E31FB03FC3EFB13F32CF3CF3C23F3C4
:104FF000CF33CCEA0343CAF80030130C1B04A042A1
:1050000043EA124316D1AF4214D131FB03F13EFB08
:1050100013F321F3CF3123F3CF33C1EA0341CAF8AD
:1050200004100AF1080ADA45CFD1DDF838B04FEAAA
:10503000880C0AE5B3F5803F07D39AB22AB10C9ADF
:105040004AB15A4012F0802F05D00699DDF82CE0C5
:105050003D460446D9E70C93D7E7B3F5803F07D325
:1050600099B229B10C9931B1594011F0802F02D079
:105070003D460446B2E70C93B0E74FEA880CEAE4F9
:10508000DDE9087400230A9DCBF80830CBF8143012
:105090008BF80D30059B2BB9029BDDE904019A00CA
:1050A00031F0DEFC96F82C30F2E4DDE908740A9D5C
:1050B000CBF80820EEE7DAF82830FFF7AEBBBBF1FB
:1050C000000F3FF40DAD4FEA8B020021384631F05E
:1050D000C7FC9AF80E30002B7FF402AD9AF80C3022
:1050E000102B7FF4EFAC0BF1FF3107EB81013B1F7D
:1050F0004FF0802053F8042F92FA40F28B421A604E
:10510000F8D1EDE44FEA4803012B7FF66AAD049A2B
:10511000CDF83880010408F1FF3306913904AAF173
:1051200002090AEB430ECDE90B1B02F1020A059AB4
:10513000904639F8023FB27B19041B0201F07F410F
:105140009BB219431AB94FF0802391FA43F18BB205
:10515000A04243EA014350D1AF424ED122044FEA6C
:10516000054C32FB03FB3CFB13F32BF3CF3B23F348
:10517000CF33CBEA03434FEA134B0BF47F4BC3F31C
:1051800007234BEA030B0B0C1B04A0422AF802BCBA
:1051900043EA11431CD1AF421AD132FB03F23CFB6C
:1051A00013FC22F3CF332CF3CF32C3EA02431A0CA1
:1051B00002F47F42C3F307231343F1452AF8043B6B
:1051C000B7D1DDF83880DDF830B04FEA880C3CE428
:1051D000B3F5803F0BD399B249B1B8F1000F00F09D
:1051E000AD8183EA080111F0802F00F0A781069AB3
:1051F000DDF82CC03D460446CFE7B3F5803F0BD326
:105200009AB24AB1B8F1000F00F09A8183EA08021D
:1052100012F0802F00F094813D4604469EE7012B5A
:105220007FF6DFAC049A08F1FF330AEB4303AAF1DF
:10523000020E02F1020A0022069202040B923A04C4
:10524000CDE90EB80C929B463EF8023FB27B1904A2
:105250001B0201F07F419BB219431AB94FF0802322
:1052600091FA43F18AB2A04242EA014264D1AF42CC
:1052700062D123044FEA054C33FB02F83CFB12F2E7
:1052800028F3CF3822F3CF32C8EA02493AF8028C29
:105290004FEA08424FEA08281FFA88F802F07F42D6
:1052A00042EA080299FA12F24FEA124808F47F48DB
:1052B000C2F3072248EA02080A0C1204A0422AF8A4
:1052C000028C42EA114225D1AF4223D133FB02F3D3
:1052D0003CFB12F223F3CF3322F3CF32C3EA024373
:1052E000BAF800100A04090289B202F07F420A43A8
:1052F00093FA12F31A0C02F47F42C3F30723134309
:10530000F3452AF8043B9FD1DDE90EB84FEA880C3B
:10531000FFF79BBBB2F5803F09D391B239B1069933
:1053200019B1514011F0802F01D10692CEE7DDE98D
:105330000B3C3D460446C9E7B2F5803F09D393B222
:105340003BB1069B1BB1534013F0802F01D1069255
:105350008FE73D4604468CE7B8F1010F7FF641AC7C
:10536000020404990B924FEA58033A04CDE90EB8AF
:10537000AAF1040A0C9201EBC30EB046CDF818C096
:105380005AF8043F4FF0802293FA42F91FFA89F34A
:10539000A04243EA09434BD1AF4249D122044FEA2C
:1053A000054C32FB03FB3CFB13F32BF3CF3B23F306
:1053B000CF33CBEA03430E6893FA16F30B604FEA40
:1053C00019431B04A04243EA19431BD1AF4219D130
:1053D00032FB03F23CFB13FC22F3CF332CF3CF322E
:1053E000C3EA02424B6892FA13F34B6008318E45D0
:1053F000C6D14646DDF83C80DDF838B04FEA880C6F
:10540000FFF723BBB3F5803F0DD31FFA83F9B9F142
:10541000000F08D0069E26B183EA060919F0802FF6
:1054200001D10693D4E7DDE90B2C3D460446CFE7D6
:10543000B3F5803F09D39AB23AB1069A1AB15A40ED
:1054400012F0802F01D10693A8E73D460446A5E758
:10545000B8F1010F7FF6C5AB049ACDF838804FEA5A
:10546000580302EBC30301049146059A06913904DF
:10547000CDE90B1BAAF1040AB346984616465AF822
:10548000043F4FF0802293FA42FC1FFA8CF3A042B3
:1054900043EA0C4344D1AF4242D12204290432FBF7
:1054A00003FE31FB13F32EF3CF3E23F3CF33CEEACB
:1054B0000343C9F800304FEA1C431B04A04243EAEF
:1054C0001C431AD1AF4218D132FB03F231FB13F364
:1054D00022F3CF3223F3CF33C2EA0343C9F80430B7
:1054E00009F10809C145CAD1DDF838805E464FEAA6
:1054F000880CDDF830B0FFF7A8BAB3F5803F0AD3C7
:105500001FFA83FCBCF1000F05D0EEB183EA060C54
:105510001CF0802F18D0069A0B993D460446D3E71D
:10552000B3F5803F07D39AB22AB15EB183EA06028F
:1055300012F0802F06D03D460446AEE798462CE692
:1055400098460BE61E46A8E71E46BDE7BBF1000FD6
:105550007FF4C9ADFFF7C4BA2DE9F04308468BB01C
:1055600011461A462E4B04ACCDE90034062332F026
:10557000BBF940F28463FF220121049832F010FA53
:1055800040F21533022201210746069832F008FA4C
:1055900040F2925204460121099832F0F5F9079D34
:1055A000082D804601D0102D37D107F10D001D497F
:1055B00080003CF0D9FFE4B29DF820300093059ABA
:1055C000CDF808800194EBB2F9B2064609F0B8FFB5
:1055D000002F17DDDFF8548098F8083008EB8303BC
:1055E00006F13005D3F810900024002319461A461E
:1055F0004046C847013445F8040F31460AF064F8C4
:10560000A742F2D196F82C0006F134013DF064FC7B
:10561000306330460BB0BDE8F08303486DF0D6FA36
:105620000CCA0B005CCA0B00F8830B0038CB0B00D4
:1056300000B583B0019000F0BBFB019809F0BCFFFE
:1056400000280CBF1E203E2003B000BD00B583B073
:10565000019000F0ADFB0198006B03B000BD00BFEE
:1056600030B551F8044B89B005462046CDE90221FA
:1056700000F09EFB05AB01930E4B0093DDE9022188
:10568000681E032332F088F894F82C20069840F224
:1056900083630021013A32F083F9C0B204EB800049
:1056A0009DF81C200599406B09F0CAFF204609B0FF
:1056B00030BD00BF44CA0B0030B551F8044B87B071
:1056C00005462046CDE9022100F072FB05AB0193AF
:1056D0000C4B0093DDE90221681E012332F05CF8D7
:1056E00094F82C20059840F283630021013A32F0AF
:1056F00057F9C0B204EB8004606B09F0E7FF0E209D
:1057000007B030BD3CCA0B0090F82C307BB170B5AF
:10571000064600F13005002455F8040F09F0A2FFF9
:10572000013496F82C20E3B29A42F5D870BD704748
:1057300000B5084683B01146002231F0F3FF054959
:1057400028203CF009FF019009F050FF019803B0B8
:1057500000BD00BF38CB0B0008B509F05FFF0E207D
:1057600008BD00BF09F060BF08B509F05FFF002861
:105770000CBF1E203E2008BD09F05ABF08B509F035
:1057800059FF00280CBF1E203E2008BD10B584B074
:1057900002AB51F8044B0193074B009301380223ED
:1057A00031F0FAFF20469DF80C20029909F048FFDD
:1057B0000E2004B010BD00BF28CB0B0008B509F0C7
:1057C00071FF0E2008BD00BF10B5044608463CF02E
:1057D000FFFC0146204609F06DFF0E2010BD00BF02
:1057E00008B509F069FF0E2008BD00BF10B584B0F0
:1057F00003AB51F8044B0193054B0093013801238F
:1058000031F0CAFF204609F061FF0E2004B010BD40
:1058100020CB0B0008B509F0BDFF0E2008BD00BF6E
:1058200070B5456A86B0002D00F0A68004460029B8
:1058300053D011460A98A568056094F9540088422F
:105840006FD0C2F1010284F8542094F84420B2FAD7
:1058500082F2520904EB820184F8442084F8552036
:105860004A6B1A602046164631F026FE002120467B
:1058700031F0E0FD014600286ED0D4E90B239B1ADD
:105880000493636A1344059300230093206933460D
:1058900004AA05A9F5F72EFD431C20D0226B04991C
:1058A000521AE26230B3002103902A46304631F0AA
:1058B000D7F894F84510039B002960D1023319D022
:1058C000A2680391304631F0CBF80A9A039911602F
:1058D000012384F84530022021E00A46AAE703901C
:1058E0002A460021304631F0BBF894F84520039B4E
:1058F000002A44D1A36D03EB55032046A36531F084
:10590000DBFD0021204631F095FD0546D4E90B0171
:10591000A26A091A521AB2F5007F16DC284606B0B0
:1059200070BD94F9551004EB81010120496B01EB26
:1059300042021A60FF210A9B84F854101A68A36D72
:1059400003EB5203A36506B070BD1749224604F16C
:10595000140000F079FBE1E7A2680391304631F0D2
:105960007FF80A9B0399196094F8450080F00100C4
:105970004000C0B206B070BD0A9B1D60ABE7A268D4
:1059800003930021304631F06BF8039B03330A9BED
:105990004FF001024FF000018CBF00200120196080
:1059A000904084F84520BAE7B976060070B51E46E7
:1059B0000D4686B0114628461C4A31F0B3FE3468C5
:1059C0001B4B2340062B1ED0A30718D001212046D5
:1059D00037F0A8FB037C13F0010324D1012D1AD862
:1059E0001E46144901935C203CF0BEFD019B3246EB
:1059F0002146054609F06EFE284606B070BD0E4BE6
:105A000022689A42E2D121460C4845F2863233F0B0
:105A100025FE0446DAE77068062203A937F00CFB7E
:105A2000DDE90363DDE706486DF0BCF80400020021
:105A30000F0080FF1CCC0B0050660B00F8990B0088
:105A4000F07F0B0000B583B0019000F0B1F9019830
:105A5000006C03B000BD00BF00B583B0019000F042
:105A6000A7F9019809F0A8FEB4EE400AF1EE10FA89
:105A700009D610EE103A23F0030040F00200A0F126
:105A8000FF4003B000BD0148FBE700BF020040003B
:105A900000B583B0019000F08BF9019809F0CCFEBD
:105AA000400040F0010003B000BD00BF10B582B05F
:105AB0000446019100F07CF90199064845F28632CE
:105AC00033F0CCFD0146204609F0B8FE0E2002B0AE
:105AD00010BD00BFF8990B0038B50C46054600F024
:105AE00067F90121204637F01DFB037CDB0705D455
:105AF0002846214609F0A2FE0E2038BD01486DF06F
:105B000051F800BFF07F0B0009B1012A24D010B575
:105B1000044682B000F0ECFA94F8453023B902B0A4
:105B2000BDE8104000F0C0BA0022206C114663F0BE
:105B300011F90028F3D1FF23C4E90B0084F84500D4
:105B4000A065019084F85430204631F0B5FC0199ED
:105B5000204631F06FFCE2E7704700BF08B509F05E
:105B600041FF0E2008BD00BF10B5084688B01146A1
:105B70001A46114B0DF1140CCDE9003C032331F012
:105B8000B3FE05984FF48C6170F0DEF940F271516C
:105B90000446069870F0F0F90849039024203CF080
:105BA000E3FCBDF81C30039A0290214609F0E2FEA6
:105BB000029808B010BD00BF08CD0B0030CD0B001F
:105BC00010B5044609F050FF38B9204609F052FFDD
:105BD00000280CBF1E203E2010BD59F0F7FF00BF6B
:105BE00010B5044609F040FF38B9204609F044FFDB
:105BF00000280CBF1E203E2010BD59F0E7FF00BF5B
:105C000010B5044609F030FF40B9204609F034FFD2
:105C100030B1204609F03CFF0E2010BD59F0D6FFF0
:105C200001486CF09FFF00BF7C8B0B0030B50C6807
:105C300087B005462046CDE9022109F015FFDDE9D0
:105C4000022188B904AB0193084B0093681E02231C
:105C5000043131F0A1FD20469DF81420049909F08B
:105C60001FFF0E2007B030BD59F0B0FF20CD0B0054
:105C700010B5044609F0F8FE50B9204609F0FAFEC6
:105C800008B90E2010BD204609F0BEFF0E2010BD41
:105C900059F09CFF10B5044609F0E6FE20B92046F5
:105CA00009F0C2FF0E2010BD59F090FF3E4BD3F813
:105CB0000021D00050D510B53C4B84B003F1100446
:105CC00053F8040BB8B1C27F42B98168D1F804C15E
:105CD000BCF1000F02D04277C1F80421427F52B1DB
:105CE000827F62B18268D2F8101141B3D2F81411E8
:105CF00069B3012151609C42E2D104B010BDC27F62
:105D0000002AF8D190F82220002AF4D18168D1F835
:105D100008C1BCF1000F38D1D1F80C214ABB90F971
:105D20001C20002AE7DB5109DFF87CC002F01F02CB
:105D30006031012000FA02F24CF82120DBE7D2F8B2
:105D400008110029D7D1D2F814110029D1D1D2F8E5
:105D50000C110029CFD1CCE7D3F804219107AAD4A4
:105D6000D3F804215207A6D4D3F804319B04A2D45B
:105D7000704700210293019025F092FF0198029B49
:105D800082680021C2F80C11C9E70121CDE9023275
:105D9000019025F085FF0198039A8168029BC1F864
:105DA00008218168B8E700BF00E100E0380A01205F
:105DB00008B5437B03B108BD59F008FF407BB0FA3A
:105DC00080F04009704700BFF0B583B004460E462E
:105DD000014640F21A50CDE90032089D40F00EFD18
:105DE00007462046FFF7EAFFDDE9003240B9089593
:105DF000BD6831462046AC4603B0BDE8F040604780
:105E0000002202201A602A6003B0F0BD0023437311
:105E1000704700BF30B583B00C46054640F21A50BB
:105E2000019240F0EBFC2046FFF7C2FF61686B680F
:105E3000019A994211D16B7B62B9627B9A421BD164
:105E4000227B2B7B9A4212D1A27BAB7B9A4209D157
:105E500003B030BD022BF0D1F2E70A4840F2925174
:105E60006CF0BCFE074840F2C7516CF0B7FE054825
:105E70004FF43A716CF0B2FE024840F215316CF00A
:105E8000ADFE00BFCC880B0008B5437B23B1007B7F
:105E9000400040F0010008BD59F098FE407B18B169
:105EA000400040F00100704708B559F08FFE00BF78
:105EB00000B5437B83B063B10146019040F21A50B4
:105EC00040F09CFC01994868400040F0010003B09C
:105ED00000BD59F07BFE00BF38B5437B93B104464B
:105EE0000D46014640F21A5040F088FC28463AF030
:105EF000C5FF40F29252012131F046FD0346636036
:105F00000E2038BD59F062FE2DE9F04104460F46DF
:105F100040F21A502146164640F070FC05462046D5
:105F2000FFF74CFF30B96B68324639462046BDE872
:105F3000F0411847BDE8F081704700BF014B0022D7
:105F40001A7070472D7C01200349044B0120002268
:105F500008701A60704700BF2D7C0120446C01203E
:105F6000014B1878704700BF2D7C0120024B186848
:105F7000003818BF01207047446C012008B50D4B54
:105F8000186818B10C4A12680AB1002008BD65F003
:105F900059F9084B1A681B688242A0EB030088BFBE
:105FA00000F1FF3040F2EE23984294BF0020012020
:105FB00008BD00BF446C0120B4460120014B002203
:105FC0001A607047446C0120024A136823EA0003F8
:105FD00013607047B4460120024A136803431360FC
:105FE000704700BFB4460120134B1B7813B1134B0D
:105FF0001B6803B1704700B5114B83B01A6801925A
:1060000065F020F90E4B019A1860196811B132B190
:1060100003B000BD196801311960002AF8D10120D0
:1060200064F0AEFB074B03F178029A6203B05DF8AF
:1060300004EB57F027BC00BF2D7C0120B4460120A3
:10604000446C01205C710120C0E9001200F000B82E
:1060500000B583B0019011F01BFE0198C368BBB975
:106060000F490A68824213D00E4A8360D2F800C0FA
:106070001368C0F80CC00BB1136898600B6863B16B
:10608000106011F04BFE03B05DF804EB57F0FABB63
:1060900003B05DF804EB11F041BE0860F0E700BF0B
:1060A000C4460120CC46012008B511F0F1FD044A98
:1060B0001368013B1360BDE8084011F02FBE00BF1C
:1060C000B846012010B5054B1C682CB1606827F05C
:1060D00025FEA468002CF9D110BD00BFC4460120E4
:1060E000024B1868003818BF01207047C4460120D1
:1060F00008B511F0CDFD044A136801331360BDE803
:10610000084011F00BBE00BFB84601202DE9F04356
:10611000DFF8709083B00027019711F0B9FDD9F82E
:1061200000504DB30DF104083E4602E00023E36049
:10613000ADB12C462846AD68A66028F00BF90028C2
:10614000F4D1606828F006F90028EFD13B46C8F882
:106150000040274604F10808E360002DE9D1019AC8
:106160000649074BC9F8002000220F601A6011F0A1
:10617000D5FD03B0BDE8F0832F46F0E7CC46012003
:10618000B8460120C44601202DE9F041164E57F0D3
:106190003DFA336833B3DFF8588011F079FDD8F851
:1061A0000050DDB93468114B35600122C8F8002079
:1061B0001D608CB12346D3E90067A468C3E902558A
:1061C00011F0ACFD384606B1B04711F061FD002C6E
:1061D000F0D1D8F80050013DC8F80050BDE8F041BA
:1061E00011F09CBDBDE8F081C4460120CC460120E1
:1061F000B846012008B53AF0BBFE03460348D988EB
:10620000972914BF972242226CF0D4FC28830B00FC
:10621000014A042358F076B8240D0C0000B5084656
:1062200089B011461A460F4B0DF1100CCDE9003C18
:10623000042331F059FB4FF47A720698012131F0B2
:10624000A3FB0949039018203CF08EF907990091AF
:10625000059A0290DDE903315EF01AF8029809B060
:1062600000BD00BF10CE0B00A8CE0B0008B55EF03D
:1062700055F80E2008BD00BF10B504465EF06CF85E
:1062800038B920465EF0FEF800280CBF1E203E20E4
:1062900010BD59F09BFC00BF10B504465EF05CF8E1
:1062A00020B920465EF000F90E2010BD59F08EFC9A
:1062B00038B504460D465EF04FF878B920465EF0DA
:1062C0004FF868B128463AF0D9FDC1B220465EF0D9
:1062D00049F800280CBF1E203E2038BD59F076FC3E
:1062E00007F0BCF9F0B50C6887B0064620460D46AD
:1062F00017465EF031F8C0B920465EF031F8B0B113
:1063000002AB01930B4B00930423E9183A46701E2D
:1063100031F042FADDE90430DDE902120090204656
:106320005AF04EF90E2007B0F0BD59F04FFC07F0BF
:1063300095F900BF88CE0B0070B505465EF00CF8ED
:10634000F8B9044628465EF00BF8E0B12146204635
:106350003CF034FC0824064602E00134782C0ED0D0
:10636000E1B228465DF0FEFF0028F6D0610041F062
:106370000101304601343BF0B1FF782CF0D13046BA
:1063800070BD59F023FC07F069F900BFF0B50C6847
:1063900087B0064620460D4617465DF0DDFFD0B9B2
:1063A00020465DF0DDFFC0B102AB01930C4B0093C2
:1063B00004233A46E918701E31F0EEF9DDE90431A4
:1063C0000120CDE90010039A0299204671F066FD84
:1063D0000E2007B0F0BD59F0F9FB07F03FF900BF00
:1063E00030CE0B002DE9F0410C688AB007462046FC
:1063F0000E4690465DF0B0FF18BB054620465DF0A6
:10640000AFFF00B3114B009303AB4246311D781E22
:106410000193072331F0C0F9DDE90631049ACDE993
:1064200000152046039971F039FDDDE90830059A21
:106430000090039920465AF0C3F80E200AB0BDE838
:10644000F08159F0C3FB07F009F900BF50CE0B00F3
:106450002DE9F0410C6886B0074620460E4690466E
:106460005EF00AF9002839D1054620465EF008F9A9
:10647000002835D01C4B009302AB4246311D781EDC
:106480000193042331F088F9029840F2D7220121C8
:1064900031F07AFA2946074640F20953039801225F
:1064A00031F07EFA2946064640F2F943049801226B
:1064B00031F076FA40F2E6230546092205980821D4
:1064C00031F06EFAC0B20090EBB22046F2B239461B
:1064D0005EF026F80E2006B0BDE8F08159F076FB9C
:1064E00002486CF03FFB00BFF8CF0B00508E0B0052
:1064F00000B5084689B011461A460A4B0DF1140C36
:10650000CDE9003C032331F0EFF9074918203CF0B6
:106510002BF8DDE90623059903905EF029F803982E
:1065200009B000BD78CF0B0018D00B0008B55EF0A5
:1065300075F80E2008BD00BF10B504465EF09CF84B
:1065400038B920465EF0B4F900280CBF1E203E206A
:1065500010BD59F03BFB00BF10B504465EF08CF84F
:1065600020B920465EF0BAF90E2010BD59F02EFB7E
:106570002DE9F0410D688CB0074628460E4690463E
:106580005EF07AF8002842D1044628465EF078F89A
:10659000002839D01F4B009308AB4246311D781EAE
:1065A0000193042331F0F8F8062205A9089836F083
:1065B00043FD22469DF81C10402031F023FB044689
:1065C000DDE9090104AA039003A8069BB3FBF4F3D9
:1065D00004934FF0C7FEDDE9031304FB01F103FB55
:1065E00004F2CDE903121AB90E200CB0BDE8F08117
:1065F00005989DF82C30014428465EF045F80028A7
:10660000F2D105206CF08AFA03486CF0ABFA59F02D
:10661000DDFA00BFC0CF0B00508E0B002DE9F0411A
:106620000D688AB0074628460E4690465EF024F86C
:10663000002840D1044628465EF022F8002837D0D2
:106640001E4B009304AB4246311D781E0193032379
:1066500031F0A2F8052207A9049836F0EDFC224695
:106660009DF82410402031F0CDFA0446DDE9050103
:1066700003AA029002A8089BB3FBF4F303934FF024
:1066800071FEDDE9023204FB03F304FB02F2CDE903
:1066900002321AB90E200AB0BDE8F08107992846E7
:1066A00019445EF021F90028F4D105206CF036FA87
:1066B00003486CF057FA59F089FA00BFE0CF0B009D
:1066C000508E0B002DE9F0410E6892B0074630461F
:1066D0000C4690465DF0D0FF002866D10546304656
:1066E0005DF0CEFF00285DD0314B00930CAB211D37
:1066F0004246781E0193062331F04EF8052206A982
:106700000C9836F099FC2A469DF82010402031F074
:1067100079FA0446DDE90E0103AA029002A8079B5C
:10672000B3FBF4F303934FF01DFE062209A90D9865
:1067300036F082FC2A469DF82C10402031F062FA97
:106740000546DDE9100105AA049004A80A9BB3FBE5
:10675000F5F305934FF006FEDDE90213049A059860
:1067600004FB03F305FB02F200FB05F504FB01F15A
:10677000AB42CDE903320291059510D11BB90E2031
:1067800012B0BDE8F0810998069C024421443046CD
:106790005EF004F80028F2D105206CF0BFF905483E
:1067A0006CF014FA04486CF0DDF959F00FFA00BFF0
:1067B00090CF0B00C0830B00508E0B002DE9F843E7
:1067C000047B076E064604F01F044FF0FF33A3401E
:1067D0008C4200687568884627EA030728D24FF084
:1067E000000919E038B9B568B36F4FF40072294653
:1067F0003046984770B315F8013B0138B9F1000FE6
:1068000010D023B386F864304FF00009FF2308341A
:10681000A04543EA07270BD996F86430002BE1D056
:10682000FF23F4E7FF2BF2D1A0454FF00109F3D885
:10683000C6E900052346A3EB0803A4EB080404F013
:106840001F043766337327FA04F0BDE8F8839946CE
:10685000FF23DCE76FF00100BDE8F8830EF098BA83
:106860002DE9F04317885488B2F80480D68893B095
:106870002422E41B0546894601340DEB0200002169
:1068800030F0EEF804EBD4725210B5F94A3EADF890
:1068900030204FF48872A6EB0806A3EB0803ADF88E
:1068A0003220012201360D92002B4FF6FF72CDF8F7
:1068B0002C90ADF82840ADF82A60ADF844203BDDBF
:1068C000B5F9482ED21B002A32DDB342B5F9460E87
:1068D000B5F9441EA8BF33469442A8BF1446B5F884
:1068E000402EB5F8426EA0EB0800C91B4ABF521AF1
:1068F00009B200210028B6BF361A00B20020CDE947
:1069000000101BB224B20393029495F8554ED5F8AB
:106910003C0E0794D5F8504E069495F8544E0594C5
:10692000D5F84C4E049433B212B209A909F056FDC1
:10693000012013B0BDE8F083002013B0BDE8F08360
:10694000F0B50E2A83B06CD0154604460E460EF004
:10695000DBF9002868D1B2072CD0F30731D5A18824
:10696000E38801FB03F3B3EB660F4FEA660052D9ED
:1069700090FBF1F201FB1200042D06B217B240D0D9
:1069800028463AF07BFA054620460EF0FFF94FF014
:10699000FF32C0F12003DA402846A223002130F064
:1069A000FFFF3A460346314620460EF051FA0E20CC
:1069B00003B0F0BD214B32689A42CED120486CF032
:1069C00099F8304601AA02213AF066F9019B18684D
:1069D0003AF054FA061EA38828DB9E4226DA019B71
:1069E00058683AF04BFA021EE38803DB9A42B8BFBC
:1069F0003046C1DB1348013B00224FF4D5616CF0F7
:106A00006DF83A46314620460EF0E4F9400040F079
:106A1000010003B0F0BD0B48013B00225C216CF08B
:106A20005DF809486CF042F859F0D0F80548013B90
:106A3000002240F2A2616CF051F800BF34630B00F9
:106A400088890B00E8940B0020910B00F0B52F4BC8
:106A50008DB007ACCDE90034052330F09DFE2C4904
:106A600007984FF45C7231F02DF8294940F2EE524C
:106A7000DDE9075031F026F8DDE90860244940F2ED
:106A8000EF5231F01FF8DDE9097420463BF06AFA55
:106A900010BB012204A9204636F0CEFA40B3059B74
:106AA000B3F5805F24D1049B13B30B980E2811D04B
:106AB0004FF490621649039331F004F80B9A039B4C
:106AC00000932846134631463A465DF075FF079815
:106AD0000DB0F0BD0022F3E721460E4832F094FDE0
:106AE0000446012204A9204636F0A6FA0028D6D191
:106AF00020463AF03DFAC2880092074840F221232E
:106B0000432240F275416CF055F800BF0CD10B00E8
:106B1000D4E20B0068D20B0090940B0030B5174BF9
:106B200087B003ACCDE90034032330F035FE1449BF
:106B3000039840F2E32230F0C5FF124940F2ED42E3
:106B4000DDE9035030F0BEFF049C40F2ED42A06846
:106B50004FF4807130F034FF05980E280CD00849AE
:106B60004FF4906230F0AEFF0599626828465EF0FF
:106B70005DF8039807B030BD0021F6E744D10B0063
:106B8000D4E20B0050E60B002DE9F04F2DED028B07
:106B90005F4BA9B005ACCDE90034032330F0FCFD18
:106BA0005C49059840F2E32230F08CFFDDE90530C6
:106BB00003933AF0DDF9C37B002B40F08E80069DF5
:106BC0002E462F4628AB0DF12008B3EE0F8A0DF1AB
:106BD0001F040DF13F09C3F1810A0AEB040307EE1C
:106BE000103AB8EEC77A2846C7EE087A17EE903A00
:106BF000F4EE677AF1EE10FA23F0030B4BF0020B80
:106C00006CBFDFF818B1ABF1FF4B594632F0FCFC1A
:106C10003AF0BAF820EE080A5AF044FEFDEEC07AC7
:106C2000B54217EE902A594604F8012F30460BD092
:106C300032F0EAFC3AF0A8F820EE080A5AF032FEE8
:106C4000FDEEC07A17EE902A4C4584F86020C4D13E
:106C50006FF01E049FED308A304D08F15F06A4EB03
:106C6000080404EB090307EE103AB8EEC77A384679
:106C7000C7EE087A17EE903AF4EE677A23F0030134
:106C8000F1EE10FA41F0020174BFA1F1FF41294673
:106C900032F0BAFC3AF078F820EE080A5AF002FE18
:106CA000FDEEC07A17EE903A09F8013F4E45D8D173
:106CB00007980E280FD017494FF4906230F002FF6A
:106CC0000799039842465EF039F8059829B0BDEC63
:106CD000028BBDE8F08F0021F3E706983AF048F9FF
:106CE000044606983AF044F9C27B0D4B04EB82044B
:106CF00022699A427FF463AF069C40F27542606855
:106D0000032130F05DFED4E9025726695AE700BF3F
:106D10005CD10B00D4E20B0000007C42020040007A
:106D2000E54D07002DE9F0414F4B92B003ACCDE9A2
:106D30000034032330F030FD4C49039840F2E32245
:106D400030F0C0FE3022002106A8039F2FF088FEFD
:106D5000049E16F0030410D030463AF009F9C288B8
:106D6000434840F21313CDE9003240F23A214FF488
:106D7000897340F23B226BF031FF33683D4A934206
:106D80003FD03D4A93424ED03C4A934221D03C4AA8
:106D90009342E1D106AD44F00101042230463DF0BA
:106DA000CDFE39F0F1FF0234182CA5EC010AF2D126
:106DB00005980E2823D02D494FF4906230F082FEC2
:106DC0000599384606AA5EF00BF8039812B0BDE8A4
:106DD000F0812C4B610041F0010104223046A3FBFD
:106DE00004353DF0ABFE39F0CFFF04EB550501341F
:106DF0000DEB8505092C85ED060AEAD1D8E70021BF
:106E0000DFE706AD44F00101042230463DF096FE76
:106E100039F0BAFF02342B46062C05F1140583ED38
:106E2000000AEFD1C4E70DF1180845460224A11E5F
:106E300041F00101042230463DF080FE39F0A4FF0C
:106E400044F0010188ED000A042230463DF076FE50
:106E500039F09AFF04340E2C85ED030A08F114086A
:106E600005F11005E3D1A3E78CD10B00D4E20B00B0
:106E700058750B00B8D30B0068D30B000CD30B0074
:106E8000A4D20B00ABAAAAAA2DE9F04F2DED028BDC
:106E90008FB04F4B04AF07F10804CDE9003408234D
:106EA00030F07AFC4B49B86840F2E32230F00AFE39
:106EB000786ABB687B600E286ED046494FF49062BA
:106EC00030F000FE7B6A3B60786939F05DFFD7F8EF
:106ED0000C804046B0EE408A3BF0BAF9002869D0F9
:106EE000C30767D5461007EE906AB8EE670AB5EE9D
:106EF000400AF1EE10FA58D4F1EEC07AFDEEE77ACE
:106F000017EE909A19F0010F5FD009FB09F39E422A
:106F10005BD1B300073323F00703ADEB030D0DF195
:106F2000100A002E3BD00024AAF1040B2546610074
:106F3000042241F0010140463DF000FE39F09EFF81
:106F40000134A6424BF8040F0544F0D138690E28ED
:106F500018D039F019FF97F82020FB69CDE90132EC
:106F60003B7E0093D7E90010F0EE480A53464FEA03
:106F700059025DF0E9FFB8682C37BD46BDEC028BC5
:106F8000BDE8F08F75B107EE905AF8EEE77AB7EEEC
:106F9000007A87EE270ADEE700233B6094E7386932
:106FA0000E28D6D1B7EE000AD5E760F073F9F0EEFF
:106FB000407AA3E7404639F0DBFF4FF41072C388F4
:106FC00005484FF4D2616BF009FE04486BF0FEFDFA
:106FD000A4D10B00D4E20B007C940B006C750B0069
:106FE00000B52DED028B184B89B00DF1140CCDE9D5
:106FF000003C032330F0D0FB0698F8B139F0C4FE12
:10700000B0EE408A1149059840F2E32230F05AFD73
:107010000798059B0E2814D00C4903934FF49062F7
:1070200030F050FD0799039B1846B0EE480A5EF019
:10703000DBF9059809B0BDEC028B00BDB6EE008A05
:10704000E0E70021F0E700BF74D10B00D4E20B00B1
:107050002DE9F04F2DED028B624B93B008ACCDE9DA
:1070600000340A2330F098FB5F49089840F27132EF
:1070700030F028FD5C4940F2DF520546099830F0B7
:1070800021FD594906464FF4BC620A9830F01AFDBA
:1070900007460C980E2800F0848039F075FEB0EE9B
:1070A000408A0D980E2875D039F06EFEF0EE408AB9
:1070B0000B994E484FF44B721BF01AF940F2F12233
:1070C0000E9904464A481BF013F9AA88B3889342E4
:1070D000804677D1EA88F188914273D1A87BB27B50
:1070E00082426FD1B88898426CD1FB888B4269D1BB
:1070F000B97B914266D1E4B2092C69DC0123A3403B
:1071000013F0AA0F41D1092C62D1082966D10F983A
:107110000E2852D039F0B2FE4FF0000A8146109886
:107120000E2841D039F0AAFE034611980E284FF0E0
:10713000000B40D02C4907934FF4906230F0C2FC12
:10714000AA888188914240D1C188EA88079B9142F0
:107150003BD1827B082A3ED1CDE902A35FFA88F3B6
:10716000CDE904B000932846CDF80490F0EE680A0B
:10717000B0EE480A23463A46314608F07FFD0E201D
:1071800013B0BDEC028BBDE8F08F1029BFD01948B9
:107190006BF01CFDF7EE007A77EEC87AF0EE678AA6
:1071A00086E7B6EE008A7CE711980E284FF0010BB7
:1071B0004FF00003BED10020CEE74FF0010A4FF0A0
:1071C0000009ACE70C486BF001FD0C486BF0FEFCCD
:1071D0000B486BF0FBFC0B486BF0F8FC0A486BF0BB
:1071E000F5FC00BFD8D50B00D4E20B00F8E30B0090
:1071F00000D80B00648E0B00FC910B00D48C0B00AC
:10720000A0860B00E88C0B00808E0B002DE9F0436C
:107210002E4B97B00FACCDE90034072330F0BCFA09
:107220002B490F9840F2E32230F04CFC0546052232
:107230000CA9109835F000FFEC88264BAA8811A9FC
:107240000AA800F0F3FB2246234B12A90DF12A00F5
:1072500000F0ECFBBDF92860BDF92A70BDF92C8067
:10726000BDF92E909DF83810A9EB07030022A8EB7A
:107270000604402003FB04F430F0C4FC15990D9B78
:10728000B3FBF0F30E2902461BD0CDE908300846C7
:10729000079139F0F3FDDDE90713099A9C4212D8F2
:1072A0000E3918BF0121049003912846CDE90189C8
:1072B0000C990097334609F023F80E2017B0BDE86B
:1072C000F0830020EAE705486BF000FCD8D40B00FF
:1072D000D4E20B0098D60B0090D60B00447E0B0036
:1072E00013460A46014640F2E5201AF0EFBF00BF00
:1072F00070B52B4B86B002ACCDE90034042330F0DE
:107300004BFA2849039840F2DE5230F0DBFB254966
:10731000054640F27132029830F0D4FB05990446DC
:107320004FF42A7220481AF0E3FF40F2E352049926
:1073300006461E481AF0DCFFAA88A3889A4223D189
:10734000EA88E3889A421FD1A37B102B01D0012B3E
:1073500020D1C2B2092A1ADC0123934013F0AA0FEC
:107360000CD1092A13D1AB7B082B16D12046F3B2DE
:10737000294609F0A1FA0E2006B070BDAB7B102B98
:10738000F4D00B486BF00EFC0A486BF00BFC0A487B
:107390006BF008FC09486BF005FC09486BF002FC37
:1073A00080D40B00D4E20B0054D70B00F8E30B00A1
:1073B000AC770B0000840B00DC750B00B8770B007A
:1073C000A4770B0013460A46014640F2E5201AF066
:1073D0007DBF00BF2DE9F04F394B97B00CACCDE924
:1073E00000340A2330F0D8F936490C9840F2713253
:1073F00030F068FB40F2A2638288044600210E98B8
:1074000030F0CEFA4FF4D563E288002182460F981F
:1074100030F0C6FA2B4940F2DE5283460D9830F028
:1074200051FBC6888288284B054610A90AA800F09F
:10743000FDFA3246254B11A90DF12A0000F0F6FAAB
:10744000A27BAB7BBDF92860BDF92A70BDF92C8009
:10745000BDF92E909A422FD314980E2822D039F0DD
:107460000DFD034615980E284FF0000221D0CDE9FE
:10747000083239F003FDDDE908320021CDE90601CB
:10748000CDE904322046CDE90289CDE900670FFA43
:107490008BF30FFA8AF2294608F0A0FF0E2017B0EE
:1074A000BDE8F08F15980E284FF001024FF0000351
:1074B000DDD101210020E1E705486BF087FB00BF2B
:1074C00008D40B00D4E20B0098D60B0090D60B002A
:1074D000C8770B0000B51E4B89B00DF10C0CCDE93F
:1074E000003C052330F058F940F2713219490398F5
:1074F00030F0E8FA837BDDF818C001229A40944509
:107500001FD2079B6FF000418B4201D09A421BD9DA
:10751000BDF91010002911DB828891420EDABDF905
:107520001420002A0ADBB0F806E0724506DA009360
:10753000634609F0ADF80E2009B000BD06486BF0B7
:1075400045FB06486BF042FB05486BF03FFB00BF74
:1075500068D50B00D4E20B001C790B0098750B006A
:1075600030840B002DE9F0411E4B88B003ACCDE90F
:107570000034052330F010F940F271321A490398B3
:1075800030F0A0FA827B079D012393409D4225D2D3
:10759000BDF91060BDF91470BDF9188082880446E9
:1075A00040F2A2630021304630F0FAF9E2884FF44D
:1075B000D5630021384630F0F3F940F22F52002114
:1075C000404630F0E1F92046009543463A463146C0
:1075D00009F0E4FA0E2008B0BDE8F08103486BF032
:1075E000F5FA00BF58D40B00D4E20B001C790B0055
:1075F00000B5134B89B00DF1080CCDE9003C062312
:1076000030F0CAF80F49029840F2713230F05AFA5D
:10761000827B07990123934099420ED2BDF918C08D
:10762000BDF91430BDF91020CDE900C1BDF90C1031
:1076300009F076FB0E2009B000BD03486BF0C6FAD6
:1076400038D50B00D4E20B001C790B0030B5264B6B
:1076500091B00BACCDE90034052330F09DF82349FF
:107660000B9840F2713230F02DFA052205A905463B
:107670000C9835F0E1FC052208A90D9835F0DCFCEA
:107680009DF81C100022402030F0BCFA9DF8281014
:1076900004460022402030F0B5FA84421AD1069BFD
:1076A000099AB3FBF4F3B2FBF4F2934218D1A87B2E
:1076B0000E990122824091420FD29DF83C20029205
:1076C000CDE900412846089A059909F063FB0E2090
:1076D00011B030BD06486BF079FA06486BF076FAC7
:1076E00005486BF073FA00BF10D50B00D4E20B0015
:1076F00030900B001C790B0044900B0070B51B4BB5
:107700008AB004ACCDE90034062330F045F840F2ED
:1077100071321749049830F0D5F9827B099D012315
:1077200093409D421FD28288124B0446C08805A90F
:10773000064602A800F07AF9324606A90DF10A00C1
:107740000D4B00F073F9BDF90E10BDF90C30BDF909
:107750000A20CDE900152046BDF9081009F0ACFB60
:107760000E200AB070BD05486BF030FA90D50B00C2
:10777000D4E20B0098D60B0090D60B001C790B00BE
:1077800000B5114B87B00DF10C0CCDE9003C032383
:1077900030F002F80D49039840F2E32230F092F9FC
:1077A000827B049901239340994207D2059A9A4219
:1077B00004D209F065FD0E2007B000BD044840F278
:1077C00027316BF00BFA00BFC0D50B00D4E20B00E1
:1077D0005C940B002DE9F0432DED028B5A4BA1B0C8
:1077E00013ACCDE900340D232FF0D6FF5749139881
:1077F00040F2713230F066F940F2DE5204465349ED
:10780000149830F05FF9A27B837B9A42C0F0988095
:10781000054615980E2800F08F8039F02FFB0FFADF
:1078200080F916980E2800F0838039F027FB0FFAB4
:1078300080F819980E2878D039F020FB06B21A98F3
:107840000E286FD039F01AFB07B2189B00930DF188
:107850004203029310AB179901930FAA0DF13E0357
:1078600020466EF0BBF91C9B00930DF14A03029376
:1078700012AB019328461B990DF1460311AA6EF035
:10788000ADF91D980E284AD039F07EFAB0EE408A44
:107890001E980E283BD039F077FAB5EEC00AF1EE0B
:1078A00010FAF0EE400A32D41F980E2834D0CDEDF5
:1078B0000D0A39F0E3FADDED0D0A0023CDE90A03E4
:1078C000BDF94230BDF9402005972046BDF94A4038
:1078D0000994BDF948400894CDE90235BDF9464008
:1078E000BDF93E300794BDF944400496CDE900321D
:1078F000B0EE480ABDF93C3006944246494609F0CC
:10790000EBFC0E2021B0BDEC028BBDE8F0831F988C
:107910000E28F7EE000ACAD101230020CEE79FED22
:107920000C8AB5E7EF887F088FE7AE88760886E790
:10793000E3884FEA53087CE7A3884FEA530970E7CE
:1079400004486BF043F900BF28D60B00D4E20B00CB
:1079500000000000C8770B0000B52E4B8DB00DF174
:10796000140CCDE9003C07232FF016FF2A49059897
:1079700040F2E32230F0A6F8DDF820C00CF1FF332E
:10798000012B20D9BCF1040F40D1079B022B2FDD26
:10799000A3F1040EBEF11C0F2CD8204A012101FADC
:1079A0000EF10A4052B39DF82C109DF82820CDE925
:1079B00001219DF8242000920699624609F0BCFA44
:1079C0000E200DB000BD079B022B11DD1A1F1C2AD3
:1079D00010D812494FF0010E0EFA02FE0EEA010114
:1079E0000029E0D1142A05D1BCF1010FDBD008E059
:1079F000002BD8DC0A4819466BF0F0F8BEF1140FE2
:107A0000F8D10848182261466BF0E8F8064861464C
:107A10006BF0E4F8A0D40B00D4E20B0011100010BE
:107A2000407D0B00307D0B00207D0B00F8B50F462C
:107A30001D46196806461446386830F097F82B68DA
:107A4000002122462FF0ACFF3080B8680E2809D004
:107A5000696830F08BF822466B68B6F900102FF099
:107A60009FFF0446B480F8BD30B585B004461D467E
:107A700002A8094B0191FFF7D9FF0199074B0DF1BE
:107A80000A002A460431FFF7D1FF02AB03CB206086
:107A90002046616005B030BD98D60B0090D60B0033
:107AA0002DE9F0430D4685B0002191464BF0F0F8EA
:107AB0000446002128464BF0EBF82379662B68D06A
:107AC0000379662B054664D0002308208DF80F301B
:107AD0002CF06EFF804608202CF076FF0746082029
:107AE0002CF072FF4346CDE9007006460DF10F02FF
:107AF000294620464AF04CFE00284DD0B9F1040F2B
:107B000056D8DFE809F01A25303B03002046CDE9BE
:107B100000769DF80F202946434601F0B7F8044649
:107B200040462CF043FF38462CF040FF30462CF006
:107B30003DFF204605B0BDE8F0832046CDE9007644
:107B40009DF80F202946434600F03CF80446E7E73D
:107B50002046CDE900769DF80F202946434600F0E7
:107B600017FA0446DCE72046CDE900769DF80F20A1
:107B70002946434600F0F2FB0446D1E72046CDE912
:107B800000769DF80F202946434600F0CDFD0446BF
:107B9000C6E708486BF01AF840462CF007FF384655
:107BA0002CF004FF30462CF001FF03486BF00EF878
:107BB0000024B5E7847A0B00C0790B000022FFF7A0
:107BC0006FBF00BF2DE9F043074610463A7983B0F6
:107BD0008C46622A19460A9D0B9EFB69DCF81C4004
:107BE0005ED019D8422A2CD0482A11D19CF804E042
:107BF000BEF1480F00F00C81BEF1680F00F02D813E
:107C0000BEF1620F55D003D8BEF1420F00F0828062
:107C1000002003B0BDE8F083682AF9D19CF8042065
:107C2000682A00F04081622A43D0F1D89946B046D4
:107C3000BE46422A23462E4667464C464546F446F3
:107C4000D2D19CF80420622A00F095806AD8422A9A
:107C50003BD0482ADCD101934DF054FB019BD0F876
:107C60001CC04FF0000E002127881A783A402CF8EB
:107C7000022B0269D5F80480776801318A424344B7
:107C80003C44F1D8296802FB18110B44316802FB0F
:107C90001711C2680EF1010E72450C44E3D8B8E723
:107CA000A046AE4662461C463546BC46434676462E
:107CB00017463A79622A00F01B81482A00F03D817C
:107CC000682A7FD0622A8DD9A2E701934DF01AFB72
:107CD000019BD0F81CC04FF0000E002127781A78C5
:107CE0003A400CF8012B0269D5F80480776801311D
:107CF0008A4243443C44F1D8296802FB18110B44E2
:107D0000316802FB1711C2680EF1010E72450C4476
:107D1000E3D87EE7B6461A462E462346BC4675464D
:107D200014468EE7682A7FF473AF01934DF0EAFAA8
:107D3000019BD0F81CE000270021B4F800C01A789D
:107D400002EA0C022EF8022B0269D5F80480D6F85C
:107D500004C001318A4243446444EED8296802FBDE
:107D600018110B44316802FB1C11C2680137BA427A
:107D70000C44E1D84DE7682201934DF0C3FA019B12
:107D8000D0F81CC04FF0000E002194F900701A7852
:107D90003A402CF8022B0269D5F80480776801314B
:107DA0008A4243443C44F0D8296802FB18110B4432
:107DB000316802FB1711C2680EF1010E72450C44C6
:107DC000E2D826E701934DF09DFA019BD0F81CC044
:107DD0004FF0000E00211F8894F900203A402CF843
:107DE000022B0269D6F804806F6801318A4244444C
:107DF0003B44F0D8316802FB18110C44296802FB9F
:107E00001711C2680EF1010E72450B44E2D800E76B
:107E100001934DF077FA019BD0F81CC04FF0000E93
:107E2000002127881A883A402CF8022B0269D5F8DD
:107E30000480776801318A4243443C44F1D8296880
:107E400002FB18110B44316802FB1711C2680EF1D6
:107E5000010E72450C44E3D8DBE6724601934DF007
:107E600051FA019BD0F81CC04FF0000E002127886A
:107E70001A883A402CF8022B0269D5F804807768FA
:107E800001318A4243443C44F1D8296802FB18116D
:107E90000B44316802FB1711C2680EF1010E7245E6
:107EA0000C44E3D8B5E601934DF02CFA019BD0F8D1
:107EB0001CC04FF0000E002127881A883A402CF889
:107EC000022B0269D5F80480776801318A42434465
:107ED0003C44F1D8296802FB18110B44316802FBBD
:107EE0001711C2680EF1010E72450C44E3D890E6FA
:107EF00001934DF007FA019BD0F81CC04FF0000E23
:107F000000211F7822783A400CF8012B0269D6F83C
:107F100004806F6801318A4244443B44F1D831689F
:107F200002FB18110C44296802FB1711C2680EF1FC
:107F3000010E72450B44E3D86BE601934DF0E2F974
:107F4000019BD0F81CC04FF0000E00211F8894F94F
:107F500000203A402CF8022B0269D6F804806F68A2
:107F600001318A4244443B44F0D8316802FB181185
:107F70000C44296802FB1711C2680EF1010E72450C
:107F80000B44E2D845E600BF0122FFF789BD00BFE0
:107F90002DE9F043074610463A7983B08C46622AB1
:107FA00019460A9D0B9EFB69DCF81C405ED019D86F
:107FB000422A2CD0482A11D19CF804E0BEF1480F87
:107FC00000F00C81BEF1680F00F02D81BEF1620F50
:107FD00055D003D8BEF1420F00F08280002003B0DC
:107FE000BDE8F083682AF9D19CF80420682A00F0E3
:107FF0004081622A43D0F1D89946B046BE46422A13
:1080000023462E4667464C464546F446D2D19CF858
:108010000420622A00F095806AD8422A3BD0482A80
:10802000DCD101934DF06EF9019BD0F81CC04FF0EC
:10803000000E002127881A783A432CF8022B026997
:10804000D5F80480776801318A4243443C44F1D832
:10805000296802FB18110B44316802FB1711C26832
:108060000EF1010E72450C44E3D8B8E7A046AE46C7
:1080700062461C463546BC464346764617463A7924
:10808000622A00F01B81482A00F03D81682A7FD0D7
:10809000622A8DD9A2E701934DF034F9019BD0F803
:1080A0001CC04FF0000E002127781A783A430CF8D4
:1080B000012B0269D5F80480776801318A42434474
:1080C0003C44F1D8296802FB18110B44316802FBCB
:1080D0001711C2680EF1010E72450C44E3D87EE719
:1080E000B6461A462E462346BC46754614468EE7CB
:1080F000682A7FF473AF01934DF004F9019BD0F827
:108100001CE000270021B4F800C01A7842EA0C02F3
:108110002EF8022B0269D5F80480D6F804C001318C
:108120008A4243446444EED8296802FB18110B4488
:10813000316802FB1C11C2680137BA420C44E1D815
:108140004DE7682201934DF0DDF8019BD0F81CC08B
:108150004FF0000E002194F900701A783A432CF881
:10816000022B0269D5F80480776801318A424344C2
:108170003C44F0D8296802FB18110B44316802FB1B
:108180001711C2680EF1010E72450C44E2D826E7C1
:1081900001934DF0B7F8019BD0F81CC04FF0000ED2
:1081A00000211F8894F900203A432CF8022B026921
:1081B000D6F804806F6801318A4244443B44F0D8C9
:1081C000316802FB18110C44296802FB1711C268C0
:1081D0000EF1010E72450B44E2D800E701934DF019
:1081E00091F8019BD0F81CC04FF0000E00212788A9
:1081F0001A883A432CF8022B0269D5F80480776874
:1082000001318A4243443C44F1D8296802FB1811E9
:108210000B44316802FB1711C2680EF1010E724562
:108220000C44E3D8DBE6724601934DF06BF8019BFA
:10823000D0F81CC04FF0000E002127881A883A435E
:108240002CF8022B0269D5F80480776801318A4244
:1082500043443C44F1D8296802FB18110B443168AF
:1082600002FB1711C2680EF1010E72450C44E3D8EF
:10827000B5E601934DF046F8019BD0F81CC04FF0D5
:10828000000E002127881A883A432CF8022B026935
:10829000D5F80480776801318A4243443C44F1D8E0
:1082A000296802FB18110B44316802FB1711C268E0
:1082B0000EF1010E72450C44E3D890E601934DF0A7
:1082C00021F8019BD0F81CC04FF0000E00211F7850
:1082D00022783A430CF8012B0269D6F804806F68C3
:1082E00001318A4244443B44F1D8316802FB181101
:1082F0000C44296802FB1711C2680EF1010E724589
:108300000B44E3D86BE601934CF0FCFF019BD0F8E3
:108310001CC04FF0000E00211F8894F900203A4342
:108320002CF8022B0269D6F804806F6801318A426A
:1083300044443B44F0D8316802FB18110C442968CE
:1083400002FB1711C2680EF1010E72450B44E2D810
:1083500045E600BF0222FFF7A3BB00BF2DE9F043B3
:10836000074610463A7983B08C46622A19460A9D20
:108370000B9EFB69DCF81C405ED019D8422A2CD039
:10838000482A11D19CF804E0BEF1480F00F00C819E
:10839000BEF1680F00F02D81BEF1620F55D003D8F9
:1083A000BEF1420F00F08280002003B0BDE8F083F0
:1083B000682AF9D19CF80420682A00F04081622ADA
:1083C00043D0F1D89946B046BE46422A23462E46AF
:1083D00067464C464546F446D2D19CF80420622AB2
:1083E00000F095806AD8422A3BD0482ADCD101931C
:1083F0004CF088FF019BD0F81CC04FF0000E00210C
:1084000027881A787A402CF8022B0269D5F8048064
:10841000776801318A4243443C44F1D8296802FB21
:1084200018110B44316802FB1711C2680EF1010EDE
:1084300072450C44E3D8B8E7A046AE4662461C46F7
:108440003546BC464346764617463A79622A00F0DE
:108450001B81482A00F03D81682A7FD0622A8DD98D
:10846000A2E701934CF04EFF019BD0F81CC04FF0E7
:10847000000E002127781A787A400CF8012B026947
:10848000D5F80480776801318A4243443C44F1D8EE
:10849000296802FB18110B44316802FB1711C268EE
:1084A0000EF1010E72450C44E3D87EE7B6461A463B
:1084B0002E462346BC46754614468EE7682A7FF44E
:1084C00073AF01934CF01EFF019BD0F81CE0002716
:1084D0000021B4F800C01A7882EA0C022EF8022BB0
:1084E0000269D5F80480D6F804C001318A424344B9
:1084F0006444EED8296802FB18110B44316802FB72
:108500001C11C2680137BA420C44E1D84DE7682219
:1085100001934CF0F7FE019BD0F81CC04FF0000E09
:10852000002194F900701A787A402CF8022B026925
:10853000D5F80480776801318A4243443C44F0D83E
:10854000296802FB18110B44316802FB1711C2683D
:108550000EF1010E72450C44E2D826E701934CF06F
:10856000D1FE019BD0F81CC04FF0000E00211F88E7
:1085700094F900207A402CF8022B0269D6F8048086
:108580006F6801318A4244443B44F0D8316802FBB1
:1085900018110C44296802FB1711C2680EF1010E74
:1085A00072450B44E2D800E701934CF0ABFE019B0F
:1085B000D0F81CC04FF0000E002127881A887A409E
:1085C0002CF8022B0269D5F80480776801318A42C1
:1085D00043443C44F1D8296802FB18110B4431682C
:1085E00002FB1711C2680EF1010E72450C44E3D86C
:1085F000DBE6724601934CF085FE019BD0F81CC06F
:108600004FF0000E002127881A887A402CF8022BA0
:108610000269D5F80480776801318A4243443C44BA
:10862000F1D8296802FB18110B44316802FB1711BD
:10863000C2680EF1010E72450C44E3D8B5E6019311
:108640004CF060FE019BD0F81CC04FF0000E0021E2
:1086500027881A887A402CF8022B0269D5F8048002
:10866000776801318A4243443C44F1D8296802FBCF
:1086700018110B44316802FB1711C2680EF1010E8C
:1086800072450C44E3D890E601934CF03BFE019B0D
:10869000D0F81CC04FF0000E00211F7822787A40DD
:1086A0000CF8012B0269D6F804806F6801318A4208
:1086B00044443B44F1D8316802FB18110C4429684A
:1086C00002FB1711C2680EF1010E72450B44E3D88C
:1086D0006BE601934CF016FE019BD0F81CC04FF0E6
:1086E000000E00211F8894F900207A402CF8022BFC
:1086F0000269D6F804806F6801318A4244443B44E1
:10870000F0D8316802FB18110C44296802FB1711DC
:10871000C2680EF1010E72450B44E2D845E600BF77
:108720000322FFF7BDB900BF2DE9F04117460279DA
:10873000CC6982B0622A9C46089DC369099E6ED0AE
:1087400038D8422A00F0A380482A40F09C8009795A
:108750000193422900F03E81622900F044824829B9
:1087600000F083816146384668224CF0CBFD019BC6
:10877000D0F81CC04FF0000E0021B4F900701A8828
:10878000BA402CF8022B0269D5F8048077680131D1
:108790008A4243443C44F0D8296802FB18110B4438
:1087A000316802FB1711C2680EF1010E72450C44CC
:1087B000E2D869E0682A66D109790193422900F07C
:1087C0009880622900F0C18148293846614600F04E
:1087D00027814CF097FD019BD0F81CE00027002179
:1087E000B4F900C0B3F9002002FA0CF22EF8022B03
:1087F0000269D5F80480D6F804C001318A424344A6
:108800006444EDD8296802FB18110B44316802FB5F
:108810001C11C2680137BA420C44E0D834E00A792E
:108820000193422A6146384600F08A80622A00F0AD
:10883000B481482A00F0408168224CF063FD019B1E
:10884000D0F81CC04FF0000E0021B4F9007093F96D
:108850000020BA402CF8022B0269D5F80480776812
:1088600001318A4243443C44EFD8296802FB181185
:108870000B44316802FB1711C2680EF1010E7245FC
:108880000C44E1D800E0002002B0BDE8F0810A7994
:108890000193422A6146384678D0622A00F0CC81A2
:1088A000482A00F02E8168224CF02CFD019BD0F864
:1088B0001CC04FF0000E0021B4F900701A78BA40C5
:1088C0002CF8022B0269D5F80480776801318A42BE
:1088D00043443C44F0D8296802FB18110B4431682A
:1088E00002FB1711C2680EF1010E72450C44E2D86A
:1088F000CAE7614638464CF005FD019BD0F81CC024
:108900004FF0000E00212778B3F90020BA402CF870
:10891000022B0269D5F80480776801318A4243440A
:108920003C44F0D8296802FB18110B44316802FB63
:108930001711C2680EF1010E72450C44E2D8A3E78C
:1089400068224CF0DFFC019BD0F81CC04FF0000EF9
:108950000021277893F90020BA402CF8022B0269F5
:10896000D5F80480776801318A4243443C44F0D80A
:10897000296802FB18110B44316802FB1711C26809
:108980000EF1010E72450C44E2D87DE74CF0BAFCC2
:10899000019BD0F81CC04FF0000E002127781A78F8
:1089A000BA400CF8012B0269D5F8048077680131D0
:1089B0008A4243443C44F1D8296802FB18110B4415
:1089C000316802FB1711C2680EF1010E72450C44AA
:1089D000E3D859E7614638464CF094FC019BD0F847
:1089E0001CC04FF0000E002127781A88BA402CF8DE
:1089F000022B0269D5F80480776801318A4243442A
:108A00003C44F1D8296802FB18110B44316802FB81
:108A10001711C2680EF1010E72450C44E3D833E71A
:108A20004CF070FC019BD0F81CC04FF0000E0021F0
:108A3000B4F900701A88BA402CF8022B0269D5F8F4
:108A40000480776801318A4243443C44F0D8296865
:108A500002FB18110B44316802FB1711C2680EF1BA
:108A6000010E72450C44E2D80EE70A4638466146CC
:108A70004CF048FC019BD0F81CC04FF0000E0021C8
:108A800027881A88BA402CF8022B0269D5F804808E
:108A9000776801318A4243443C44F1D8296802FB9B
:108AA00018110B44316802FB1711C2680EF1010E58
:108AB00072450C44E3D8E7E64CF024FC019BD0F867
:108AC0001CC04FF0000E0021278893F90020BA4007
:108AD0002CF8022B0269D5F80480776801318A42AC
:108AE00043443C44F0D8296802FB18110B44316818
:108AF00002FB1711C2680EF1010E72450C44E2D858
:108B0000C2E64CF0FFFB019BD0F81CC04FF0000EFA
